:020000021000EC
:10F00000F0FF002039F5010061F5010063F5010012
:10F0100065F5010067F5010069F5010000000000D9
:10F020000000000000000000000000006BF501007F
:10F030006DF50100000000006FF501009519040056
:10F040004154020073F5010035560200A15402003C
:10F05000ED54020091660200E557020073F50100CD
:10F0600073F50100D919040073F5010073F501006F
:10F0700073F501005161020073F5010073F50100A1
:10F08000D51904000D2D020073F5010073F5010080
:10F09000152E020069DD0300911E020073F50100C8
:10F0A00073F5010073F5010073F50100F1680200CA
:10F0B00073F5010073F5010000000000000000007E
:10F0C00073F5010073F5010073F5010073F501009C
:10F0D00073F501001D63020073F5010000000000DC
:10F0E0000000000000000000000000000000000020
:10F0F0000000000000000000000000000000000010
:10F1000000000000000000000000000000000000FF
:10F1100000000000000000000000000000000000EF
:10F4000010B5054C237833B9044B13B10448AFF35E
:10F4100000800123237010BD202E0020000000007A
:10F42000C05F060008B5034B1BB103490348AFF3A7
:10F43000008008BD00000000242E0020C05F0600F0
:10F44000154B002B08BF134B9D46A3F5803A0021B6
:10F450008B460F461348144A121A00F063F80F4BFC
:10F46000002B00D098470E4B002B00D0984700206F
:10F47000002104000D000D48002802D00C48AFF315
:10F48000008000F02BF82000290025F05BF900F047
:10F4900011F800BF00000800F0FF0020000000008D
:10F4A00000000000202E002084D00020000000007A
:10F4B0000000000008B5074B044613B10021AFF36C
:10F4C0000080054B1868836A03B19847204600F016
:10F4D00031F800BF0000000054AE050070B50D4DBE
:10F4E0000D4C641BA4100026A64209D10B4D0C4CF8
:10F4F0003BF0A4FC641BA4100026A64205D170BDFD
:10F5000055F8043B98470136EEE755F8043B984719
:10F510000136F2E7042E0020042E0020042E0020E5
:10F52000082E002002440346934200D1704703F89E
:10F53000011BF9E7FEE700BF0649074A074B9B1A84
:10F5400003DD043BC858D050FBDC06F0D5FFFFF7C5
:10F5500077FF0000CC5F0600402C0020202E00200A
:10F56000FEE7FEE7FEE7FEE7FEE7FEE7FEE7FEE773
:10F57000FEE7FEE71FB501238DF80030054B8DF83F
:10F58000080001916846D3E90012904705B05DF884
:10F5900004FB00BF20BB002061DF704748DF7047DD
:10F5A00010B50388012B11D8094A02EB03124388D6
:10F5B0005189CC1A032C09D4C3F57F43FD330B4486
:10F5C0005381002303804380184610BD0420FCE7CC
:10F5D00020C0002010B5124A0B6802EB00104268F0
:10F5E00073B15888033003EB800302F580524FF665
:10F5F000FF749A4202D91868013004D1002009E052
:10F6000002F10803F1E79888A04204D0188810B1ED
:10F610000B60012010BD5888033003EB8003E8E73E
:10F6200020C0002073B5436804460D4613B31E4A3C
:10F6300011688B421ED3526893421BD813F003000B
:10F6400018D11A4A21891289914213D121689A68E6
:10F6500091420FD1164A5268934201D80A2004E021
:10F6600002F580529342F9D22880B0FA80F0400926
:10F6700002B070BD00232B801E46019601A9288888
:10F68000FFF7A8FF30B92B8801339BB22B80002BEA
:10F69000F3D0EDE7019B226899689142EED1636057
:10F6A000024B1B892381E3E70C2E0020E4BC0020E1
:10F6B00020C00020033083B240F2FD32934230B5C7
:10F6C0000ED909200BE0228965892A441A4492B296
:10F6D000B2F5806F08D2088062891344638130BD1F
:10F6E000024C20780028EED00720F8E720C0002048
:10F6F00010B50A494A788C78531CDBB29C4208BF8B
:10F7000000230C789C421FBF0370486802EB420242
:10F7100000EBC20008BF002010BD00BF9CBF00204E
:10F72000AADF7047A9DF7047A7DF704785DF704702
:10F730007FDF70477EDF7047084A30B500230C2416
:10F7400004FB03F18D5A854202D10A44508830BD32
:10F750000133082BF4D14FF6FF70F8E74EBC0020C0
:10F760006EDF7047012804D0043804288CBF0020C5
:10F77000012070478378013B072B07D8DFE803F0AF
:10F7800007060606060704091423038070470123B1
:10F79000FBE743689B8809339B08F6E770B5054D86
:10F7A0000646002455F8043B304601349847052CA2
:10F7B000F8D170BD14B00500114BF0B5002214262D
:10F7C0001D4606FB02F4E75A874212D12344142651
:10F7D00000249A788A420AD001342246072A0BD89C
:10F7E00006FB02F3EF5A874208D1EB18F1D1184615
:10F7F000F0BD0132082AE4D10023F8E70132EDE739
:10F80000BCC10020F8B5074D074E074600243378E9
:10F81000A34200DCF8BD55F8043B38469847013454
:10F82000F5E700BFC0BC002071BE00207DDF70473F
:10F8300079DF70476DDF704758B1CB0801F00701E1
:10F84000C25C012303FA01F10A4214BF18460020EA
:10F85000704701207047000070B50A4E34680546B5
:10F8600054B1706860B1FF2D08D02946FFF7E4FF5E
:10F8700030B1F36803FB0544204670BD0024FBE76C
:10F880000446F9E7ACC1002030B5072185B0FFF789
:10F8900093FF044600283AD04568002D39D1007CFA
:10F8A000FFF7DAFF0721CDE902558DF80A1040B3C2
:10F8B000E368039003EB83031B019BB29B0802A840
:10F8C000ADF80830FFF756FF9DF80A00FFF74AFF32
:10F8D000D8B1114B1B789B0715D5BDF808500DF119
:10F8E00006012846FFF7E6FE48B9BDF80630A380BA
:10F8F000E5800A4B185C092803D005B030BD092803
:10F90000F7D90320F9E70220F3E70846F5E70520D9
:10F91000F3E70020F1E700BFE1BC002070AE050076
:10F9200038B54FF6FF73984218BF01300D4614BF2B
:10F9300084B20024FF2C03D94FF6FF74204638BD53
:10F9400021462846FFF778FF0028F7D10134A4B2FA
:10F95000F0E7000038B5074C051E04F1080318BF96
:10F960001C4623682BB11A6822605B6828469847BA
:10F97000F7E738BDF8BB002040DF70473FDF704736
:10F980000023435082B043580193019B02B070475B
:10F990002DE9F0470D789DF820609DF824A00446DD
:10F9A0000F469946002D60D1D0F8243192F800809E
:10F9B0009BB14FF49271FFF7E3FF012363613B704A
:10F9C000B04550D1D4F80431002B4CD04FF48271A3
:10F9D0002046FFF7D5FF00251DE0D0F81C31FBB114
:10F9E0004FF48E71FFF7CCFFD0F824311BB14FF4E8
:10F9F00092712046DFE713789E4207D919F8033049
:10FA0000C0F81C35137801331370D9E70123BAF11C
:10FA1000000F03D0C3612846BDE8F0874361CFE7FC
:10FA2000D0F80831002BCBD04FF48471FFF7A8FF3A
:10FA3000D0F82431002BDAD113789E42C0D9D0F807
:10FA4000181509F8031013780133DBB21370721E16
:10FA5000934205D10223C0F8003201232362AFE7AD
:10FA60009E42FAD1ACE70125D5E74FF49271FFF73A
:10FA700087FF4FF48E71FFF783FF4FF48471FFF718
:10FA80007FFF9FE72DE9F3470C4605464FF482714F
:10FA900020461F469046FFF773FF4FF49271FFF721
:10FAA0006FFF4FF48E71FFF76BFF4FF48471FFF718
:10FAB00067FF0023012F85F8263085F8233008BF23
:10FAC00002224FF001030CBFC4F80022C4F8003238
:10FAD000236223602E6846BB05F1260A05F123093F
:10FAE000CDE900764346524649462046FFF750FF8F
:10FAF0000028F5D195F82330EBB1D4F8C434C4F81C
:10FB0000C434C3B113F0010F14BF4FF402400320FB
:10FB100048F2012213F0020F18BF104613F0040F31
:10FB200048F2022318BF184606E040F28623AB6075
:10FB3000AB68C4F80433002002B0BDE8F0872DE9BB
:10FB4000F3470C4605464FF4827120461F46164681
:10FB50009DF82880FFF714FF4FF49271FFF710FF14
:10FB60004FF48E71FFF70CFF4FF48471FFF708FF1D
:10FB70000023C4F8003285F8263085F823300123AD
:10FB80002362A36095F82620974232D9B35CC4F86B
:10FB90001C3595F82630013385F826302B687BBB61
:10FBA00005F1260A05F12309CDE9007833465246CE
:10FBB00049462046FFF7ECFE0028F5D195F82330A2
:10FBC00023B3D4F8C434C4F8C434FBB113F0010F28
:10FBD00014BF4FF40240032048F2012213F0020F39
:10FBE00018BF104613F0040F48F2022318BF18463E
:10FBF0000DE0B8F1000F01D0E361CFE76361CDE71D
:10FC000040F28623AB60AB68C4F80433002002B036
:10FC1000BDE8F0870023435082B043580193019B15
:10FC200002B0704708B502464FF492710068FFF7C2
:10FC3000F1FF4FF484711068FFF7ECFF13680122A5
:10FC40001A6008BD10B5CB7D0A464FF4847123B904
:10FC5000FFF7E0FFD0F8183510BDFFF7DBFF537E4C
:10FC6000D168D0F81805C854537E0133DBB25376FF
:10FC7000F2E70A4610B54FF48E71FFF7CBFF938A77
:10FC800091689BB2C95C938A01339BB29382C0F89E
:10FC90001C1510BD2DE9F04793F9005090B00024D9
:10FCA000013D6E46AD002746A446A0465FF0000E1B
:10FCB00003E05FEA080EBEEB050EB8EB0E0952F842
:10FCC00009A051F80E90A9FB0A9A14EB090457EB0E
:10FCD0000A075CF1000C1EF1040EAE4501DCC645BE
:10FCE000EBDD46F808403C4667465FF0000C18F133
:10FCF0000408A845DADDB8EB450FDADD46F8084020
:10FD0000D3F8B0303146984710B0BDE8F0871346BD
:10FD10000A46FFF7BFBFF0B5154689B01C46074637
:10FD20000E461A4629466846FFF7F1FF23466A4603
:10FD300039463846FFF7AEFF23462A4669466846ED
:10FD4000FFF7A8FF23466A4631463046FFF7A2FF79
:10FD500009B0F0BD00EB81010023884200D3704759
:10FD600051F8042D43EA52030B60D307F5E710B5B1
:10FD7000013A52B2130601D5002010BD50F82240BE
:10FD800051F822309C4205D802F1FF32F2D24FF0F6
:10FD9000FF30F2E70120F0E710B500235CB2A24289
:10FDA00000DC10BD51F8234040F823400133F5E753
:10FDB000013910B549B2041D0A06CBB204D4013989
:10FDC00054F82120002AF7D001335BB273B103F15C
:10FDD0008042013A50F82220002022B9013B00EB7A
:10FDE000431318B210BD52080130F6E71846F9E780
:10FDF000002310B51C465AB2914200DC10BD40F8F9
:10FE000023400133F7E7000000000000000000007D
:10FE1000C3F10803DB0070B50133002403A500BF64
:10FE20005B1920C940CAAD1B20C0184720C940CA71
:10FE3000B54120C020C940CAB54120C020C940CA30
:10FE4000B54120C020C940CAB54120C020C940CA20
:10FE5000B54120C020C940CAB54120C020C940CA10
:10FE6000B54120C06441B4FA84F0400970BD00BFC0
:10FE7000C3F10803DB0070B50133002403A500BF04
:10FE80005B1920C940CAAD1920C0184720C940CA13
:10FE9000754120C020C940CA754120C020C940CA50
:10FEA000754120C020C940CA754120C020C940CA40
:10FEB000754120C020C940CA754120C020C940CA30
:10FEC000754120C06441204670BD00BFF0B50822D6
:10FED00089B00C460646FFF75FFFCB6A03930B6BB6
:10FEE00004934B6B05938B6B0693CB6B07930027A7
:10FEF00008236A4669466846CDE901770097FFF70F
:10FF0000B7FF082305466A4631463046FFF7B0FF83
:10FF1000236B0393636B0493A36B0593E36B05441B
:10FF2000CDE906376A46082369466846FFF7A0FF11
:10FF3000082305446A4631463046FFF799FF236A95
:10FF40000093636A0193A36A0293A36B0693E36B26
:10FF50000793054408236A4631463046CDE90477C5
:10FF60000397FFF785FF636A0093A36AA26B01936F
:10FF7000E36A02930492636BE26B0393CDE905237A
:10FF8000236A0793054408236A4631463046FFF743
:10FF90006FFFE36A0093236B0193636B0293236A01
:10FFA0000693A36A0793054408236A463146304600
:10FFB000CDE904770397FFF72BFF236B0093636B67
:10FFC0000193A36B0293E36B0393636A0693E36A63
:10FFD00007932D1A08236A4631463046CDE9047747
:10FFE000FFF716FF636B0093A36B0193E36B029320
:10FFF000236A0393636A0493A36ACDE90537236BED
:020000022000DC
:1000000007932D1A08236A4631463046FFF700FF52
:10001000A36B0093E36BCDE90137636A0393A36A93
:100020000493E36ACDE90537636B07932D1A082320
:100030006A4631463046FFF7EBFE2D1A0D4C0FD4C1
:1000400035B9082231462046FFF791FE01280FD02E
:100050000823224631463046FFF7DAFE2D1AEFE735
:100060000823224631463046FFF702FF2D18F7D409
:1000700009B0F0BD88AE05002DE9F04391B00F4600
:100080001C220021804609A8FFF74CFA01251C22FA
:10009000002101A80895FFF745FA394608AA11F989
:1000A000046B009533461046FFF7E2FE314608A880
:1000B000FFF77EFE013804B2012C07DC32466946A8
:1000C0004046FFF769FE11B0BDE8F0833A46684646
:1000D0006946FFF71CFE10AB601103EB80001FFAAE
:1000E00084F909F01F0350F8202C05FA03F313429A
:1000F00005D03B46424669466846FFF7CBFD09F10D
:10010000FF3424B2D8E770B5036813F00105064642
:10011000144605D013460A460146FFF7A9FE0546D8
:1001200021463046FFF716FE45B104F18042013A00
:1001300056F8223043F0004346F8223070BD70B5C7
:100140009DF910401E4623460546FFF761FE38B173
:100150002346324629462846BDE87040FFF788BE50
:1001600070BD2DE9F0438BB01446129D15F9046B58
:1001700000961F46804689462B460246214602A825
:10018000FFF7DDFF02A9129A0846FFF7C0FD129B98
:1001900002AA41464046FFF77DFD129B02AA214676
:1001A0002046FFF777FD2B464A46394638460096EB
:1001B000FFF7C5FF129A394602A8FFF7A8FD02A96A
:1001C0002B46424608460096FFF7B9FF02A92B4688
:1001D000224608460096FFF7B2FF2B4642462146CC
:1001E00020460096FFF7ABFF129B22464946484641
:1001F000FFF750FD2B4602AA414620460096FFF726
:100200009EFF129B224639463846FFF743FD2B4698
:100210004A46394638460096FFF791FF324602A912
:100220002046FFF7B9FD0BB0BDE8F08370B59DF92E
:1002300010401E4623460546FFF71AFE30B92246F7
:1002400029463046FFF793FD012807D02346324662
:1002500029462846BDE87040FFF7DABD70BD2DE99C
:10026000F0439BB01646229C14F9045B0095984617
:100270000746894623460246314612A8FFF75FFF2C
:1002800012A9229A0846FFF742FD229B12AA39467C
:100290003846FFF7FFFC229B12AA31463046FFF793
:1002A000F9FC23464A46414612A80095FFF7BEFFD7
:1002B00023464A46414640460095FFF740FF234605
:1002C0003A4631460AA80095FFF739FF229B0AAA51
:1002D00049464846FFF7DEFC2346324639460AA81F
:1002E0000095FFF7A3FF229A41463046FFF70FFD26
:1002F00023460AAA314630460095FFF720FF2346E1
:100300003246394602A80095FFF719FF229B02AA40
:1003100041464046FFF7BEFC23464A46414640461A
:100320000095FFF70CFF229A12A902A8FFF7EFFC35
:1003300002A923460AAA08460095FFF700FF2346B4
:100340003A4602A90AA80095FFF7F9FE0AA9229BDE
:1003500012AA0846FFF79EFC23464A460AA94846C9
:100360000095FFF7ECFE2A4602A93846FFF714FD78
:100370001BB0BDE8F0832DE9F04115468AB0044674
:1003800088461C22002103A8FFF7CCF82E1D95F902
:10039000007003232A46414620460293FFF7B7FC2C
:1003A000334602AA214620460097FFF7C8FE2B4697
:1003B000424621462046FFF76DFC0097334605F183
:1003C000840221462046FFF731FF0AB0BDE8F081E4
:1003D0000C4B1B78062B10D10B4B1B681A070CD14A
:1003E0000A4B186800F0F003302B08D000F0E00052
:1003F000A0F1400358425841704700207047012047
:10040000704700BFE00F00F0E40F00F0E80F00F0CD
:10041000094B1B78062B0CD1084B1B681A0708D117
:10042000074B186800F0F000A0F130035842584123
:1004300070470020704700BFE00F00F0E40F00F0AD
:10044000E80F00F010B9024B01221A60704700BF9C
:100450000050004010B50C494A6E042A044611D0E1
:100460000B6E1344032B02F101024A6688BF043B62
:10047000182202FB031318460021FFF753F82060EF
:10048000012010BD0020FCE7C0C0002010B50446CC
:1004900086B01422002101A8FFF744F86088ADF867
:1004A0000800FFF749F92378ADF80600092B0CD8AE
:1004B000DFE803F005051014161B1D0E1F2107238E
:1004C0008DF8043008238DF80C3001A8FFF79AF955
:1004D00006B010BD0D238DF80430F6E70E23FAE7C1
:1004E00007238DF804300523EDE70F23F3E71023EE
:1004F000F1E70523EFE706238DF80430A3680393A3
:10050000A388ADF80630E0E72DE9F041067904460E
:10051000407B174603360023834204DB51B93E601B
:100520000020BDE8F081226912F833200132164420
:100530000133F1E73B68B34229D3237833F0030852
:1005400027D10B7022794A708D1C2846A1683AF099
:100550000DFC2279617BA954AB180133627B4245C3
:10056000DDDD226912F8382003F8012B226902EB45
:10057000C801184612F8382049683AF0F7FB22699A
:1005800012F838200346134408F10108E6E7042076
:10059000C7E70720C5E738B504461546084631B118
:1005A00062682B68934206D321683AF0DFFB6368E8
:1005B0002B60002038BD0420FCE708B5134644F248
:1005C0000102904203BF5A681988986800221BF004
:1005D000C3FF000030B50B4B1B68012293F850108D
:1005E0000D338A4204DB405CB0FA80F0400930BD34
:1005F00013F8014B855CA54201D10132F1E70020DF
:10060000F5E700BF60BA002003681A78302A27D1C6
:100610005A1C02605A7802F0DF024F2A03D10233DB
:10062000036008207047582A03D10233036010206A
:100630007047422A04D0082013F8012F22B97047CE
:1006400002330360022070472E2A07D0A2F138013E
:10065000012903D9303A092AEED970470A20EBE77D
:100660000A20704770B5244B0022C3F80025234AA6
:10067000516831B12249C3F8081322490420C1F856
:100680008000D3F80C55D3F81445D3F80815D3F8E7
:1006900010054FF0FF36B542C3F8146518BF05F5D5
:1006A000E075C3F80C65C3F80865C3F810651EBF94
:1006B0004FF0A043022643F82560651C1FBF4FF092
:1006C000A04304F5E074022543F82450441C1FBFE6
:1006D00000F5E0704FF0A043022443F820404B1C8B
:1006E0001FBF4FF0A04301F5E071022043F8210045
:1006F0000023D376536070BD0020004020BB002053
:100700008402020000E100E070B58AB00C460146A8
:1007100068461E462CF0F9FF0022214605A82CF061
:10072000F4FF68462CF0DFFE044605A82CF0DBFE43
:10073000844205460DD0039832F06CFB089832F0E5
:1007400069FB002C01DB002D00DA56B9601B0AB0F2
:1007500070BD002C07DA039832F05CFB089832F089
:1007600059FB0020F3E768462CF075FC05A82CF037
:1007700072FCD6E7044A138A9BB223F0410343F08C
:1007800040031382704700BF482E00200000000085
:100790002DE9F04F85B08A460390039C25782846C2
:1007A0002CF0B0FA0746C8B92D2D1AD10134012317
:1007B00003940193DDF80CB0BAF1000F01D0CAF830
:1007C00000B003A8FFF720FF8046002835D1624D16
:1007D00000242046294605B0BDE8F08F013403947B
:1007E000DBE72B2D04BF013403940190E2E71846A8
:1007F00002932CF055FAB0F10009029B20DBC845AA
:100800001EDD404639F034FD22462B4639F09AFD74
:1008100004460D46484639F02BFD22462B4639F05A
:10082000DBFB013604460D460396039E3378002B0E
:10083000DDD1B8F10A0F37D113E000240025F4E729
:10084000B8F10A0F30D12E2B0BD10FF20419D9E9D0
:10085000008901360396039E30783038C3B2092BE5
:1008600039D9039B1A7802F0DF02452A1CD15A1CA1
:1008700003925A782D2A01D02B2A05D12D3A5742BE
:1008800003F10203574103934FF000080A20039A33
:100890001378303BD9B2092936D9002F39D12F4FDF
:1008A0000026B8F1000F46D1039BBAF1000F01D02A
:1008B000CAF800309B458AD09BF800202E2A03D12D
:1008C0000BF1010B5B4582D0019B002B81D005F120
:1008D00000431D467DE739F0CBFC42464B4639F0DC
:1008E00031FD02460B462046294639F075FB0022B1
:1008F00004460D4640464946184B39F04DFE013638
:10090000804689460396A6E7013200FB0838039229
:10091000BDE7124FC8F100080026B8F1000FC3D0A0
:100920002046294632463B4639F036FE08F101089A
:1009300004460D46F1E72046294632463B4639F04B
:1009400001FD08F1FF3804460D46AAE7AFF3008029
:100950009A9999999999B93F0000F87F000024402D
:1009600070B586B014460E460022014601A82CF050
:10097000CCFE2546DDE901239A4204D3049832F0E7
:1009800049FA601B04E02DB9049832F043FA20467E
:1009900006B070BD01A82CF0B1FD013D06F8010BB9
:1009A000E8E710B586B00A46014601A82CF0ADFE76
:1009B0000023DDE90112914203F1010401D2013368
:1009C0000AD1049832F026FA202029F05DF914F1BA
:1009D000FF340AD206B010BD01A82CF08FFD0A2802
:1009E000EFD029F051F92346E3E70820EDE70000B6
:1009F00070B50D2028F0AEF90028264B46DB264CBA
:100A00001871A17D01229A7000293DD1234DA18248
:100A100004334FF48E712846A360A275FFF7FAF8ED
:100A20002146AA60FFF725F9636893B92646A27D9F
:100A3000A38A9A420ED8A38A9BB2B3F5807F1BD0BB
:100A4000164BD3F81C21002AFBD00122DA600023C8
:100A5000A37570BDD5F81C3123B9A38A9BB2B3F539
:100A6000807FF7D1A38A9BB2B3F5807FE0D0314677
:100A70002846FFF7FEF8DAE70023A3750F210848A0
:100A8000BDE870402DF082B81121F8E700229A707D
:100A9000DFE700BF99C2002020BB002000200040FB
:100AA0002AB1050030B58BB04FF4D8230193054629
:100AB00008B1002303602022002102A8FEF732FDC6
:100AC000002202A94FF4D82035F014F9D0B1002447
:100AD000029B039A23F07F43033323F00303203365
:100AE00052B11C44032202A901A835F08BF9002859
:100AF000EED120460BB030BD002DF3D02A68134450
:100B00002B60EFE70446F4E72DE9F04F202291B087
:100B100000244FF4D825824688460DEB020021467A
:100B2000CDE904540694FEF7FDFC012208A92846ED
:100B3000079535F0DFF8A8B905AB019306AB52462F
:100B40004FF4EC21009304A8434635F09DFB049834
:100B5000013835F047F9049035F0DAFB012011B087
:100B6000BDE8F08F099B002B5DD0049E069BDDF84D
:100B70001C901E444E4523D0089B23F07F43203316
:100B80004B4401250D2702936A1E3E497A4302EB2E
:100B9000010B5846039231F041FAA8B1DBF800107E
:100BA000894508D8029B994205D2A6EB09030B445C
:100BB000039A34495350013540F6C4239D42E3D98A
:100BC00020230DEB030214E0584631F031FA0028DF
:100BD000F1D0DBF800300C33B3FBF7F31D44EAE748
:100BE00012F8011B0AF804100134B4FBF8F108FBF9
:100BF000114413F1FF33F3D2069B089E2033069372
:100C0000079B26F07F46033603F1200905AB26F04B
:100C10000306019306AF009743465246494604A88F
:100C200035F032FB2EB9012208A907A835F0EAF801
:100C300081E7069B059AA8EB0300A8EB0405854213
:100C400028BF0546A24203D9121B954228BF15466C
:100C50000293ADB1B54228BF354649460AEB0400C0
:100C60002A463AF083F8029B2C442B440693B4FBAB
:100C7000F8F308FB134405AB761BA9440193CAE7BC
:100C800028466CE7682E002030B58BB04FF4D8248E
:100C90002022002102A80194FEF744FC002202A9B0
:100CA000204635F041F870B1032202A901A8DDE920
:100CB000015435F0A7F80028F6D124F07F442335FD
:100CC0002C4424F00304C4F5EC200BB030BD00002C
:100CD000F0B40023124D0D271C4640F6C42607FB36
:100CE00003519A1CC87ACC72087B0C73C2F30B00B8
:100CF0004A79087122F00F02013342EA1022B3420E
:100D00004A71ECD148F6EB33064AEC54537823F0A1
:100D10000F035370044B01221A80F0BC31F0CEB99E
:100D2000682E002053BA0020662E002037B501231C
:100D3000009300231A460549054632F069FA044635
:100D4000284632F067F8204603B030BD09B00500F0
:100D5000F8B50646437A807A000150EA13100C4633
:100D600019D030F091FF074633F080F9451C384622
:100D700032F050F8284631F039FF214632F052FE69
:100D8000044638B10146304633F0E6F9204632F0E9
:100D900041F8681CF8BD0125ECE7000038B5074CA8
:100DA00025780023EDB202461946237034F08AFB01
:100DB00025700348BDE8384028F0F0B8642E0020C4
:100DC00000270600002370B50B6005460E4631F083
:100DD000D5FD044670B1294632F025FD0546204672
:100DE0001DB932F017F8284670BD31F02BF930608C
:100DF0002046F6E70546F6E72DE9F341002400F426
:100E00007F6715461470A7F54072502A0E4600F40D
:100E1000704312D8484A11F0100F484908BF1146D4
:100E2000002B79D0B3F5805F78D0B3F5005F444CE8
:100E300018BF00244FF440784BE0A7F50072202A39
:100E40000DD8002B6CD0B3F5805F6BD0B3F5005F8D
:100E50003C4C18BF00244FF400783B4939E0A7F51B
:100E60002072302A0AD8002B5ED0B3F5805F374C51
:100E700018BF00244FF4207835492AE0B7F5C07F29
:100E800009D1002B52D0B3F5805F324C18BF00243B
:100E9000B84631491DE0A7F11002B2F5887F47D866
:100EA00044F64302ADF80020C3F302321B0402F102
:100EB000310248BF4E2329494CBF8DF804408DF8BC
:100EC00003408DF8022048BF8DF803306C464FF088
:100ED0001008F00703D50F22284639F099FFB20712
:100EE0000BD5284639F08CFFA7EB08073F110122EC
:100EF00029180A23B8182BF0C4FC54B1330708D5BD
:100F0000284639F07DFF2146C0F10F02284639F00E
:100F10007FFF02B0BDE8F081114C8BE7114C89E7EF
:100F2000114C98E7114C96E7114CA3E7114CAFE731
:100F3000A0461149CDE700BF4CAF050045AF050005
:100F40009FEE05006BAF05006CE5050077AF05006F
:100F500073AF050056AF05005AAF050052AF05004C
:100F6000D8E405005EAF050061AF050066AF05007F
:100F70006FAF05007BAF0500012706002DE9F843A0
:100F8000394F03791C2202FB03720646506820B1D8
:100F900032684FF40174C2F808431C2202FB037349
:100FA000DA7D52B11A7E002A41D020B133684FF465
:100FB0000172C3F80423112037E00120D875D960ED
:100FC0005A761A7635791C2303FB05739B7E1BB971
:100FD00012B93046FEF726FE4FF01C0808FB0578D4
:100FE0003068D8F80430002B35D14FF4A271FEF7E9
:100FF00011FEC5EBC50907EB89093068D0F824312B
:10100000D0F80821D0F84441A2B90CB9002BF4D093
:101010001C2202FB05750022EA750BBB14BBA97EDE
:1010200033680122A9B11A600020BDE8F883196174
:101030000122C6E7002BEBD1002CE9D14946FEF78F
:1010400001FE98F8193098F817209A42D5D823460F
:10105000DEE75A60E8E74FF40173C0F80433E3E7D2
:101060000320E2E70F20E0E720BB00200A490B48FD
:1010700008B5FFF783FF014610B109482CF086FD43
:1010800008490648FFF77AFF014620B10648BDE847
:1010900008402CF07BBD08BD99C200207CAE050045
:1010A000E4B005009AC2002007B1050038B500225F
:1010B000054633F035FA044650B100231A4601467E
:1010C000284629F0B7FB2046BDE8384031F0A2BEE3
:1010D00038BD0000F0B54FF080530220D3F8501413
:1010E000D3F85424284BC3F804032848C3F8040356
:1010F000274B93F800E093F801C09F78DE781D79C4
:101100005C7998794EEA0C033B4333432B432343EA
:101110000343204B2AD083F800E083F801C09F707E
:101120001E715D719C71D8711D789C785A785E79BA
:10113000586885EA0401514081F08801D970197915
:1011400071409E797140DE7971401972120203215B
:10115000597242EA05420C4B2243C3F8942500BA67
:101160004422C3F89005C3F8A025F0BD080A197001
:10117000090C9970110A1A715971110C120E5870DC
:101180009971DA71D0E700BF00500040800008007C
:1011900094BF00207FBF002070B5EFF3108672B6B9
:1011A0000D4A94680123A4B993600C4B0C4DD3F8FD
:1011B000801029401160C3F88050D3F8841051602A
:1011C0004FF0FF32C3F88420047006B962B60020E5
:1011D00070BD0370F9E700BF64C2002000E100E0C9
:1011E000FC06FFBC437882781B01120202F4E06225
:1011F00003F030031343027802F003021343C27872
:10120000120302F4805213430279120402F4E02222
:1012100013434279120502F48012134382791206B5
:1012200002F080721343054AC2F81835C379017A77
:10123000C2F81415C2F81035704700BF00700040A6
:1012400038B5054631F0BDFC044630B3B5F90000B1
:1012500039F00EF841EC100B31F0B6FC10490246A3
:10126000204633F030F9B5F9020039F001F841ECCD
:10127000100B31F0A9FC0B490246204633F023F94C
:10128000B5F9040038F0F4FF41EC100B31F09CFC90
:1012900005490246204633F016F9204638BD00BF06
:1012A00022FC0500E2FC050076FE050010B588B0C2
:1012B00012788DF80C200021FF2202918DF80D206C
:1012C00001214FF6FF72104C01908DF81C10ADF803
:1012D0000E208DF8103027F0EBF970B12BF0B8FA32
:1012E00058B914F1FF34F6D2084904202CF08EFDD1
:1012F00001A827F0EDF908B010BD002CF4D02BF0B8
:10130000A7FA0028F0D1F3E780841E00F0AF0500B3
:1013100010B588B00023CDE9030102930E4C019271
:1013200002238DF81C3027F0C3F970B12BF090FA2E
:1013300058B914F1FF34F6D2084904202CF066FDA8
:1013400001A827F0C5F908B010BD002CF4D02BF08F
:101350007FFA0028F0D1F3E780841E00F0AF05008B
:1013600038B50B4C0B4D2B785BB12BF071FA40B9B3
:1013700014F1FF34F7D208490420BDE838402CF0BE
:1013800045BD002CF7D02BF063FA0028F3D138BD0F
:1013900080841E0084C2002092AF0500F7B5354F4F
:1013A000354C7E797601A31905465A7E002A5FD115
:1013B000A2590AB101225A7695E80F0004EB060EF5
:1013C0000EF1080C8CE80F0006F1180323445A793B
:1013D00022F003025A719EF81A20FF2A1FBF012330
:1013E00093404FF0A042C2F80C352A6822B102F0B7
:1013F0006043B3F1005F06D1AB6853B103F06043C3
:10140000B3F1005F05D0344400236376102003B0AD
:10141000F0BD3B682979C3F84425C3F848152A7BF9
:10142000A968C3F834150020C3F83825C3F818019B
:10143000D3F818210192019AC3F850050122C3F88C
:1014400040051A61A2597AB9D3F81821002AFBD0B5
:101450003444A27EFF2A05D0012393404FF0A042DE
:10146000C2F808350020D2E74022C3F80423CEE7B3
:101470001120CCE7B42C002064BB0020F0B5154649
:1014800085B01C4E07460C46FFF76AFF0123FF2D6F
:1014900033702B4628BFFF231FB3FA1816490A6082
:1014A0000CB3E218154900970A60154A0294002C03
:1014B000A5EB0305DBB21560684614BF1A4600228F
:1014C0008DF80C208DF80430FFF768FF024660B1FC
:1014D000002404200B4934702CF098FC204605B001
:1014E000F0BD3A46DAE72246DCE7FFF739FF012094
:1014F000F5E700BF84C2002088C2002080C200201F
:1015000078C200207FAF050013B51A4B1B78044644
:1015100063B3FFF725FF184B1B680022012004214D
:10152000C3F80025C3F80005C3F80813C3F8082161
:10153000D3F80811009100991049E4B20870C3F87B
:101540001C45D3F808010028FBD0C3F80821D3F8C4
:10155000080101900198D3F818050A70C3F8002516
:101560000722C0B2C3F8002502B010BD4FF0FF3013
:10157000FAE700BF7CC20020B42C002084C2002007
:1015800037B50B015BB249B2044643EA01008DF85E
:1015900004001A4D50B20343120152B28DF80530C7
:1015A0002B78114302438DF806108DF8072013B3F2
:1015B00002AB03EB941302AA13F8040CC4F3011357
:1015C000134413F8043C43EA00201FF0C3F92B78BE
:1015D0008BB102AAC4F3810304F00304134414443E
:1015E00013F8040C14F8043C43EA002003B0BDE8EF
:1015F00030401FF0AFB903B030BD00BF7CC2002047
:10160000C30914BF13020B0210F0400F70B5064659
:1016100014BF10460846184314460D46FFF774FFE2
:10162000B1064CBF23022B0216F0100F14BF204648
:1016300028461843FFF768FF32074CBF23022B02EE
:1016400016F0040F14BF204628461843FFF75CFF2E
:10165000B3074CBF2002280216F0010F08BF2C462A
:101660002043BDE87040FFF74FBF000020292DE95F
:10167000F0470BD9244A254E2139C9B2002314461C
:10168000DFB2B94205D814F801C0B6BB4008BDE8C6
:10169000F08712F8017B01333E44F1E7745CC82CFB
:1016A0001ED81EF80450DFF86C90194B4FF000085C
:1016B0005FFA88FA54450DD803EB0509994511D115
:1016C00001316145EADB0232504320F070400730BF
:1016D0000009DCE719F801AB08F101085344E7E71A
:1016E0000023E9E713F8018BB8FBF7F407FB148438
:1016F000E4B2A242B8BF2246E0E700210A46DFF882
:1017000014E00D27DDE700BF4BB105002AB205004C
:101710004EB4050085B3050010B5074A002332F822
:10172000024B8C4203D1184100F0010010BD01337F
:10173000082BF4D10020F9E768BA0020F0B5224B5D
:101740009F7C1C4600221D46D6B2B7420ED895F8A3
:1017500078701D4C0022D6B2B74216D895F8DE50EC
:101760000022D4B2A54220D800200DE0B4F814C065
:10177000844502F1010204F10A04E5D142F64D2349
:1017800001200B808870CE70F0BDB4F87AC060453F
:1017900002F1010204F10A04DDD142F64D230B806F
:1017A00002238B70CE700120EEE7B3F8E060B04208
:1017B00002F1010203F10A03D3D142F64D230B805B
:1017C00003238B70CC70EEE7F0BC002010B50C4CFE
:1017D000226886B0034682B104208DF804000868B0
:1017E000D989ADF80C10123333F8021C0290ADF811
:1017F0000E10049301A92046904706B010BD00BF0B
:10180000F0BC00207FB54B89022B0FD1094A136829
:1018100063B1097B0068029011F0010F14BF02212F
:1018200003218DF80410104601A9984707B05DF810
:1018300004FB00BFF0BC002070B50D4D002435F84E
:10184000026B964210D10122A240D2B2D543EDB232
:10185000014410F8014B2BB11443884200F8014CAD
:10186000F7D170BD2C40F8E70134082CE7D1F8E738
:1018700068BA002070B50023084C1A4641FA02F5F8
:10188000ED0706D504EB420600EB4305B688AE80B3
:1018900001330132082AF1D1036070BD64BA00201F
:1018A00010B586B004460022684616F091FA20462C
:1018B000009916F0BBFB204606B010BD38B50123D9
:1018C0000B7004460D4630F056FB88B100220B49E0
:1018D000204632F025FE10B133F0A3FA28702046DE
:1018E0000022074932F01CFEBDE8384033F060B9F1
:1018F0002046BDE8384032F0B9BB00BF38AF050024
:101900003DAF05002DE9F04F2DED028B8DB0436A00
:10191000059390ED048B1F02836A07671E024667DA
:10192000B0EE480AF0EE680A0446069336F080FBF3
:1019300059EC108BB0EE480AF0EE680A36F068FCFD
:1019400094ED067B404653EC172B49465BEC10ABFD
:101950008DED007B38F020FE0022614B38F0F2FC68
:101960000022604B38F038FB38F09CFFDDE90023A3
:101970000790A0675946504638F00EFE0022584B9B
:1019800038F0E0FC0022574B38F026FB38F08AFF95
:10199000E0670546059838F06BFC29F00043CDE977
:1019A00008010698CDF80880039338F061FCDDE962
:1019B0000223CDE90A01DDE9080138F0C3FCD04675
:1019C0002BF0004942468B464B468246DDE90A0130
:1019D00038F0B8FC02460B465046594638F0FCFA3F
:1019E000DDE9002338F0AEFC00223E4B38F0F4FA7B
:1019F00038F058FF42464B468346DDE9080138F08F
:101A0000A1FCDDE90A2380468946DDE9020138F0C0
:101A100099FC02460B464046494638F0DDFADDE9BE
:101A2000002338F08FFC2F4B002238F0D5FA38F025
:101A300039FF94F820305BB1226863680BEBDB71EF
:101A4000A2EB6102226000EBD072A3EB6203636041
:101A50002368059A5B44A36063680344E360079BC3
:101A60000BFB03F3013300FB053303EBD373D2010C
:101A7000A2EB6303C4F88030079B58430130069BF8
:101A80000BFB150505EBD575D80194F82130A0EBBB
:101A90006505C4F884503BB90DB0BDEC028BBDE8C0
:101AA000F08F3B44C4F88030D4F88030002BF8DB52
:101AB000D4F880309F420BDDD4F88430002B0BDB50
:101AC000D4F884309E42E7DC9B1BC4F88430F7E7EF
:101AD000DB1BC4F88030EBE73344C4F88430EBE719
:101AE000000070400000E03F1F4B204A1B6800BF11
:101AF00000BF00BF00BF00BF00BF00BF00BF9342D8
:101B00002FD000BF00BF00BF00BF00BF00BF00BF9D
:101B100000BF00BF00BF00BF00BF00BF00BF00BFCD
:101B200000BF00BF00BF00BF00BF00BF00BF00BFBD
:101B300000BF00BF00BF00BF00BF00BF00BF00BFAD
:101B400000BF00BF00BF00BF00BF00BF00BF00BF9D
:101B500000BF00BF00BF00BF00BF00BF00BF00BF8D
:101B600000BF0138C3D17047A42C00200024F4002A
:101B700008B1FFF7B9BF7047084B5A6E013A5A6671
:101B800022B907490A7822F002020A701A6E01325D
:101B9000042A08BF00221A66704700BFC0C0002098
:101BA000E2BC002030B5044685B00D46102200216D
:101BB0006846FDF7B7FC237A012B0AD0022B0ED022
:101BC00063680193236829469B686846984705B077
:101BD00030BD23690293A38AADF80C30F0E70123EE
:101BE000A2898DF80030E389ADF80A20D31AADF848
:101BF0000830E5E728DF704729DF704738B51C4B10
:101C00005A6E19465AB31C6E182202FB04331A7A14
:101C1000012A07D0022A23D018460921BDE83840FE
:101C2000FFF7C0BF1825D88A9A8A05FB0414D4E9A7
:101C30000314121AB2F5806F4FEA80000144B4BF5A
:101C400092B24FF480622044FFF7D6FF11280BD1E7
:101C5000084A137823F0020343F00403137038BDDD
:101C60009889FFF7C7FFF1E70028F8D0D4E700BF55
:101C7000C0C00020E2BC0020054A137813F0060F14
:101C800004D143F002031370FFF7B8BF704700BFE1
:101C9000E2BC00202DE9F3411F4B1B781746DA0701
:101CA000064688462BD51D4D1D4B9D4229D31D4B05
:101CB0009D4226D239B330B341EA00039B0724D1B9
:101CC0002B68984223D36A6800EB87039A421ED39D
:101CD000FFB101A8FEF7BEFB78B1019B0024C3E968
:101CE0000054019B01221A72C3E903869F82FFF709
:101CF000C3FF204602B0BDE8F0810720FAE70120CB
:101D0000F8E70220F6E70320F4E70620F2E70520D3
:101D1000F0E70420EEE700BFE2BC00200C2E00201C
:101D20000C2E00201C2E002038B5074B074A59689E
:101D3000948810684A880332032592B200EB84002D
:101D40001D70FFF7A7FF38BDE4BC002064C1002070
:101D500010B501220C460649FFF79CFF28B905493A
:101D600001EB041101238B7310BD0E20FCE700BFB3
:101D700028B0050020C0002008B502220149FFF765
:101D800089FF08BD2CB0050008B5034B034918684E
:101D90000222FFF77FFF08BD64C1002034B00500B8
:101DA00073B51B4B1B78DB0705462BD5194E1A4B19
:101DB0009E4229D3194B9E4226D238B3C0F30B045E
:101DC000D4B93368984219D3726800F580539A42A7
:101DD00014D301A8FEF73EFB90B1019BC3E9006458
:101DE000019B02221A722D0B01229D811A82FFF79C
:101DF00043FF204602B070BD0620FBE70520F9E74F
:101E00000720F7E70120F5E70220F3E70320F1E7D9
:101E1000E2BC00200C2E00200C2E00201C2E0020E6
:101E200010B50B4C0B4B628803EB02139A892AB94D
:101E30005868FFF7B5FF0423237010BD05232370F6
:101E4000054B022218689A80FFF7AAFFF5E700BF4A
:101E5000E4BC002020C0002064C1002008B5074B6E
:101E6000191D5888FDF7B6FB18B1BDE80840FFF70B
:101E70005BBFBDE80840FFF7D3BF00BFE4BC002054
:101E800010DF7047002208B511461AF065FB00000C
:101E90002DE9F347254B1B681BB1984730B3FFF77B
:101EA000F1FF234B1B7803F0FF07FBB1214D224EBE
:101EB0002C68DFF88C90B4FA84F46409B046337867
:101EC000A3B901A8FDF76AFB052812D00028E6D1C6
:101ED000019B0BB9FDF73EFD184B1B680BB1019838
:101EE00098474CB10124EAE7002CFBD002B0BDE8D2
:101EF000F087002CFAD13C46DFF848A098F8003073
:101F0000002BF3D1B9F80030ADF80430DAF8003026
:101F100001A91846FDF740FB0528E5D00028BED1F1
:101F20002A6818469047002CE8D1C8E7D0BC0020AA
:101F300061C100209CBA002062C100206CC1002059
:101F400098BA00205CC2002010B5084B9A685AB1BC
:101F500050B9EFF3108172B6054A1C6814605C68D2
:101F60005460986001B962B6002010BD64C20020C0
:101F700000E100E02DE9F3411D4F7B6806460D4668
:101F80009BB304292FD943697BB3437C0024012BE5
:101F90000DF107000CBF8846A0468DF80740FFF7FB
:101FA000FBF80DF10600FDF7A3FBD0B10123037090
:101FB000104B4660D3F80435C0E90484C0E902350B
:101FC0009DF806307B709DF80700FFF7BDFF24B930
:101FD000094B4FF48012C3F80021204602B0BDE83F
:101FE000F0810424EFE70724F7E70824F5E700BFB2
:101FF0009CBF00200010014000E100E02DE9F3410A
:10200000CE0801F007044FF0010808FA04F4855DDA
:10201000E4B22540074613D10DF107008DF80750B3
:10202000FFF7BAF8BB5D9DF807001C4202BF1C43D6
:10203000BC554546FFF788FF284602B0BDE8F08151
:102040000025F9E72DE9F3478146002701261FFA0D
:1020500087F84FEAD80A08F0070406FA04F419F8DA
:102060000A50E4B2254008D00137B7F5807FEED1A1
:10207000B846404602B0BDE8F0870DF107008DF884
:102080000750FFF789F819F80A309DF807001C423D
:1020900002BF1C4309F80A400125FFF755FF002D38
:1020A000E2D0E6E773B50546B8B1C1F3C70401F065
:1020B000070301269E40035D33420ED000230DF13D
:1020C00007008DF80730FFF767F82B5D9DF80700D4
:1020D00023EA06062E55FFF737FF02B070BD000059
:1020E00038B50A4B1A687AB15D686DB1FF280BD01C
:1020F00084B221462846FDF79FFB28B12146284699
:10210000BDE83840FFF7CEBF38BD00BFACC10020EE
:102110002DE9F74F9846531E072B81460F4615466B
:1021200000F2BB80FF2800F2B88001465E48FDF750
:1021300083FB0646002800F0B08039464846FDF78C
:102140003BFB044600283ED0C3689D4247D805D2D9
:102150005FFA85F9E368207C994543D394F81090A1
:10216000B9F1FF0F40F09780504B1A689B46002A48
:1021700041D14FF6FF732380A3700023C4E90133DC
:10218000E360238A03F4784343F0FF0323821120A2
:1021900084E0237C1844C0B2FFF7A2FFE3685FFA33
:1021A0008AF083420AF1010AF3D84FF6FF732380C5
:1021B000A3700023C4E90133E360238A03F4784366
:1021C00043F0FF032382FF214FF6FF70FDF7F4FA7F
:1021D00004460028DBD0A0F800908770BEE74FF0DF
:1021E000000ADBE74844C0B209F10109FFF778FFB4
:1021F0005FFA89F9AEE75B68002BBAD00023DBF801
:1022000008205FFA83FA924502D34FF0FF0912E0EB
:10221000DBF8040060B351460193FFF7EFFE019B2A
:1022200030B3B9F1FF0F08BFD146AAEB090A0AF192
:10223000010AAA4521D1B9F1FF0F84F8109098D076
:10224000E560207CFDF708FB58B305EB85052D0103
:10225000ADB2AD0888F80270C8F80400A8F80050C4
:1022600026B1082F02D1AD00063D8580002015E083
:10227000B9F1FF0F0CD14FF0FF090133BFE748461A
:10228000019309F10109FFF72BFF019B5FFA89F91F
:10229000D145F4D3EFE70026D2E7072003B0BDE82D
:1022A000F08F0320FAE700BF78C00020ACC1002007
:1022B00038B504460025E368AB420ED84FF6FF73ED
:1022C0002380A3700023C4E90133E360238A03F46D
:1022D000784343F0FF03238238BD207C2844C0B2FA
:1022E000FFF7FEFE0135E6E737B5FDF765FA05466F
:1022F000A0B144682CB10A4B01941B789B0706D40B
:1023000003242846FFF7D4FF204603B030BD01A8C0
:10231000FDF746F904460028F3D0F1E70524F3E77A
:10232000E1BC0020FF2810B5044609D80146054845
:10233000FFF7B8FE21460448BDE81040FFF7B2BEE3
:1023400010BD00BF78C0002098C0002013B50DF16B
:1023500006010446FDF766F970B1BDF80620084B8A
:1023600003EB02139A894AB1A17A39B1013A0020EC
:102370009A81A07202B010BD0A20FBE70620F9E79F
:1023800020C0002037B50D460DF106010446FDF7CB
:1023900049F988B1BDF80620084B616803EB0213C8
:1023A00000209A8901329A81296063680C336B603E
:1023B0000123A37203B030BD0A20FBE720C0002038
:1023C0002DE9F043DFF88480D8F874E0BEF1030F04
:1023D0000F46944635D81C4E756CC1F108039D42DA
:1023E0002FD8D8F8704074441C2304F003048146AD
:1023F00003FB0484B9E80F000FC499E807000EF14D
:10240000010384E80700C8F87430C7B1336C2B446B
:1024100003F0070306EBC303002206F138040CEBBC
:10242000C20103C9A34202F1010283E8030014BF01
:102430000833054B9742F2D1736C1F447764012037
:1024400000E00020BDE8F083A8BB0020A4BF00206E
:102450002DE9F0411C46184B1B789B0706460F469A
:10246000154627D5DFF85880A3880BB10A201FE056
:1024700098F800302BB92146A088FDF7ABF820B9B9
:102480002060A3880133A380EEE723681EB19988FA
:1024900032889142EFD11FB119883A889142EAD12E
:1024A0009B682B6023686B60044B1B892B81002089
:1024B000BDE8F0810220FBE7E1BC0020E4BC002085
:1024C00020C0002030B587B04CF2070305460C460B
:1024D000ADF8043003AA0F4B01A90020FFF7B8FFA5
:1024E00010B1002007B030BD01A903A8FFF74AFFD3
:1024F0000028F6D10723A370019B5A882280029AF4
:1025000062609B8803F580432B8003A8FFF71EFFC2
:102510000120E7E7D4BC00201FB50023A0F58040D0
:10252000A1F58041CDE90233ADF80400ADF8061005
:1025300002AB0DF1060101A8FFF78AFF002818BFC2
:10254000052005B05DF804FB2DE9F04102230B8066
:10255000164B00251C6800F5805E2F4608304FF6AC
:10256000FF7870450AD305B11C6002B11770BDE851
:10257000F08101270EE0344601250BE006680136A4
:10258000F1D086884645F4D00688002EF1D08668C2
:10259000A642F0D8468806F1030C00EB8C00B1F897
:1025A00000C00CF1030C66440E80DAE76CBE00201C
:1025B00070B5064D0646002455F8043B0BB1304675
:1025C00098470134082CF7D170BD00BF84BB0020B0
:1025D0002DE9F047AA4C266F1C2707FB06F586B0AD
:1025E000635D013B8046052B00F22A81DFE813F092
:1025F0000600640064001D011D017E0130B1A14A86
:10260000137823F00103137001201FE025442B7978
:10261000032B15D8DFE803F002072C34FFF7B4FBD7
:1026200001232B7109E0984D2B78022B40F03C825E
:102630006868FFF7A1FB00232B70002800F0F080F2
:10264000904A137823F0010313700E201C23734368
:10265000E218E35C0290023B012B00F232818B4BCB
:10266000907D196C5A6C0144121A19645A6428E15D
:10267000874F3868FFF794FB0223BB800023D0E725
:10268000834FDFF804823868FFF776FB814BD7F879
:1026900000E05B88B7F804C01B0108EB0302516837
:1026A000A2F808C0C2F804E00222BA800022396011
:1026B00008F803202A71C0E707FB0647724BB7F8FA
:1026C00012A04FEA0A1A03EB0A029946118960B177
:1026D000FB8803F103088844C3F57F435189A2F8BE
:1026E0000880FD330B4453818EE7536803EB810868
:1026F0003B7C062B00F29780DFE803F02D733C4D06
:102700001F84040041F61D501C2303FB0643D144E3
:10271000DB88B9F80810DA1C0A44A9F80820C3F5C8
:102720007F43B9F80A20FD331344A9F80A3041F673
:102730001D53984200F0C38088E75748574900234B
:1027400043601C2303FB06439B690360FCF76AFF9D
:10275000002800F04C81291D012221444046FFF74A
:1027600099FA1C2303FB064302221A74002857D04F
:102770000E20C9E705F10C010122214408F10800EF
:10278000FFF788FA1C2303FB06439A7D002A14BF37
:1027900003220122E9E73D4B5A6C002A00F08C81AC
:1027A000196C1C2505FB0645481C00F0070003EBCF
:1027B000C1071864A88A53F83110013A5A6408EB2B
:1027C0008000BA88FFF766FAAB8ABA881344AB82F6
:1027D000AB7D013BDBB2AB75002BC7D101232B7462
:1027E000C4E705F108010122214408F10400FFF7C4
:1027F00051FA1C237343E25C032A0CBF0522062214
:102800002344B2E7254B1988234B5868FFF7A0FAF9
:102810001C2303FB064306221A7400287FF474AFBE
:1028200006B0BDE8F0870F206EE700287FF4ECAE1D
:1028300007FB06473B79012B32D01BB1022B3ED060
:102840000F2003E7CDE90200FB6801930DF10201BF
:1028500001A8FCF7E7FE80B10298BDF8021083885A
:10286000FB8003883B81FFF773FA1C2303FB0643BD
:1028700002221A710028D3D059E70A20F5E700BFD9
:10288000A4BF0020E1BC002020C00020A8BB002085
:1028900064C10020E4BC00203C2E002070C2002057
:1028A000864FA81D3B4601AA41462044FFF7D0FDB4
:1028B000B8B9B9880298FFF74BFA0A28DAD1002391
:1028C00002931C2303FB06F2A25C013A052A00F2E4
:1028D000B580DFE812F08E009200A000CB00D5009A
:1028E000E1000A28C7E90088E9D020E700287FF442
:1028F0008BAE734BDA7AAAB1D8721A78013A062AEB
:102900009ED801A151F822F0B9290200B329020092
:10291000C9290200CF29020041280200D52902005E
:10292000E52902001A78072AE7D801A151F822F018
:1029300051290200FB280200FB2802006D29020039
:10294000812902009F2902009F29020069290200B3
:102950001A8901321A8100225A80DA72594A127891
:10296000B2FA82F252099A72012207E05649586877
:102970008A884088033202448A8002221A70BCE7A7
:102980005D88504A504902EB05120868556850604E
:102990008888108102228A800D600622EEE70722D5
:1029A000ECE7484900229A728A8942B9897B31B1A1
:1029B0005A80FFF753FA5DE79A7A002AF1D1002294
:1029C0001A705A805A607AE7FFF7AEF952E7FFF7BC
:1029D00027FA4FE75A883B4B03EB02135868FFF77F
:1029E000CBF947E700225A60FFF7CEF942E70A2009
:1029F0002CE600238DF8043020E003FB064301227F
:102A00008DF804201A89ADF810209A88ADF81220AC
:102A1000DB68039312E003FB064302228DF80420D7
:102A20001A89ADF810209A88ADF81220DA681B7C5C
:102A300003929A1F534253418DF8143001A8FFF7B7
:102A4000B7FD206F1C22002102FB0040FCF76AFD4D
:102A5000636F1BB3226F013202F00302013B226756
:102A60006367DBB10020FFF7B3FDD9E603FB064344
:102A700003228DF80420DA88ADF810201A89C5E702
:102A800003FB06430422DB88ADF8103000238DF8E9
:102A90000420ADF81230D1E70523ABE70B4A1378D9
:102AA00023F004031370BBE6084A137843F00203D3
:102AB00023F00103137002E71368FFDE90C20020C9
:102AC000E4BC002020C0002064C10020E1BC002044
:102AD0000846FFF77DBD0000054A137813F0040097
:102AE00004D143F004031370FFF772BD704700BFB9
:102AF000E1BC0020F0B51C463D4B1B789E0789B019
:102B000007460D466FD509884FF6FF7399426CD082
:102B10006B88002B69D06968B5F808C000239C4514
:102B200003D8BAB9164604310AE051F833008007D9
:102B300057D10133F3E731F83200304486B2013225
:102B40009445F8D80DF102013046FCF7B3FD28B1E9
:102B500009B0F0BD13885688ADF8023000238DF817
:102B60001430BDF80230ADF816300323ADF818303C
:102B7000204B8DF804401A6829898DF81A1001320B
:102B80001A602B88ADF80C30032C6B88ADF8083038
:102B900004BF04238DF81430049208BF3B686A68B0
:102BA00008BF0793002401A8ADF80A60ADF80E40F5
:102BB000FFF706FC50B9BDF802200F4B03EB0213E0
:102BC00058890338801B58810820C1E7049B3B606B
:102BD0000A4B7C601B89BC723B81FFF77DFF20465E
:102BE000B6E70320B4E70220B2E70420B0E700BF55
:102BF000E1BC00206CBE002020C00020E4BC00200E
:102C000030B58BB0FF28044601921D4645D88B781D
:102C10001846FCF7A7FD00283FD04A6802920A88B0
:102C2000ADF80C20A4F58042ADF81C20A3F580423D
:102C3000ADF81E2002AA08920122ADF82420194600
:102C400004AA2046FFF768FC0528019A0ED102234A
:102C500052B907A904A8FFF74DFF07281FD010D8C5
:102C6000B0B103200BB030BD01AAF2E732B10E4B78
:102C70001B789B0702D501A8FCF792FC03230022D6
:102C8000E7E708280DD00E280CBF11200320E9E744
:102C9000002DE7D0049B2B60E4E70720E2E78620C5
:102CA000E0E71120DEE700BFE1BC002073B5154E60
:102CB000736805461BB343690BB3002404740DF11C
:102CC00007008DF80740FEF767FA0DF10600FCF7E4
:102CD0000FFD90B1022303709DF8063045607370BC
:102CE0009DF80700FFF730F924B9074B4FF4801225
:102CF000C3F80021204602B070BD0424F0E7082488
:102D0000F8E700BF9CBF002000E100E02DE9F84398
:102D10002649274B0025C1F84051C1F84451C1F85C
:102D20004851C1F84C51C1F80051C1F804511B6819
:102D3000002B39D0D1F804451E49DFF88C80096892
:102D4000641A24F07F442F461A68A24217D8A41AA6
:102D500015441A7CDE6982B1D8F800901F74D3E95B
:102D60000521B9F1000F06D01046C84728B1FFF77A
:102D700089F83346E8E708469047002EF9D10E4A15
:102D80000E4B11781B788B4205D10133DBB2022B3D
:102D900008BF002313701278094B43F82250094BE7
:102DA0004FF48012C3F80021BDE8F8830010014001
:102DB00060C200207CC1002079C1002078C10020C1
:102DC00070C1002000E100E0CCBC00200D4B0E499A
:102DD0004FF4003210B5C3F8802001244FF4803343
:102DE000C1F848332F20C1F808334C60FEF77CFE51
:102DF000064B8C602F2000211960FEF775FE044BF6
:102E0000197010BD00E100E0001001407CC10020FD
:102E100059C100202DE9F04FB64AB7491378097817
:102E2000B64D85B09942D5F80080019500F09580A7
:102E30000133DBB2022B08BF002313701278B04BB2
:102E400053F82260019A08EB060323F07F431360D6
:102E50000127AC4BAC4A18680290AC48117890F846
:102E600000904FF0000CE2465078884278D1BCF1D7
:102E7000000F02D0A54981F80090002F40F0BB80E0
:102E80001F6802997F1A18BF012700201968029154
:102E90009E49039191F800E000244FF001080028BA
:102EA00040F0AD8092F80190D2F804C092F802A0F0
:102EB0001178494540F0C1801B68029A9A4201D1BD
:102EC000002F44D0002B00F01281D3F80090904CDA
:102ED000019BD4F8046519688E4F751A3B7825F06C
:102EE0007F450335A3B94FF48033C4F84433C4F8A5
:102EF0000433894B4FF400324FF00108C3F88021AE
:102F00002F201A60C4F80080FEF7EEFD87F80080DD
:102F1000A9452CBF4944491921F07F41C4F8401507
:102F2000D4F804359B1B23F07F43891B033321F026
:102F30007F418B420BD9D4F80435C4F840352F209B
:102F4000FEF7D2FD744B4FF40032C3F80021039A10
:102F50000023137005B0BDE8F08F0026374678E7F0
:102F600001EB4104506892F802B000EBC40E01314D
:102F700010F834401868C9B28B4508BF0021022CF4
:102F800004D0032C7FF470AF002410E0DEF804B00E
:102F900004468646002C3FF467AFA34500F0C0808E
:102FA000A646E469F6E780F810A0C069012400286D
:102FB000F9D1002C3FF458AF186055E7D4F80C90C5
:102FC000C4F800E0761A8C44E1691960B9F1000F89
:102FD00007D008EB0C0121F07F41C4E90119E06141
:102FE00020461C68002C3FF451AF2168B142E5D95E
:102FF0008E1B26604AE7002084468646F1E701469C
:10300000C069019DD1F804A02E68444DD1F8089004
:10301000AAEB060C2CF07F4CAC4535D80CEB09061E
:103020000E60D3F800C081F81080C1E90144CC6182
:10303000BCF1000F33D1196031E701EB410B0131D5
:10304000C9B2514514BF117014701CF83B1001290E
:103050000CEBCB067FF42CAF716891F810B0BBF18C
:10306000000F7FF425AFD6F808C0C1F804C0F5689A
:103070008D603569CD6076698E61BEF1000F0CBF41
:1030800066465E464E60BCE7A6EB0A0626F07F4623
:103090004E4502D2A9EB0606C2E70C60C1E7D1F8A3
:1030A0000090DCF80060B1451FD8A6EB0906CCF80B
:1030B0000060C1F81CC0BEE7A9EB0A09D6F81CA045
:1030C000B446BAF1000F0AD05646D6F800A0CA4559
:1030D000F2D3AAEB090AC6F800A0B2466646C1F8C8
:1030E0000090C1F81CA0F161D9E66646EDE7FFF754
:1030F0006DFE2CE778C1002079C100207CC1002042
:1031000070C1002060C200209CBF002058C1002078
:103110000010014059C1002000E100E0FEFF7F00E7
:1031200074450FD1D0F81CB0C3F800B0BBF1000F4C
:1031300008D10A4D0120A86001984FF0010CC0F899
:1031400000B0E1462068E469CEF81C40002C3FF452
:103150008BAE25682844206086E600BF0010014041
:1031600037B5074B054693E803006C46002384E817
:1031700003001A4621462846FFF742FD03B030BD42
:1031800058AE0500FDF782B910B54FF6FF7304463F
:103190009C42084609D1FEF755FFB0F5807F0446F2
:1031A00001D14FF6FF74204610BDFF2CF9D82146FF
:1031B000FEF724FF0028F6D1F3E710B5044601F02E
:1031C000EFFC2046BDE8104000F02EBF1FB503788D
:1031D00093B90279072A0FD1448803932046CDE999
:1031E00001338DF80420FCF7A7FAADF8060001A81A
:1031F000ADF80840FFF7E1FF04B010BD1FB5002394
:10320000CDE901330393ADF80600022301A88DF840
:1032100004308DF80810FFF7D0FF05B05DF804FB0F
:1032200086DF704738B504884CB9821C00F10A0566
:1032300012F8013B1BB99542FAD100200AE00B8835
:10324000A342FAD108220231023037F081FDB0FAF0
:1032500080F0400938BD08B570B171B103780A78C3
:10326000534013F0FE0F08D106220131013037F030
:103270006FFDB0FA80F0400908BD0020FCE710B5F2
:10328000044600F0BDFF2046BDE8104000F04ABFF4
:1032900043DF70476FDF7047024B0022C3E9002213
:1032A000704700BFD4BC0020F0B5FF2887B00446AB
:1032B0000E4615461F4629D80846FCF753FA28B390
:1032C00003AA2046FFF728F918B10524204607B0C5
:1032D000F0BD01A903A8FFF755F804460028F4D172
:1032E000019BAE705A882A805FB13B6892009A4277
:1032F0000AD30299686837F039FD03A8FFF726F86A
:10330000E4E7029B6B60F8E70424DFE70724DDE7CE
:103310002DE9F041CEB020AE502380460CADB8224E
:103320000021304601930395FCF7FCF80DF197035B
:1033300005930DF1AE0306930DF1C503079337AB6B
:1033400008930DF1F30309930DF585730A931C4F50
:1033500004960DF221130B930024444507D1E2B2E9
:10336000002104A8FFF796FF4EB0BDE8F08150227F
:1033700000212846FCF7D6F801AB02AA072137F84E
:10338000020BFFF791FF20F002000528ECD06B7CC8
:10339000032B12D817230DF1310203FB04630DF147
:1033A000450152F8040B43F8040B8A42F9D1118805
:1033B000198092789A700134CFE743F20220D3E764
:1033C0008AC100202DE9F04110220546A6B0002157
:1033D0002D48FCF7A7F835B929462846FCF7C0F96F
:1033E00026B0BDE8F0816A0028492748DFF89C80B4
:1033F00004AE37F0BBFC382200213046FCF792F8CF
:1034000000245023CDE9013412AF0397502200214C
:103410003846FCF787F801AB02AA072138F8020BFF
:10342000FFF742FF20F002000528D9D09DF859305F
:10343000032B26D8C4EBC402B318DDF85910B150E1
:103440000134BDF85D209A80A5429DF85F209A71F5
:10345000DCD10DF1170313930DF11E0314930DF13D
:10346000250315930BAB16930DF1330317930DF151
:103470003A0318930DF1410312961993E9B23846B5
:10348000ACE743F20220ABE79AC100208AC10020DA
:103490002DE9F043037889B00546002B3FD101792F
:1034A00007293CD104AA4088FFF7FEFEB8BBFFF70E
:1034B000F3FE02A90DF10600FFF704F878B36E8859
:1034C000BDF80670BE42F4D0059C631C184611344A
:1034D00013F8012B12B9A342FAD1EAE7DDF80C8008
:1034E000102208F1010137F033FC08F11101814687
:1034F0002046FFF7B0FEB9F1000F01D00028D8D068
:103500003046FCF719F90023ADF81A0006A88DF82B
:103510001830ADF81C60ADF81E70FFF7B0FE09B0B2
:10352000BDE8F083CA1F012A73B5064654D80025AA
:10353000CDE900558DF80210FCF73EF9044600284D
:103540004CD0437CDB074BD4007CFCF785F910B9E9
:10355000032002B070BDE368019003EB83031B01FD
:103560009BB29B086846ADF80030FCF703F962682F
:1035700004F1080369463046FFF742FB637C03F021
:103580000603062B01BF174A136803F1FF331360CC
:1035900030B9637C23F0070343F001036374D8E779
:1035A00011280BD10F4A136801331360637C23F099
:1035B000060343F0040363740020CAE7862809D198
:1035C000084A136801331360637C23F0060343F059
:1035D0000203E3E70728BBD10720BAE70520B8E7D5
:1035E0002846B6E774BE00202DE9FF4105461022AB
:1035F00000216846FBF796FF68882979ADF802003C
:103600008DF80410FCF7D8F82B78454E092B5ED8BE
:10361000DFE803F00505684D4D6C7173757D00287A
:103620003FD0437CDC073CD5FEF742FE2B78581E8A
:1036300043424341002468468DF800408DF808302D
:10364000FCF7ACF833684BB3364E002537464FF0E5
:10365000140808FB05735B7C5A0703D49B0759D5F4
:10366000002C57D0B1783088FFF75CFF002851D08C
:1036700014235D437B1986289B788DF804307A5B90
:1036800016BF0290082309236846ADF802200CBF3C
:103690008DF800308DF80030FCF780F804B0BDE8FC
:1036A000F08101238DF80030AB68029316E080B101
:1036B0008268AB689A420CD1437CD90709D532683D
:1036C00023F00503013243F0040332604374002405
:1036D000B8E702238DF80030EB6803936846FCF7E7
:1036E0005DF8F4E703238DF80030F7E704238DF845
:1036F0000030EB68D9E70523F5E70623F7E7072352
:1037000068468DF800300124FCF748F89AE7EB682A
:103710000293DCE70135082D06F1140699D1BDE7C7
:1037200074BE0020BCC1002070B500238CB02D49B0
:103730002C4E4FF6FF70CDE90033FCF7F1F84FF651
:10374000FF750446AC420BD0A4F58043ADF81430AD
:1037500002AA6B46002105A8FEF77AFE0A2822D0AD
:10376000214B1A781846E2B94FF6FF718C4218D0F7
:103770001E4E367801251D70B607A4F580439BB216
:103780001DD58B422CD005218DF8141005A81146AB
:103790008DF81850ADF81A30FEF712FE60B1FFF741
:1037A0009BF90CB070BD2046FEF7BCFD20463146AB
:1037B000FCF7B6F80446C5E70D4B1D70F1E7022390
:1037C0000022092102708DF8141005A8FF21ADF820
:1037D00016408DF81810CDE90723FFF705FFE0E745
:1037E0000423EDE798C0002031C00020E1BC002098
:1037F00032C00020F0B5426805783D4C85B0B2FA81
:1038000082F149090391691E0346042924D8DFE89F
:1038100001F0030330496A009989DE8901F580418E
:1038200089B243F6FE77B94204D906F5804080B2EA
:10383000B84211D8012DADF802108DF8046013D1F3
:10384000002A14BF032100218DF8001003929B6809
:1038500002936846FFF7C8FE23781BB1002323704C
:10386000FFF762FF05B0F0BD002A14BF042101215B
:10387000EAE79989DD8901F5804189B243F6FE7650
:10388000B14204D905F5804080B2B042E4D8002AA4
:103890000CBF02220522ADF802108DF804508DF8FD
:1038A0000020D4E7988900F5804080B243F6FE718D
:1038B0008842D1D8DB89002BCED1FF23ADF802009E
:1038C0008DF804305AB906238DF80030FEF72AFD32
:1038D000084A002323701370FFF726FFB9E7072378
:1038E0008DF80030F4E708238DF80030B1E700BF11
:1038F00032C0002031C00020F8B50D490D4DFCF755
:103900000FF84FF6FF760446A5F12007B44201D127
:103910002046F8BDFF2CFBD821462846FBF78CFF3C
:103920000028F5D020463946FBF7FAFF0446EDE7BC
:1039300078C0002098C0002073B5104B104C93E85D
:1039400003006D46002385E803001A4629462088B7
:10395000FFF756F94FF6FF762388B34201D01128BE
:1039600001D102B070BD1846FFF7C6FF00231A460A
:1039700029462080FFF744F9EEE700BF60AE05005E
:10398000BCBC00201FB50378012B044615D101797A
:10399000012912D1002302AA4088FFF785FC60B9F3
:1039A00002238DF800306388ADF80230039B68462F
:1039B0001B788DF8043000F0B5FD054B1A884FF6E2
:1039C000FF739A4201D0FFF7B7FF04B010BD00BFEC
:1039D000BCBC002070B504468AB0142200216846A1
:1039E000FBF7A0FD6588ADF804502846FBF7A4FE60
:1039F0002378ADF80200092B15D8DFE803F005168F
:103A00003048525E8614A1A507238DF80030237933
:103A10008DF808309DF80A3043F001038DF80A3024
:103A20006846FBF7EFFE0AB070BD07238DF8003043
:103A300023798DF808309DF80A30444AA168039133
:103A400043F001038DF80A301368002BE8D0994247
:103A5000E6D1002313603E4A03931580E0E7082374
:103A60008DF8003023798DF80830E3680493374BE4
:103A7000A1681A680391002AD2D09142D0D1354969
:103A800000221A600B680392013B0B60C8E7072312
:103A90008DF8003023798DF8083001238DF8093036
:103AA000BEE708238DF8003023798DF80830012314
:103AB0008DF80930A3680493B2E7274D09238DF8E8
:103AC00000302B78002BABD04FF6FF70FFF714FFC0
:103AD0004FF6FF7398420646A2D12049FBF720FF1C
:103AE000B04204469CD1142200210DEB0200297043
:103AF000FBF718FD0B238DF81430ADF81840ADF826
:103B0000164005A8FBF77EFE8AE70A238DF80030F1
:103B1000114BA4681A780294002A81D01422002143
:103B20000DEB02001970FBF7FDFC0C238DF814302F
:103B30004FF6FF73ADF81830ADF816300794E0E794
:103B400005238DF800306BE70623FAE774C00020E8
:103B500068BE0020B8BC0020BEBC002098C0002079
:103B60002DE9F047474B1B788AB00546002B00F043
:103B70008780454B454F93E803003C7803AE86E8C9
:103B80000300BCB94FF6FF70FFF7B6FE0123ADF896
:103B9000143001AB06930423029305AA02AB06215D
:103BA00080460194ADF81640FFF77EFB07284AD106
:103BB00001233B70364B1C689846002C5AD1354A7D
:103BC000354F12883B68AA4241D1002B3FD01422C6
:103BD00021460DEB0200FBF7A5FC072328468DF8D4
:103BE0001430FBF7A9FD0623ADF8160005A8ADF8C3
:103BF00018508DF81C30FBF705FE20460AB0BDE8D2
:103C0000F087CDF804A0019B4046A34224BFC146E3
:103C10001C46FFF771FEBDF814309B00029305AA05
:103C200002AB06218046FFF73FFB0028EBD00528BA
:103C3000E7D04FF6FF7398451CD1164BA3F80090C0
:103C4000154B1C60B4E74FF6FF79A246EDE7013350
:103C50003B6000220E4B31462846FEF7D1FF00287C
:103C6000CCD00023C8F800303B68112803F1FF33A3
:103C70003B6001D11120C1E7862818BF0320BDE7B2
:103C80000820BBE770BE002068AE050073C00020AE
:103C900074C0002068BE0020B8BC002063DF7047FD
:103CA000A6DF7047A2DF70472DE9F04391B0984638
:103CB00011238DF8043013788DF805300024164652
:103CC00001254FF0000365F34203074689461C2295
:103CD000214609A88DF80630FBF724FCB3788DF84F
:103CE0000930C3F30302A24214BF1A2212228DF834
:103CF000242001AA0E9203AB72788DF80820049359
:103D0000224602AB65F34202059308238DF80A2090
:103D1000CDE9064404AAADF81C3009A94346388809
:103D20008DF80E50ADF80C900894FFF7BBFF11B062
:103D3000BDE8F083A0DF7047044A01231168834087
:103D40000B401ABF1218507E1846704764BA002004
:103D500070B4094D134601262A6806FA01F414428C
:103D600007D001F1190402463146281970BCFDF74D
:103D700063BD70BC704700BF64BA00201FB500234C
:103D8000CDE9013303938DF80A201A46074BADF8AD
:103D9000081006241978ADF806008DF80440FFF7E6
:103DA000D7FF01A8FFF709FA04B010BDAF2C00201F
:103DB00010B4084A012314688B40234006D00A44FB
:103DC0005DF8044B0146507EFDF7A6BC18465DF831
:103DD000044B704764BA002010B50A4B19780446AA
:103DE000FFF7E6FF58B1084B00205A88A24201D1E4
:103DF000C0B210BD0130082803F10C03F5D1FF203B
:103E0000F7E700BF4CBC00204EBC00202DE9F84372
:103E10000546FBF791FC234B0746002214209846E9
:103E200000FB02F1CC5AAC422AD10B4400263446A6
:103E30004FF014095BB199782846FEF755FA10B196
:103E4000052818BF032401363246072A1DD9A4B914
:103E5000FF2D24D8144928464FF6FF75FFF794F933
:103E6000FFF762FCAF4208D03846FFF7B5FFFF28E6
:103E700003D00C2343430D4AD5522046BDE8F883B6
:103E80000132082ACCD10023D0E709FB02F338F82D
:103E90000310A94201D14344CCE70132D5E70724FE
:103EA000EBE700BFBCC1002098C000204EBC002042
:103EB0002DE9F0411F46154B9DF818400E469046DF
:103EC00019780546FFF744FFB8F1000F17D0104BE3
:103ED0003A4619782846FFF73BFF0E4B22461978E1
:103EE0002846FFF735FF44B12846FFF775FFFF2846
:103EF00003D00C234343084AD652BDE8F081002C7E
:103F0000FBD03046BDE8F041FFF780BFAF2C00206A
:103F1000B12C0020B02C00204EBC002008B5FFF7CB
:103F20005BFFFF281DBF0C234343034A4FF6FF707E
:103F300018BFD05A08BD00BF4EBC00202DE9F04389
:103F400085B00546FFF7EAFF4FF6FF739842074634
:103F500041D001224FF0030901AB0821384602F19C
:103F60000108FEF7D5F81FFA88F8064648BB029903
:103F70000A46032342F8049B06312846FBF7D0FB90
:103F8000044660B908213846FFF7CCFA0446112CE4
:103F90003FD01AD80CB30C2C2FD107231EE00C28CD
:103FA0000DD0052800D1344608213846FEF79CF98B
:103FB000002818BF03244246002ECDD1E7E7012692
:103FC000F2E70728E9D00446E1E7862C13D043F254
:103FD00002039C4211D100221CE0012328468DF8E7
:103FE0000430ADF80850FFF799FFADF8060001A8BE
:103FF000FFF7C8F8EFE70823F0E7092328468DF814
:104000000430FFF78BFFADF80850ADF806000394BD
:10401000EDE70122034B28461978FFF799FE05B01A
:10402000BDE8F083DEBC00200378072B02D1408876
:10403000FFF784BF704700002DE9F0434FF6FF758E
:10404000A84285B0044668D0FFF768FFA84227D190
:1040500000260327B0464FF001093B463246414651
:104060002046FBF75FFB042805464DD0082847D0C3
:104070000B282DD117F002031FD1B8F1000F20D16A
:104080001EBB032320468DF80430FFF747FFADF831
:104090000840ADF8060001A8FFF774F8002237E0E9
:1040A000002301AA0821FFF7FFF80028D0D1029BC6
:1040B00003F106089E881F68CDE701274FF000092D
:1040C000CBE703271E469846F8E703274646F5E761
:1040D000B9F1000FD5D0112819D043F2020398424C
:1040E000DCD008B90223CDE7092320468DF804303F
:1040F000FFF714FFADF80840ADF806000395CAE7D6
:10410000B9F1000FEED1BCE7B9F1000FB9D001222F
:10411000034B20461978FFF71BFE05B0BDE8F0837E
:10412000DDBC002037B50578012D044614D1408848
:10413000FFF782FF6088FFF7F1FE00236A462946F9
:10414000FFF7B2F840B9019B1B782BB1034B608895
:1041500019782A46FFF7FCFD03B030BDDFBC002014
:10416000F0B587B004460E461746FFF7D7FE4FF668
:10417000FF739842054624D01E4B20461978FFF75E
:1041800017FE80B30023CDE90033029304238DF89A
:104190000030194BADF802401978ADF804602046A4
:1041A0008DF80670FFF704FE68B12846FFF72EFE73
:1041B000124B204600221978FFF7CAFD6846FEF729
:1041C000FCFF07B0F0BD07212846FEF78DF8052853
:1041D000EED10923049003A88DF80C30ADF80E4001
:1041E000FEF7EBFFE4E73A4631462046FFF7C6FD0F
:1041F000E7E700BFB12C0020B02C0020AF2C00203E
:1042000010B5027886B004461AB1012A09D006B06A
:1042100010BD0E4B1B78002BF9D0C088FFF7F6FDC0
:10422000F5E70B4B40881978FFF792FD1422002127
:1042300001A8FBF777F96088ADF80600FFF76EFE7E
:10424000ADF8080001A8FBF7DDFAE0E770BE00203A
:10425000A0BA002070B5044686B01422002101A83F
:10426000FBF760F923786088ADF80600013B0B2B63
:1042700000F29080DFE803F02106233A4E585C6894
:10428000747A7C8C2679444B321C19784FF00105E6
:1042900018BF01228DF80450FFF75AFD731B5A42D4
:1042A0005A413E4B60881978FFF752FD6088FFF74E
:1042B00035FEADF80800002D42D106B070BD0223D6
:1042C0008DF804302379002B14BF012302238DF8CD
:1042D0000C30314B01221978FFF73AFD2F4B227930
:1042E00019786088FFF734FD0125DFE703238DF897
:1042F00004302A4B1978FFF75BFD002814BF012317
:1043000002238DF80C30A3798DF81030A388ADF816
:104310000E30E9E7204B1978FFF74AFD0028CCD191
:1043200002238DF80430DFE703238DF80430EAE739
:104330000723A2888DF80430ADF808208DF80C30E2
:1043400001A8FBF75FFAB8E708238DF80430A388CB
:10435000ADF8083007238DF80C30A3680593EFE71C
:1043600006238DF8043063680393BDE70523D8E77F
:1043700003238DF80430094B1978FFF719FD002845
:1043800014BF012302238DF80C3041F20113BEE764
:104390000423C6E7002589E730C00020A0BA00202A
:1043A0001FB50D294FF0000301930393ADF80600EC
:1043B000029108D10B2301A88DF80430FFF74AFFC2
:1043C00005B05DF804FB86290CBF0A230923F2E738
:1043D00030B508490A680023012505FA03F4224292
:1043E000D8B202D122430A6030BD0133182BF4D178
:1043F0001846F9E764BA002010B50378182B044674
:1044000002D1FFF7E5FF207010BD000010B5024B90
:10441000197DFDF72FFA10BD64BA00202DE9F04F89
:104420003D4D89B02878FFF787FC60B103A8FFF7FE
:10443000EDFFDFF8E8A0DFF8E8B00DF11009002784
:10444000039B9F4202D309B0BDE8F08F39F8024BBD
:1044500029782046FFF7ACFC064678B39AF800109E
:104460002046FFF7A5FC804640BBBBF800304FF666
:10447000FF7219462046FBF757F943F203029042B8
:1044800029D10133ABF80030EFE7052320468DF842
:104490000030FFF743FDADF802006846ADF8044078
:1044A000FEF770FEB046324629782046FFF750FCF2
:1044B00042469AF800102046FFF74AFC0137BFE752
:1044C0002046FFF72BFDFEF74BFE0026EBE72046CC
:1044D000FFF7B2FDE7E70828F2D012D80028D4D0C1
:1044E0000628EDD00923029020468DF80030ADF863
:1044F0000440FFF713FDADF802006846FEF742FEE8
:10450000D1E743F202039842CDD043F201439842EF
:10451000DDD01128E6D1C6E7DFBC0020E0BC0020DA
:104520008CC200201FB5044640882378ADF80600F1
:10453000012B10D05AB21AB1022B15D004B010BD05
:1045400001A88DF80420FEF71DFE6088FBF7F4F843
:10455000FFF772FDF2E78DF8043001A8A388ADF8EB
:104560000830FEF70FFEE9E72379002BE6D0FBF7D2
:10457000E3F84FF6FF739842E0D0044B012219781C
:10458000FFF7E6FBFFF74AFFD8E700BFDFBC0020DC
:1045900038B5074C0146207DFDF7BEF830B1A07D4F
:1045A000FDF7BAF8002814BF0220012038BD00BF73
:1045B00064BA00202DE9F0478CB089461646804643
:1045C000FFF7E6FF20228246002104A8FAF7AAFF9F
:1045D000BAF1000F46D0B9F1000F17D099F800508A
:1045E00015F001054FF6FF7415D04046FFF796FC15
:1045F000A042074639D14048FDF724FDB0F5807F41
:1046000001D0B84275D10025032470E04D468526BF
:104610004FF6FF775FE02E4627465CE04A4631467C
:104620004046FBF785F80446B9F1000F5DD000283D
:104630005DD199F8003013F0010F14BF0121022160
:104640004046FEF7DBFDB6F1850218BF01220024CB
:104650000095012339464046FFF72AFC20460CB05E
:10466000BDE8F08743F20204F8E7002502AB01221F
:1046700007213846FDF74CFD0446002837D1214676
:1046800050220398FAF74EFF039B83F800A0039C87
:10469000079604F13403049304F118030893631C90
:1046A00009934046154B0B93FFF796FBFF280CD060
:1046B000134A0C2101FB002050F8042FC4F81120EC
:1046C0008288A4F815208279E2753846FBF7DCF879
:1046D000044660B90646BAF1020F04AB9ED100222F
:1046E00031464046FBF724F80446002CABD00022AC
:1046F000AEE707460125B9E778C0002033C00020A7
:104700004EBC0020F0B585B00446FFF741FF324FA4
:10471000012806463D7831D12046FFF7FFFB4FF6D2
:10472000FF7398422AD0204632462946FFF710FBF5
:104730000023CDE90133039301A80C238DF8043045
:10474000ADF80640FFF786FD244B1B78E3B13978BE
:104750002046FFF72DFBB8B9214B22491A682046A5
:10476000FFF728FF8628054632D011280FD070B1F8
:1047700029462046FFF714FE05B0F0BD0022294669
:104780002046FFF7E5FADFE700221146E7E7A5F14B
:1047900011035E425E410022134B20461978FFF759
:1047A000D7FA124B324619782046FFF7D1FA104B50
:1047B000002219782046FFF7CBFA0E4B0022197819
:1047C0002046FFF7C5FA002DD6D0112DD4D0CFE763
:1047D00000260122E0E700BFAE2C00205FC10020D0
:1047E0001CC000205AC10020AD2C0020AC2C0020A1
:1047F000AB2C0020AA2C0020F0B587B0074601A8FA
:10480000FFF704FE02AD0024019B9C4201D307B0D8
:10481000F0BD35F8026B39463046FFF7C9FA10B1E2
:104820003046FFF76FFF0134EEE700002DE9F04F4F
:10483000054687B0904699460F4639B9A14B1B787B
:10484000F3B90524204607B0BDE8F08FFFF7A0FEBE
:104850000138C0B2012800F22D8100212846FAF764
:1048600069FF0446862C00F0B080112C00F099807E
:10487000002C00F09680B9F1000F00F0BF80B9E085
:10488000FFF786FE012800F09E80022840F012818A
:104890008D490B78284613F001048B4614BF4FF066
:1048A000010A4FF0020AFFF739FB4FF6FF739842F7
:1048B000064659463AD03B4602AA0721FEF7F4FCC9
:1048C0000446F0B9039B93F84420D10740F1C78018
:1048D000B8F1000F40F0D68003F1340202F112016A
:1048E0002846FAF723FF4FF0000A044600230093FE
:1048F000BAEB030318BF0123B4FA84F2520931461C
:1049000045E00528F2D1BDE004AB01220721304685
:10491000FDF7FEFB0446002840F0C1803046FAF760
:10492000B3FF0446002800F0B280B8E0002C41D06C
:104930006648FDF787FBB0F5807F834637D0B042ED
:1049400036D004AB01220721FDF7E2FB044650B943
:104950005846FAF799FF044628B95B492846FAF702
:10496000E9FE044638B107215846FDF7BDFC10B1F9
:10497000052818BF03244FF6FF73BBEB030318BFD2
:104980000123B4FA84F200935209012359462846C0
:10499000FFF78EFA002C7FF465AF51462846FEF7EC
:1049A0002DFCA4F111035E425E4100220FE0B346EC
:1049B0000324E0E72846FAF7BDFE009704460123EA
:1049C000B0FA80F29AE7404948E700260122404BBE
:1049D00028461978FFF7BCF93E4B3246197828462D
:1049E000FFF7B6F9B9F1000F08D0002C3FF42AAF59
:1049F000112C17D021462846FFF7D2FC0D2C3FF48E
:104A000021AF06D8002C3FF41DAF082C18BF03249B
:104A100018E7862C14D043F202039C423FF412AFF5
:104A2000112C1AD12C4B3A4619782846FFF790F9E9
:104A30002A4B424619782846FFF78AF9002401E7F5
:104A4000254B3A4619782846FFF782F9234B424610
:104A500019782846FFF77CF9F4E60324F2E6B8F16A
:104A6000000F0FD1598D03F1180200297FF436AFE2
:104A700003F12C01343311F8010B00287FF42EAF21
:104A80008B42F8D19BF80030DA073FF53DAF0E4975
:104A90002846FAF74FFE044600283FF427AF0721C7
:104AA0003046FDF721FC00283FF420AF052818BF51
:104AB00003241BE743F20204B9F1000F3FF4C2AE36
:104AC00098E700BF5FC100205AC1002078C00020D5
:104AD000AB2C0020AA2C0020A92C0020A82C002000
:104AE0002DE9F04786B00746FFF726F958B101A82F
:104AF000FFF78CFCDFF84880DFF8489002AE002515
:104B0000019B9D4202D306B0BDE8F08736F8024B08
:104B100039462046FFF74CF980B198F8001020463E
:104B2000FFF746F999F8001082462046FFF740F952
:104B30000123014652462046FFF778FE0135DFE7A4
:104B4000A82C0020A92C002010B50378062B0ED924
:104B5000072B1BD10E4B1C782046FFF7EDF810B148
:104B60002046FFF749FE0B4B1878FFF7B9FF0A4BB9
:104B70001C782046FFF7E0F810B12046FFF73CFE16
:104B8000064BBDE810401878FFF7AABF10BD00BF64
:104B9000AD2C0020AB2C0020AC2C0020AA2C002037
:104BA0001FB503780446092B09D8DFE803F0050A8E
:104BB00020202020202020204088FFF7A3FD04B0E3
:104BC00010BD144B197819B3134B00791B7803F0FF
:104BD0000102904206D86179C3F34003994294BF21
:104BE00000210121012300226088FFF71FFE2378A6
:104BF0008DF80430043434F8023CADF8063094E803
:104C0000030004AB03E9030001A8FFF723FBD6E789
:104C10000121E7E75FC100205AC1002037B5174BDB
:104C2000174A5B881188174C174D994208D852884B
:104C30009A4205D36369FBB900232B7003B030BDE2
:104C40002B783BB16369002BF6D000228DF804204D
:104C500001A80FE00D490E480978D4E90123002985
:104C60000CBF11461946FDF785F90028E4D0A36969
:104C7000002BE1D09847DFE70122E7E7AEBC002038
:104C8000B8C0002010BC0020A4BB002088C10020B8
:104C90002CBC00207BDF70477ADF704776DF7047DF
:104CA00075DF704737B5164B18884FF6FF7398427B
:104CB00010D0144A144D1378297B0133DBB299428A
:104CC00013702C4608D31149FFF7EAFF10B1AB6906
:104CD00003B1984703B030BD002313702B7C33B170
:104CE0003B21FFF7DBFF10B1AB6903B19847636964
:104CF000002BEFD000228DF8042001A8E9E700BFC7
:104D00000CBC002088C1002010BC0020B8C00020CE
:104D100065DF70472DE9F74F0C9CBDF834B027884C
:104D2000002580468A4691462E46B8F80020B242B9
:104D30000BDC35B12288013AD21B92B2FF2A39D856
:104D4000DA55002003B0BDE8F08FD8F8042052F8FF
:104D50002600019000220DF1030101A8FFF7D8FF02
:104D60000028EFD19DF803204A4521D12288002D4B
:104D700014BF0020022002EB09010144594519DC4F
:104D80003DB9013292B2228003F802A0228801329A
:104D9000228022880DF103011A4401A8FFF7B8FF11
:104DA0000028CFD121889DF803200A4422800125C4
:104DB0000136BAE70C20C5E72DE9F341089CBDF8A0
:104DC00024501746CDE9004502220646FFF7A2FF10
:104DD00048B9102239463046CDE9084502B0BDE851
:104DE000F041FFF797BF02B0BDE8F0812DE9F04F29
:104DF00000231688138090F82D3085B007460D46A5
:104E000014465BB3082E01D80C2008E102A8FAF77B
:104E100011FD002840F0038113880822CA5423881A
:104E200001339BB21B222380CA54238801339BB2D7
:104E3000CA18DDF809102380E950BDF80D309380C1
:104E400023889DF8082006339BB212F0FE0218BF9B
:104E500001222380EA54238801332380BB78FBB1ED
:104E600023880433B342CFD802A8FAF7E1FC002824
:104E700040F0D58023880322EA54238801339BB273
:104E800019222380EA542388BDF8082001339BB2FD
:104E9000E9182380EA54120A4A70238802332380D7
:104EA000FA789AB12388D91CB142ADD80221E954CD
:104EB000238801339BB201212380E95423880B44CA
:104EC0009BB22380EA5423880B4423807A68AAB1DA
:104ED0002388D91CB14297D8022192F90020E954C5
:104EE000238801339BB20A212380E95423880133AC
:104EF0009BB22380EA542388013323803B89002B13
:104F000040F081803B8A53B1CDE900462B46072211
:104F1000032107F11000FFF74FFF00287FD13B8BE3
:104F200053B1CDE900462B461522142107F1180094
:104F3000FFF742FF002872D13A6A002A72D1D7F8EF
:104F40002480B8F1000F30D0B8F804302188981CC4
:104F50008A1C0244B2423FF657AFFE283FF654AFD8
:104F600003336B54238801339BB2FF222380EA541E
:104F7000238801339BB22380B8F80020EA54E91853
:104F8000120A4A702088023080B22080B8F80420CB
:104F90005AB1D8F8081000294ED0284435F0E6FE62
:104FA0002388B8F804201344238097F82C30002B72
:104FB0007DD1387898B33B88012B3DD0228802F10F
:104FC000020CB4453FF620AF012805D17B780233AF
:104FD00013449E42FFF418AF023EB61AB6B202A9BD
:104FE00005EB0C00ADF80860FAF720FCB8B93B7887
:104FF000022B40F09F80BDF80830B34240F2B580EC
:10500000ADF808609FE0CDE900462B46062202215C
:1050100007F10800FFF7D0FE00283FF473AF05B09A
:10502000BDE8F08FB4F800C00CF10603B3423FF6C0
:10503000EBAE1188052901D80720F0E76FF4486E20
:1050400001EB0E039BB24FF27D3E7345F4D95388BA
:10505000052BF1D96FF44860181880B27045EBD970
:105060004FF6FF70814203D0834201D09942E3D8CA
:10507000052305F80C30238801339BB212212380CD
:10508000E954238801339BB223801188E954E8183E
:10509000090A4170238802339BB223805288EA5464
:1050A000E918120A4A7023880233238047E7BB6A53
:1050B000002BC1D04FF000094FF00C0A4FF0160B37
:1050C00097F82C305FFA89F293427FF672AFB96A93
:1050D0000AFB02F201EB0208B8F80430981CFE2823
:1050E0003FF692AE208803332B54238801339BB2C2
:1050F000238005F803B0238801339BB223808A5AAA
:10510000EA54E918120A4A702088023080B22080DE
:10511000B8F804205AB1D8F8081000298CD02844D7
:1051200035F024FE2388B8F804201344238009F1C5
:105130000109C5E7012B7FF463AF7B789E42FFF442
:105140005FAFADF808300821BDF80830FE2B3FF600
:105150005BAE22880133AB542288013292B22280A6
:10516000A95422881344238059E70921ECE7000061
:105170002DE9F0430646B2F8009007460D469046EA
:105180000FCE9FB06C460FC40FCE0FC40FCE0FC40E
:1051900096E8070084E807003C2200210DEB02009E
:1051A000CDE90C118DF82E108DF82D1000910E9177
:1051B000FAF7B8F93C2269460DEB020035F0C8FD5C
:1051C000002840F0C9807C6B002C34D1BB6B23B12C
:1051D00004F12400002D3ED184B23B6B23B104F1D5
:1051E0001201002D62D18CB297F82E30002B00F006
:1051F000A980E11C002D7CD18CB297F82D300BB129
:105200000934A4B2BB780BB10434A4B2FB780BB15F
:105210000334A4B23878002800F08F80012840F0D1
:1052200094807B78ADF83C300020BDF83C300233F0
:105230001C44A4B281E065B1B9F1020F03D80C207F
:105240001FB0BDE8F083022223782A7011226A7011
:10525000AB700324BAE74845F1D811222A55621CE5
:1052600092B22221A954A21C03F1170115FA82F26D
:1052700003F1270C0E4651F804EB42F804EB6145AC
:10528000F9D104F1120292B21121A95404F11302CE
:1052900092B223211434A954073315FA84F453F835
:1052A000042B44F8042BB342F9D195E74945C6D8FD
:1052B00011222A55621C92B21020A854274A16685F
:1052C000023415FA84F456B1107992F805C0844579
:1052D00040D900F1010C82F804C046F820405A1E63
:1052E000013C0F3312F8010F04F8010F9342F9D17A
:1052F00079E74945A3D8601C022280B22A551C26B2
:105300001444013B2E54A4B2032B25D8DFE803F04C
:105310000205071800232B5502E00123FBE72A555D
:105320008CB2A9EB040929190FAA3846ADF83C90B4
:10533000FFF75CFDBDF83C301C44A8F800407FE757
:105340000323E8E7002DECD157E70FA90020FAF777
:105350006DFA6AE7042073E7072071E780C1002037
:10536000F0B590F82D3085B00C461546002B44D191
:1053700090F82E30002B40D1436B002B3DD0C378EA
:105380000BB15B0739D584B32B68072B33D9083BA6
:10539000B3F5803F28BF4FF6FF7304F10806ADF860
:1053A00006300DF106023146FFF7E2FE0346F8B97A
:1053B000BDF80620083292B2ACB1110AA71C617088
:1053C000F11B89B2052902902270CDF80B0012D989
:1053D00002A8FAF72FFA50B9DDF80910C4F8021044
:1053E000BDF80D10E1802A6002E02646D9E70346A9
:1053F000184605B0F0BD0423FAE70723F8E713B514
:1054000090F82D301446CBB190F82E30B3B1436BE9
:10541000A3B9C3780BB15B0710D52368B3F5803F00
:1054200028BF4FF6FF730DF10602ADF80630FFF707
:105430009FFEBDF80630236002B010BD0720FBE7D9
:1054400007B5144B1A686AB1002018601B680093F6
:105450004FF08042009B0123C2F808330E4A53707C
:10546000FAF778FA0D4B1A688AB100221A601B68A5
:105470000193019B4FF080430222C3F80823064B9F
:105480000120987003B05DF804EBFAF763BA03B03B
:105490005DF804FB00010040F0BB00200401004067
:1054A0000E4BD3F8183182B0B3B10D4B0D4800222A
:1054B0001A601B680193019B0B4B997EFF291FBF4C
:1054C00001228A404FF0A041C1F8082500225A76F7
:1054D0001A711B6802B0184702B0704700300040D4
:1054E0001831004068BB002064BB002070B52D4C13
:1054F00086B094F82130019394F820300093E3694A
:1055000004F1260204F123014FF04020FAF740FA9B
:105510002346E0B994F82360A56906BB217B8A1E67
:10552000012A1CD8E0692269904218D16269E37BA4
:10553000E261C5F34015032984F8203084F8215036
:1055400007D100954FF040212046FAF7F8FA06B04F
:1055500070BD4FF040212046FAF794FAF7E7124A5F
:1055600007CA06AC04E90700C6B14FF04021D1F8E4
:10557000C424C1F8C42490070CD501228DF808205A
:10558000002283F824206A07E1D4D3E9002102A88D
:105590009047DCE75107F3D50222EFE78DF808606A
:1055A000EEE700BF3CBB002048BB0020F7B5154626
:1055B0004FF0FF32C1F8082390F8242004460F462C
:1055C00002F0FF0E2AB18368C1F80433112003B042
:1055D000F0BD012680F82460836100F10C0C95E891
:1055E00007008CE80700AA7884F820206A68E26146
:1055F0006A78C7F888252A78B24212D012B91E1CE0
:1056000018BF012684F821600096AB786A68394695
:105610002046FAF794FA2368002BD8D184F8243076
:10562000D5E784F821E0AB786A6839462046FAF776
:1056300029FAF0E730B54A4AD2F8043313F4007F70
:1056400085B015464AD0D2F82431002B46D04FF40D
:1056500092711046FAF7DEFA4FF40173C2F808337C
:10566000404B997E09B9012151603D4902228DF8D4
:105670000020D1F88024C1F880240392DA7D8DF8CF
:105680000820DA6801920022DA751A766846D3E9B2
:10569000001290473248D0F81C313BB1314A938A0E
:1056A000917D994247D91146FAF7E3FA2C4AD2F88C
:1056B00044318BB14FF4A2711046FAF7ABFA294B83
:1056C000997E09B101211160DA7D2AB10022DA75D3
:1056D000587ED968F9F74EFF05B030BDD5F80433D0
:1056E0005B07D7D5D5F80831002BD3D01D4C1C480B
:1056F0002146FAF7A7FA637EE27D9A422346C9D192
:10570000227E52B12369E168E3600023607EE27586
:1057100023766376F9F72EFFBCE7A27E0AB9012251
:105720006A600F4A4FF40171C2F808130022DA755B
:10573000587ED968EEE74FF48E71FAF76BFA917DD7
:105740000029B3D000238DF8081091688DF800303F
:10575000019193756846D2E900139847A6E700BF08
:105760000020004020BB0020800000F1A040D0F8C5
:10577000003723F44033C0F80037D0F8003743EA4D
:105780000141C0F8001770470E4B034493F94020C5
:10579000072A02DD0021FFF7E7BFD3B2072B10D89D
:1057A000930003F1804303F5C043D3F8101521F0B3
:1057B0000101C3F81015012303FA02F2024BC3F8EA
:1057C00008237047B4BA00200060004000F1804018
:1057D00000F5C040002382B0036003680193019B81
:1057E00002B070472DE9F04F85B00024594D019467
:1057F0004FF48072012102F1804303F5C04390B25F
:105800001B68012B06D1D5F804330B4202D0FFF7F9
:10581000DDFF0C430432B2F5907F4FEA4101EAD13B
:105820004D4B1B68012B0AD14FF4BE70FFF7CEFF22
:105830004FF0A04344F00044D3F81035019314F026
:10584000FF0F1AD0454F01260025344210D0AB007F
:1058500003F1804303F5C043D3F81005D3F81015C6
:1058600057F8253023B1C1F30141C0F30420984714
:105870000135082D4FEA4606E7D1002C63DA4FF0D8
:10588000FF330022CDE90232344D354E0024A246CA
:1058900001274FF0A04816F9012B531C46D0D2B275
:1058A00022F0C0094FEAD90104A8084402F0070316
:1058B00010F808CC07FA03F31CEA030F36D005EB07
:1058C000090C92099CF940C055F82CB0BBF1000FAF
:1058D0000AD1032A2AD10DF10C0E1EF801C04CEAA0
:1058E000030C0EF801C001E0032AF4D009F5E071C1
:1058F00010F80C0C58F821101842C1F3014105D0E2
:10590000022913D1032A0BD1114604E003290DD13A
:10591000032A05D102214846FFF726FF0134E4B2ED
:10592000BBF1000F02D011464846D8470AF1010AE0
:10593000BAF1080FAFD134B14FF0A043019AD3F8B8
:105940001035934202D105B0BDE8F08F0193039B5F
:1059500002939AE7006000407C610040B4BA0020E6
:1059600014BB00200028C3B2A8BF00F160424FEA78
:10597000501010B5BABF0D4A03F00F0402F5614292
:105980004FEA41114FEA8000C9B200F16040B4BF54
:10599000115582F8001300F5614003F01F02012346
:1059A0009340C0F88031036010BD00BF14ED00E0EB
:1059B0002DE9F8430568EB175906674B41EAD51105
:1059C00004464FF0FF3268068B4208BF82420AD37A
:1059D000624A002334F0FEFF00F5006020F47F6788
:1059E00027F00F072FB929465D48BDE8F84328F096
:1059F000EDB8207923F0F2FB40B9607923F0EEFB9B
:105A000020B95848BDE8F84328F0E0B8E279E17AD7
:105A10000D2023F073FC237B534A002B00F08A8077
:105A2000537843F01003514E5370F3781BB10023A9
:105A3000F370FAF717FE257900232846F37023F058
:105A4000CDFB20B14FF4407128461BF0ADFB6579CA
:105A5000284623F0C3FB20B14FF4985128461BF091
:105A6000A3FB637A2579002B284614BF4FF00E095B
:105A70004FF0000923F0B2FB00285FD03C4B05EB50
:105A800085051D4495F801806479204623F0A6FB26
:105A9000002856D0364B04EB84041C446378354C04
:105AA000E27E002A50D15A1C0AD04FF0A0410122B8
:105AB0009A40C1F8082503F5E072032041F822005E
:105AC000B8F1FF3F2C4D1FBF4FF0A04108F5E07229
:105AD000002041F82200C5F82475C5F86C95002710
:105AE000C5F81485C5F80C35244B636028464FF47F
:105AF0008E712760FAF78EF84FF4A271FAF78AF8E0
:105B00001F4BC5F8043302210846FFF72BFF04237F
:105B1000C5F80035B8F1FF3F4FF48073E782277670
:105B2000638315D01748FAF77DF80123A376FBF7B6
:105B30009DFA0DE0537803F0EF0374E74FF0FF3860
:105B4000A2E74FF0FF33AAE708210F4828F01EF81C
:105B50000123F370BDE8F88347E8010048E801003D
:105B6000A2AF0500B7AF05005CBA002099C20020C3
:105B70003CB0050020BB00200020004025FA0300B7
:105B8000800002007CAE0500CDAF050010B50D4CC5
:105B900000226260A2602261E2600B4A106810F08D
:105BA000010002D10621FFF7DDFE084B1B7823B967
:105BB0004FF080430122C3F81825012323700020F1
:105BC00010BD00BFF0BB002000E100E061C100207B
:105BD000F8B50E46D11C48BF911D144641F387010C
:105BE0000546671EFAF704F900214AB2A24201F104
:105BF000010100DBF8BDBB1A23F00300B25C03F027
:105C00000303DB0002FA03F32A581A432A50ECE795
:105C1000F0B500254F1E6CB28C4205F1010500DB8A
:105C2000F0BD3B1B23F0030603F003039659DB0092
:105C300026FA03F30355EEE72DE9F041B3F90240EC
:105C400014F11F0548BF04F13E050F4603F1240679
:105C500045F34715904601462B4632463846FAF73B
:105C600007F9B8B9B4EB451F16DA6211012304F045
:105C70001F0403FA04F457F822301C4214BF012415
:105C800000242B46324639464046FAF7F1F82046C2
:105C9000BDE8F0810124F4E70446F2E710B50023E3
:105CA0001A465CB2A14203DCB2FA82F0400910BD90
:105CB00050F8234001332243F3E700002DE9F04F71
:105CC0008A46234F8BB00646114650461446FAF7D3
:105CD0006FF83B68FBB10425C0EB441014FB05FBD7
:105CE00000B205FB04654FF0FF38043D28FA00F8C8
:105CF0004FF040093B6859463046984758B12B68E9
:105D000003EA08032B6021463046FFF7C7FF20B1A6
:105D1000B9F10109EED1002017E023463246514681
:105D200002A8FAF775F82146019002A8FFF7B6FF1E
:105D3000019B003318BF01235B00002814BF5842A9
:105D4000C3F10100C0B20128E2D10BB0BDE8F08F71
:105D5000602E00202DE9F04FD1B0CDE905015B9D0B
:105D600095F9004048A8914622461F46FAF714F8D4
:105D7000A3000793069BA20013441946224638A8A5
:105D80000293FAF709F895F90060002F00F08C8073
:105D90003246394628A8F9F7FFFF0DF5807A3246DA
:105DA00030AF48A95046F9F7F7FF38A93846F9F758
:105DB000F3FF2B4628AA38A948A8F9F7ACFF2B46D1
:105DC00028AA38A948A8D5F8A460B0472B4628AA25
:105DD00039465046F9F79FFFBDF968310497023BF9
:105DE0001BB2002B67DCD9F80030009503F00108E6
:105DF0004FEA481840AADB4302EB080A03F001030C
:105E000030AA90445B0140AA1A44039230AAD318E6
:105E10004146039A0493504605F10409FAF71FFA24
:105E20004B4640AA48A908A80094FAF788F908A99F
:105E300008462B464246F9F72DFF08A908462B468F
:105E4000069AF9F727FF214608A8FFF727FF002841
:105E50005DD008A8F9F7CCFF08A92B46029A08469E
:105E6000F9F718FF08A92B4652460846F9F712FF22
:105E7000DDE90301434652460095FAF772F92B46D5
:105E800008AA30A940A8F9F746FF224640A905987C
:105E9000F9F782FF059B079C234430A91846F9F7C0
:105EA0007BFF51B0BDE8F08F314628A8F9F7A0FF7D
:105EB0000123289371E71FFA83F85B1108F01F0292
:105EC00059F823300095012101FA02F21A42049B8D
:105ED00013BF20270027202600260AEB070B1F44AC
:105EE0000AEB06030393049B039A1E443346394688
:105EF0005846FAF7B4F908F1FF383B4600955A4680
:105F000031460398FAF72DF90FFA88F369E710AFD5
:105F1000224608A938460DF1600BF9F73DFF20AE87
:105F200049465846F9F738FF30462146F9F760FFF1
:105F3000012328A82093F9F75BFF224659463846EB
:105F4000F9F715FF28B9224620A908A8F9F724FF78
:105F500082E73B68DA0709D421463846F9F7FAFEAA
:105F6000224649463046FAF7CEF8E6E7189BDB07AB
:105F700007D421465846F9F7EDFE2246494628A89F
:105F8000F1E7002823461CDD5A4639463846F9F722
:105F90003FFF21463846F9F7DDFE224628A9304664
:105FA000F9F7E5FE002805DA23464A463146304631
:105FB000F9F75EFF234628AA31463046F9F728FF55
:105FC000CEE73A4659465846F9F722FF2146584649
:105FD000F9F7C0FE2246314628A8F9F7C8FE002886
:105FE00005DA28A923464A460846F9F741FF28A9B9
:105FF000234632460846F9F70BFFBEE72DE9F04786
:1060000093F9006092B00446894610463146154621
:106010009846FFF743FE002840F0918042464946EB
:106020000AA8F9F774FE43460AAA214602A8F9F71E
:1060300031FE0AA908464246F9F769FE43462A4658
:1060400049464846F9F726FE08F104074246294624
:106050002846F9F75CFE3B462A4621462046009634
:10606000FAF7E4F83B462A46294628460096FAF70E
:10607000DDF83B462A46214628460096FAF75FF8A7
:1060800043462A4621462046F9F704FE3B4622466F
:10609000214628460096FAF7C9F83B4600962A465C
:1060A00021462046FAF7C2F82368DB074AD5334673
:1060B0003A4621462046F9F7DBFE31468246204625
:1060C000F9F748FE06F18043013B54F8230040EA0B
:1060D000CA7044F82300424621462846F9F717FEC5
:1060E0003B4602AA294628460096FAF728F83B467E
:1060F00002AA294628460096FAF721F802A908467E
:106100003B462A460096FAF71AF8434602AA214669
:106110002046F9F7BFFD0AAA3B46104621460096E5
:10612000FAF70DF8324629462046F9F735FE49467A
:106130002846F9F731FE0AA94846F9F72DFE12B0B4
:10614000BDE8F08731462046F9F704FEC3E70000BA
:1061500073B500230DF102008DF80230FBF71CF837
:10616000264B1B7803F0FF04002B41D1244B1A6807
:10617000002A3DD0234AD2F80813C90738D51C603D
:106180001B68214D01930DF10300019BD2F80865B6
:106190008DF80340FBF700F86A6829681F2A98BF4A
:1061A000541CA142F6B26C6004D1202C14BF611CB7
:1061B0000021296015499DF803008E542A689442F5
:1061C0003ABFC2F121021319A31AAA689A4238BF32
:1061D000AB60FBF7B9FE6B682A681F2B94BF0133D5
:1061E00000239A4201BF074A0123C2F808335360D3
:1061F0009DF80200FBF7A8FE02B070BD61C100204F
:1062000000D1004000D000404CC1002028C1002037
:1062100030DF70472DE9F74F3B4F06468846B8F10F
:10622000000F03D1012003B0BDE8F08F4546202DBB
:1062300028BF20255FFA85FB002400230DF1020012
:106240008DF80230FAF7A8FF304B1B7803F0FF09F6
:1062500093BB0DF103008DF80390FAF79DFFD7E98A
:1062600000148C4204D3641AA54207D9052414E013
:106270002134641AA542F9D8C1F12104244BA54266
:10628000194431D82A46304634F070FD3B682B441F
:10629000212B28BF00233B6000249DF80300FBF75F
:1062A00053FE1C4B00221A601B680193019B1A4B82
:1062B0000122C3F804231A609DF80200FBF744FE94
:1062C000B9F1000F08D059463046FFF7A1FF42F25E
:1062D000070398420446ADD0022CAED0002CA9D1C1
:1062E000A8EB05082E449AE72246304634F03EFDDE
:1062F000074BA5EB040A52461946301934F036FD17
:10630000C7F800A0C8E700BF4CC1002061C1002051
:1063100028C1002000D1004000D0004017B4314A0D
:10632000314B116889B90021304A106820BB002028
:106330005A79D40740D408B9002949D01C68DA88B2
:10634000234603B05DF8044B184700211160126822
:10635000D9680092009A0029E5D0254AD2F8400574
:10636000814204BFD88801EB8001C2F840155A79F8
:1063700042F004025A71D7E7002010601268986852
:106380000192019A0028D2D0194AD2F83845A04289
:1063900004BFDC8800EB8400C2F838055A7942F06B
:1063A000020214075A71C3D512F0010402BF64F34C
:1063B000C3025A712046BBE702F00601062907D145
:1063C00022F0060211075A7106D56FF3C3025A7103
:1063D00003B05DF8044B7047054AD2F83805D2F88F
:1063E0004015ABE714510240A4BA0020045102400A
:1063F00000500240A5DF7047A4DF7047A3DF70475D
:106400002DE9F0470E4690B016F0100581469246F1
:106410009846189C0CD011238DF8083023788DF8FD
:10642000093001224FF0000362F342038DF80A3075
:106430001C22002109A8F9F775F88DF8246005B130
:1064400002AD42F64D23ADF80C3063789DF8641030
:106450008DF804300022A3788DF80530134661F3DF
:10646000C303DBB243F00303CDE906220E950127F7
:1064700001AD8DF80630089203AE1A9BB9F8000002
:106480008DF80E7004AA09A9CDE90465ADF81CA029
:10649000FDF708FC58BB42F60813ADF80C306378E2
:1064A0008DF80430A3788DF80530034667F3420376
:1064B0008DF806301A9A98F800308DF8003098F868
:1064C0000130CDF81A00ADF81E008DF8013032F819
:1064D000080B8DF80E70022304A9CDE90465ADF810
:1064E0001830ADF81C30CDF820D0FFF787FF10B082
:1064F000BDE8F087A1DF704708B5F9F789FF10B153
:106500004F4B504A1A60F9F763FF28B14E4B4F4A80
:106510001B68C3F342331360F9F77AFF20B14C4A8A
:10652000D36823F08073D360F9F752FF40B14FF086
:1065300080430022C3F80C21C3F81021C3F838258A
:10654000F9F766FF10B1434B03221A60F9F760FFB9
:1065500040B1414B05221A6001229A6700229A60DD
:106560003F225A603D4B1B78062B50D13C4B1B6899
:106570001B074CD13B4B1B6803F0F003502B46D15B
:106580004FF08052384BD2F80414C3F82015D2F8DB
:106590000814C3F82415D2F80C14C3F82815D2F83F
:1065A0001014C3F82C15D2F81414C3F83015D2F80F
:1065B0001814C3F83415D2F81C14C3F84015D2F8D7
:1065C0002014C3F84415D2F82414C3F84815D2F89F
:1065D0002814C3F84C15D2F82C14C3F85015D2F86F
:1065E0003014C3F85415D2F83414C3F86015D2F837
:1065F0003814C3F86415D2F83C14C3F86815D2F8FF
:106600004014C3F86C15D2F84424C3F87025F9F788
:10661000DFFE28B1154B164A1B6803F04F031360C9
:10662000144AD2F8883043F47003C2F88830BFF3BC
:106630004F8FBFF36F8F104B104A1A6008BD00BF19
:1066400074C007400DF0ADBA440200103C05004094
:10665000F0ED00E0A005004010560040E00F00F013
:10666000E40F00F0E80F00F000C0004058020010F6
:10667000E40E004000ED00E0A42C00200090D003C8
:10668000002382B0036003680193019B02B070474E
:106690002DE9F341844BD3F8042162B3D3F80033DE
:1066A0009F0728D5814D8248FFF7EAFF2B7803F03A
:1066B000FF08F3B97F4F804E7B783C4603F0FF0222
:1066C000002B00F0AF8073684046984701A88DF812
:1066D0000480FAF761FD7B689DF8040001337B605C
:1066E000FBF732FC754B0122DA601A60744B002212
:1066F0001A6001232B706C4BD3F81821D2B1D3F858
:106700000023560616D5D3F824356E48DB08C3F3AC
:10671000080113F4FF7F18BF0239FFF7B1FF624B86
:106720004FF48052C3F808254A1EFE2A40F2A48086
:106730000122DA615C4AD2F81031D3B1D2F80033C9
:10674000DD0616D56048FFF79BFF1023C2F808331B
:106750005E4BC2F81035FF23C2F814350123D36114
:106760005B4B1C682CB15B4800231A460321006870
:10677000A0474D4AD2F84C3133B3D2F800331C0352
:1067800022D55548FFF77CFF4E48FFF779FF534865
:10679000FFF776FF4D4BC2F81035FF23C2F81435D2
:1067A0000123D3614FF48863C2F804330D23C2F888
:1067B0000C34C2F80434464B1C682CB14548002305
:1067C0001A4619460068A047374AD2F828315BB10B
:1067D000D2F80033580507D54048D2F80C34FFF7FB
:1067E0004FFF0D23C2F80C342F4AD2F81C31B3B13D
:1067F000D2F80033190612D53948D2F80414FFF73D
:106800003FFFCB0707D5374B197821B10121C2F8DB
:10681000041400221A70244B0D22C3F8042402B081
:10682000BDE8F0810DF103008DF80320FAF7B4FC08
:10683000BA68134683B93260A660636833B92A4BDD
:106840001B7803F0FF025BB1F9F798F863689DF8D5
:1068500003000133636043E7B342EED01B68E9E70E
:10686000224B1A601B680193019B4FF08043012269
:10687000C3F804231A60E9E7144A1078502803D1BA
:10688000184901220A7054E711480468002C3FF4AB
:1068900051AF4FF6FF70C3F808050E480B4600686D
:1068A0000221A04746E700BF00500040DCBC0020AA
:1068B00004510040F0BB002004BC002000B00140A7
:1068C0005C2E0020185100401051004080BE002076
:1068D0008CBF002090BF00204C5100402851004048
:1068E0001C51004060C1002061C100200001004037
:1068F00013B5284B2849D3F83C3413F0030345D192
:106900000A680132072A0A602CD9244A012414613A
:106910000DF107008DF80730FAF73EFC204B5A685E
:10692000013A5A605A6822B91E4A127802B3F9F73E
:1069300023F89DF80700FBF707FBBFF35F8F1A4AA8
:1069400000231360BFF35F8F01211160174A1468A1
:106950001CB117481A460068A047164B00221A704F
:10696000FAF7B8FB0D4B0022C3F8402102B010BD6E
:10697000114A4FF080411460D1F80C2402F001124A
:10698000B2F1011FF8D000225A70D2E700230B6049
:10699000E8E700BF005000405C2E002000B001403E
:1069A000F0BB002061C10020FC5F00408CBF0020D4
:1069B00090BF0020DCBC002004000040D0E901238F
:1069C00093423FBF026842F82310836801333ABF05
:1069D00083600020042070472DE9F04F87B00D46FA
:1069E00093460190C8B1C2B103680393ABB14FF0B5
:1069F0000009C846019B9B68434503D8CBF800902B
:106A0000002022E0B8F1000F09D1012B0CBFC023F8
:106A10008023039A52F8284044B90E2015E008F16B
:106A2000010293420CBF40230023F2E76178227AEF
:106A3000571869B9971D002D44D0DBF80020A2EB50
:106A40000902BA42029205D2042007B0BDE8F08FD5
:106A50000737F0E72B702278AA4613430AF8023B67
:106A6000227A6A7062783ABBAE1D227AE1683046BB
:106A700034F07CF9237A62781E442AB1304661688A
:106A800034F074F963781E44029BDB1B0593236981
:106A9000002BC2D005AA3146606998470028D4D19E
:106AA000059B16B11ABACAF800201F44B94405B1B3
:106AB0003D4408F101089DE743F00803EE1DAA716B
:106AC0002B70D2E7AA462E46E1E710B5144661B115
:106AD00013689BB14378027803F00F0343EA021373
:106AE00001F8013B2368013B236022464068FFF721
:106AF00073FF10B923680133236010BD0420FCE745
:106B000070478DDF704777DF7047D0E91F32816FA4
:106B10001A44D0F88430C0F880200B4490F821103B
:106B2000C0F88430C9B1016F002ABCBF5218C0F848
:106B30008020D0F880208A42A4BF521AC0F880205A
:106B4000426F002BBCBF9B18C0F88430D0F8843053
:106B50009342A4BF9B1AC0F884307047D0F88030AD
:106B6000C0F88830D0F88430C0F88C3070470368A3
:106B7000C91A436870B5D21AD0E91E6302FB03F448
:106B8000724301FB064501FB1322D0F88040D0F888
:106B900084302C441A44C0F88040C0F8842070BD72
:106BA0002DE9F04F89B00E4600AF0023044607F1EF
:106BB000140130467B612CF0F7FD05465EB318BB2F
:106BC00030462AF01FFE8046786125F049FE08F520
:106BD000807383420CD9A949012027F017F9324666
:106BE000A749012027F012F92437BD46BDE8F08FF0
:106BF00008F1070323F00703ADEB030D6D46424692
:106C0000294630462AF022FF7E693EB99D4901207F
:106C100027F0FCF8E8E70028F6D1E0E74FF003089A
:106C2000B6FBF8F303EB43039E4201D09649EEE72F
:106C3000204622F0D3FA08B99449E8E7944BC7F804
:106C400008D004EB84041C446378924C2179002919
:106C500040F00B81904A0120C2F80415FF2BC2F8C6
:106C60002415C2F82015C2F81C05C2F82815C2F870
:106C700018154FF0C051C2F81415C2F810054FF0A6
:106C8000A04118BF03F5E070C1F85887C1F8FC8A2D
:106C900018BF41F820804FF01601C2F864154FF07C
:106CA000FF01C2F8681508BF4FF0FF334FF0FF3106
:106CB000C2F860152520C2F87035C2F86C15774B04
:106CC00023600221FEF74EFE012323710323B6FB4E
:106CD000F3F39BB203EB430808F1010828F001022B
:106CE0009100ADEB010D6846FA606D4A3A604118BB
:106CF0004FF0000C796082F800C0E91C4FF0EE09FB
:106D0000851C4FF0880A4FF08E0B63455FDC0C2228
:106D100002FB030300227968994200F29E802679E3
:106D2000012E40F0A28000F06043B3F1005F40F01C
:106D3000A280FB68C3F34E02574B0021C3F85025D5
:106D4000C3F83815C3F80815C3F84005C3F80C6537
:106D50006579E28025F0090545F008056571C4E90B
:106D60000210C3F80065022323710D46002977D075
:106D70004FF6FE7208EA0202F8F7D4FB494B0022F4
:106D80001A601B68FB61FB69474B1A601B68BB619B
:106D9000BB69414B2222C3F8042301221A603A68DE
:106DA0001278042AFBD94149002222250120C3F888
:106DB00008530860C3F80025C3F808530860C3F8F7
:106DC00000253B4B2021C3F88410227150E011F8BC
:106DD000026C11F8032C360246EA024611F8012C27
:106DE00005F10C0E164306F44012B2F5001F1ED03A
:106DF000B2F5401F20D0B2F5801F20D105F802BCAB
:106E000006F44002B2F5000F1CD0B2F5400F1ED0C0
:106E1000B2F5800F1ED105F801BC0235AE454FEA30
:106E20000616E0D10CF1010C033175466DE76FF0E9
:106E3000170205F8022CE3E705F8029CE0E705F8E5
:106E400002ACDDE76FF0170205F8012CE5E705F865
:106E5000019CE2E705F801ACDFE703F8012B5AE7F4
:106E6000014623682846984788E70820FBF70AF878
:106E7000D7F808D0B8E61020F8E700BFEAD7050039
:106E800011D805003DD805005DD8050088D805005B
:106E90003CB00500A4BA0020005002409D880300C9
:106EA000F8C2002004510240145102400450024034
:106EB00000E100E010F5A24F0FD006DC10F5A34F63
:106EC0000ED04142084826F081BE10F5A14F09D0EE
:106ED00010F1220FF5D1054900E005490548F2E718
:106EE0000549FBE70549F9E79AD4050076D4050082
:106EF0008BD405007ED3050050D4050062D4050074
:106F00002DE9F04FADF51B7D00AF144605460E464A
:106F10001022002107F118009B46F8F703FB2046DA
:106F20002BF029F8002850D00022BC4920462DF033
:106F3000F7FA804638B1102207F118012AF086FDD1
:106F400040462BF067FF20460022B5492DF0E8FAB5
:106F5000044670B94FF0010920462BF05BFFB9F1F0
:106F6000000F39D10026304607F51B77BD46BDE836
:106F7000F08FAC492CF0E4F90028EBD1AA49204667
:106F80002CF0DEF9A8B9A94920462CF0D9F998B916
:106F9000A74920462CF0D4F988B9A64920462CF000
:106FA000CFF9814670B92246A349012026F02EFF71
:106FB000D2E74FF00209CFE74FF00309CCE74FF0DB
:106FC0000409C9E74FF00509C6E71CB19B4826F044
:106FD000FDFDC7E74FF001094FF48C72002107F166
:106FE0003800F8F79FFA002307F1140128467B6167
:106FF0002CF0DAFB0446002D50D0D8B928462AF0F0
:1070000001FC8046786125F02BFC08F580738342F3
:1070100004D98B49012026F0F9FEA3E708F1070304
:1070200023F00703ADEB030D6C464246214628468C
:107030002AF00CFD002307F1100130463B612CF0D3
:10704000B3FB05466EB3B0B930462AF0DBFB804691
:10705000386125F005FC08F580738342D9D808F122
:10706000070323F00703ADEB030D6D4642462946A7
:1070700030462AF0EBFC3E69F600BBF1000F13D05E
:107080003246294607F138001BF02AF98046B8F14C
:10709000000F72D04046FFF70DFF63E70028C9D10B
:1070A00060E70028E7D15DE74FF48C72594607F599
:1070B000A870F8F737FA07F140033246294607F57A
:1070C000A870FB631BF00CF98046F8B9D7F8501193
:1070D000D7F85401B9630B01C218C3583B64536815
:1070E0007B649368BB64D368FB64564E4B1E7B6025
:1070F000103A07F150037968002913DC1168196010
:107100005168596091689960D268DA60002340F252
:107110001912184607F5A871194401339342B6D0E5
:107120000870F7E7A2F1040E03F1100A5EF8040FED
:107130004549C5B216F805C0050E51F82CC0755D5D
:10714000424951F8255042498CEA050CC0F3072505
:10715000C0F30740755D305C51F825503D4951F84A
:1071600020008CEA0505454043F8045B5345DDD11A
:10717000796801397960103ABDE707F10C01786947
:10718000C7F80C80F9F71EFEFD6806460DB93248B7
:107190001DE709F1FF39B9F1040F00F22681DFE89C
:1071A00019F00500A200D60024012201D7F814A08E
:1071B0001AF00F0F40F01C81BBF1000F4ED0013DC3
:1071C0000F3405F10109BAF1000F4FD007F1180192
:1071D000A4F1100328468B4613F801CF11F8012BB8
:1071E0009C4282EA0C0200F8012FF5D14A4649463A
:1071F00007F138001AF018FF4A465B4605F1110EF8
:10720000106851689C46ACE803000832724563463A
:10721000F6D1AAF1100A10351034D2E7DBD30500FD
:107220003BF40500DED30500E2D30500E6D30500FC
:10723000EAD30500EED30500F2D3050009D405001A
:10724000EAD7050024BC050024BD050024C90500BB
:1072500024C1050024C5050033D405000F35A24420
:1072600007F5A8795445A5F10F0215D1002340F286
:107270001912184607F1380119440133934240F0BE
:10728000BA80B8F1000F3FF46EAE4046FFF712FE31
:1072900030462BF0BFFD65E62346CE4604F1100BC9
:1072A00018685968F446ACE8030008335B45E646C5
:1072B000F6D1214607F138001AF058FD07F1180100
:1072C000A5F110038C4613F8010F11F8012B9D4214
:1072D00082EA00021A70F6D199E80F0010348CE8A7
:1072E0000F001035BEE77B69E3187B6007F5A87ACD
:1072F00007F118097B68A342B8D099E80F008AE823
:107300000F004A46494607F138001AF08DFEBBF1DE
:10731000000F02D123788AF8103099F8003014F861
:10732000012B534005F8013BBBF1000F01D08AF857
:10733000103007F25113CC4607F2611E18685968E5
:10734000624603C2083373459446F7D1D2E707F586
:10735000A87B10220021584607F1280AF8F7E2F826
:10736000102200215046F8F7DDF87A694FF0000945
:10737000A3189C423FF47AAFB9F1000F0BD01AF872
:10738000092014F8011B09F101094A4005F8012BF5
:1073900009F00F09EDE75946524607F138007B60C6
:1073A0001AF042FE7B6807F5B07111F8012D013229
:1073B000D2B20A70002AE2D15945F6D1DFE7FA6865
:1073C00061192A4407F13800BBF1000F08D01AF008
:1073D0002BFE10357A6905F10F039A42EFD845E785
:1073E0001AF0C4FCF5E70025F4E7DFF810803DE76C
:1073F0006FF021083AE708703CE700BF80AFFFFF5D
:107400000023FFF77DBD0123FFF77ABD70B5002291
:10741000104905462DF084F82DF0CAFB0E4B0F499C
:107420000646032258682DF07BF8044630B100224E
:10743000B1B22CF0B8FF20462BF0ECFC084B1868DA
:107440002AF014FB00210446284614F06BFA20466B
:1074500070BD00BF02CE0500482E00200FCE0500F3
:10746000B8C2002010B5838AC3F30C0413F4604340
:1074700001D1204610BDB3F5005F02D10620604364
:10748000F8E71B0407D50022044900682DF048F8EE
:107490002DF08EFBF3E70020ECE700BF48D6050097
:1074A00008B540B2FFF72FFB40F2EA71BDE8084093
:1074B00013F09ABE38B5054608460C462AF076FD0C
:1074C000002808BF002422460F4928462CF0E4FF7C
:1074D0000E4B4FF6FF72198884B18A4206D1002004
:1074E00040F63551BDE8384013F07EBE00221888C2
:1074F000114614F08DFA0828F2D1F0E78A42EED056
:10750000188814F083FAF6E7EBCD0500682D00200B
:10751000014B188813F07CBE682D0020014B1888A1
:1075200013F076BE6A2D002008B5084B1A884FF676
:10753000FF71914209D018881321FDF7AFFB4FF47A
:10754000F171BDE8084013F04FBE08BD6A2D002060
:1075500007B500230846072269460093CDF803309B
:10756000F9F7FEF90A4B1A884FF6FF7191420BD0DA
:1075700018886A46012114F077FA40F6DF3113F0DB
:1075800033FE03B05DF804FB43F20200F5E700BFF1
:10759000682D002038B500220E4905462CF0C0FFAA
:1075A0000446A8B90C4924F02FFD0A4904460246B6
:1075B00028462CF071FF2A46084920462CF06CFF23
:1075C00000202BF00BFB0649024620462CF07BFFE7
:1075D000204638BDA2CD0500A7CD0500C1CD0500D0
:1075E000E1CD0500F8B5044628B9244A136823F410
:1075F00080431360F8BD22492BF0A2FE0028F4D18D
:1076000020462AF0F9FC0546A0B11C4A1368204622
:1076100043F4804313602DF051FE53EC102B10EE19
:10762000100A194616F07CFA40F6E121BDE8F84050
:1076300013F0DABD20462AF09EFC0028DAD00F4A6B
:107640001049136843F48043136020462A462CF007
:1076500067FF2EF021F92A4606460F4620460A49C2
:107660002CF05EFF2EF018F902460B4630463946E4
:1076700016F056FA40F6E721D8E700BFBCC200205A
:107680007FD1050084D1050090D10500084B1A6810
:1076900018B142F400521A60704722F400521A6086
:1076A000044B1860044B01221A7013F033BB00BF67
:1076B000BCC20020FCC20020FAC20020F0B583B09A
:1076C000044600AF28B9014613F060FB0C37BD46F5
:1076D000F0BD2AF047FE28B120462CF0C7FC04215B
:1076E000C0B2F1E77860391D20462CF05DF8054600
:1076F000F0B920462AF086F80646786025F0B0F802
:1077000006F58073834208D90D49012026F07EFBDF
:107710000C49012026F07AFBD8E7F31D23F007037C
:10772000ADEB030D6D463246294620462AF08EF910
:1077300079680029ECD0284613F05AFBC6E700BF51
:10774000EAD7050060DA050008B5044B044958681B
:107750002DF0E8FABDE8084013F082BB482E002067
:10776000A0DA0500F0B583B0044600AF13F078FB53
:10777000002C60D00023391D20467B602CF014F8CB
:10778000054610BB20462AF03DF80646786025F0F5
:1077900067F806F5807383420CD93149012026F041
:1077A00035FB3049012026F031FB002420460C3700
:1077B000BD46F0BDF31D23F00703ADEB030D6D4691
:1077C0003246294620462AF041F978680028E8D058
:1077D0002BF0D4F8044608B92349E3E7234B2449A6
:1077E000024658682CF058FE20462BF013FB20462A
:1077F0002AF028FC7A68294633F0B8FA20462AF0A5
:1078000021FC054620462BF0A6FF0146284613F032
:1078100037FB0023391D0A207B60F9F7D3FA7B6818
:107820000446002BC2D0134A116819605168596090
:1078300012891A81BAE720462BF0A0F8044620B935
:107840000949012026F0E2FAB0E7084B0849024650
:1078500058682CF021FE20462BF0DCFACEE700BF62
:10786000EAD7050060DA050077DA0500482E002027
:10787000A0DA05007FBF0020F0B583B0054600AF59
:1078800048B9384B384958682DF04CFAFFF75CFF7F
:107890000C37BD46F0BD0023391D7B602BF084FF03
:1078A0000646F0B9284629F0ADFF0446786024F07A
:1078B000D7FF04F58073834208D92C49012026F0B4
:1078C000A5FA2B49012026F0A1FAE1E7E31D23F0F8
:1078D0000703ADEB030D6E462246314628462AF0DB
:1078E000B5F878680028ECD013302BF047F805463F
:1078F00008B92049E6E71B4B1B49024658682CF0A3
:10790000CBFD28462AF09EFB044628462BF082FA3F
:10791000194B224603F1100153F8040B42F8040BF3
:107920008B42F9D11B8813807D6831462A4604F1C9
:10793000120033F01BFA65742544FE23AB7400205B
:10794000FFF710FF394605462BF02EFF28B10368DC
:107950002360436863600389238128462BF05AFA29
:1079600096E700BF482E002058DA0500EAD7050048
:1079700060DA050077DA0500BABB0500F0B5ADF5B1
:10798000037D064600AF50B9334B344958682DF09B
:10799000C9F9FFF7D9FE07F50377BD46F0BD00230F
:1079A000391D7B602BF000FF0446F0B9304629F00A
:1079B00029FF0546786024F053FF05F58073834264
:1079C00008D92749012026F021FA2649012026F06E
:1079D0001DFAE0E7EB1D23F00703ADEB030D6C464A
:1079E0002A46214630462AF031F87B68002BECD03D
:1079F0004FF400721C4D3A600022AA601B4A1C49D9
:107A00001460DBB228465360FEF7D8FF38B9AB6884
:107A100093B13A4607F108012846FEF7DDFF40F62C
:107A2000CC0113F0E1FB0028B5D138682AF0A6FF9D
:107A3000044618B90F49C9E70720F0E72AF002FB0E
:107A40003A6807F1080133F091F92046FFF714FF77
:107A500020462BF0DFF99EE7482E002058DA05007B
:107A6000EAD70500E2D90500842D0020B0C200202D
:107A7000142D0020F9D905002DE9F043E1B00546A9
:107A800000AF58B95E4B5F4958682DF04BF9FFF7CE
:107A90005BFE07F5C277BD46BDE8F0830023391DC4
:107AA0007B602BF081FE0646F0B9284629F0AAFE3D
:107AB0000446786024F0D4FE04F58073834208D92C
:107AC0005149012026F0A2F95049012026F09EF9E3
:107AD000DFE7E31D23F00703ADEB030D6E462246FF
:107AE0003146284629F0B2FF7B68102BECD107F114
:107AF00008044FF480733C220021204607F144051E
:107B00004FF001083B604FF00209F7F70BFD40F220
:107B100001433C2200212846BE637B8187F8089000
:107B200087F8358087F83680F7F7FCFC7E67384E9B
:107B3000384BBB67736938495B6887F84680002219
:107B40009A60736987F844905868FEF737FF0028F9
:107B50003AD1736931495868FEF730FF002833D1B4
:107B60002F4B304A1B781370DFF8D0802E4AC8F8AC
:107B70001440003318BF012388F801302B4B2C4CE4
:107B80001B78DFF8BC901370003318BF0123A0608E
:107B900031462046C9F8145089F80130FEF70EFF2F
:107BA00090B941462046FEF709FF68B9494620468C
:107BB000FEF704FF40B91F4B3A461860988007F162
:107BC00080012046FEF708FF40F6910113F00CFB00
:107BD00000287FF45EAF38682AF0D0FE044608B96A
:107BE000154972E72AF02EFA3A6807F1800133F05E
:107BF000BDF82046FFF740FE20462BF00BF948E782
:107C0000482E002058DA0500EAD7050026DA0500DC
:107C10003C2D002012DB0500E82C0020BC2C0020AD
:107C20002F2D00200CC300200DC300202E2D00207E
:107C3000302D002080C10020F9D90500902D0020B2
:107C40006C2D00202DE9F04182B0054600AF50B9FF
:107C50004E4B4F4958682DF065F8FFF775FD083712
:107C6000BD46BDE8F0812AF0A8FA28B92A4649495C
:107C7000032026F0CBF8F2E70023391D28467B606D
:107C80002BF092FD0446F0B9284629F0BBFD0646CC
:107C9000786024F0E5FD06F58073834208D93E49FB
:107CA000012026F0B3F83D49012026F0AFF8D6E7D1
:107CB000F31D23F00703ADEB030D6C46324621465E
:107CC000284629F0C3FE7D68002DECD007223449F8
:107CD000204633F03DF860B9073D07347D604FF032
:107CE000030878681B302AF049FE064680B92D4902
:107CF000DAE708222C49204633F02AF828B9083D53
:107D000008347D604FF00408EBE74FF00008E8E727
:107D10001E4B1F49024658682CF0BEFB30462AF025
:107D200091F9054630462BF075F8204B2A4603F1B1
:107D3000180153F8040B42F8040B8B42F9D11B884D
:107D400013807E6885F819802146324605F11A00B5
:107D500033F00CF8F3B203F108022E440133EB7553
:107D6000FE236A740020B376FFF7FCFC3946044614
:107D70002BF01AFD28B103682B6043686B60038900
:107D80002B8120462BF046F869E700BF482E0020E3
:107D900058DA050076D90500EAD7050091D9050023
:107DA000A8D90500B9D90500B0D90500BABB0500AE
:107DB00010B504462AF0FAF8094B0A49002808BF12
:107DC0000024224618682CF067FB201C18BF0120F5
:107DD00013F020FE40F2CC71BDE8104013F004BA5D
:107DE000482E0020EBCD05002DE9F74F464B4749C3
:107DF0000746032258682CF093FB064600283CD027
:107E000000224349DFF8088138462CF089FB3146CF
:107E10008146684625F08CF8009CF4B120462CF091
:107E200007F90022414605462CF07AFB0123002287
:107E300049468246F8F768FC10BBB5F80B3003F5ED
:107E40000073A5F80B302C46504629462CF055F807
:107E5000684625F05CF8002CDED000982AF0DAFFA6
:107E60003946002C4CD001A825F062F8019D4DB98F
:107E70003246494620462CF033F803B0BDE8F08F77
:107E80000024E1E7B5F80B3003F50073A5F80B30DB
:107E900028462CF0CDF801222946074620462CF032
:107EA000D2FC1C49804628462BF04AFA1A498246E1
:107EB00028462BF045FABAF1000F00D170B14046C8
:107EC0002CF0B6F88346B0B1BAF1000F0FD0012202
:107ED00039462EF09CFF58462AF09CFF40463A4611
:107EE00029462BF0FDFF01A825F011F8BEE7394621
:107EF0002CF0F2FCEFE7394640462BF03FFFEDE770
:107F000030462CF007FAB3E7482E002033CF0500A7
:107F10008DD005003ACF050043CF0500F8B50546E2
:107F200008460C462AF027F80646D8B100222B490D
:107F300020462CF0F5FA2CF074FF00220646284962
:107F400020462CF0EDFA044698B12AF00BF880B9DF
:107F500020462AF05FFF224622490320BDE8F84070
:107F600025F054BF2CB122461F49032025F04EFFB7
:107F7000344628462AF01AF840B33DB348F2480187
:107F80001A482AF011FE074688B1224600212CF03B
:107F900066FD2A46164938462CF07EFA154B1649DE
:107FA00018683A462CF078FA38462AF033FF281C35
:107FB000314618BF012012F0E3FF40F2DC6113F0FC
:107FC00013F92046BDE8F8402AF024BF094B0A49BE
:107FD00018682CF0A7FE0025E9E700BFA6D1050030
:107FE0004FD00500ADD10500E1D105004585020067
:107FF000FAD10500482E0020FFD105002DE9F843F5
:1080000080460C4629F0D2FF30B92F494246012064
:10801000BDE8F84325F0FABE204629F0EDFF0546FD
:108020002046C5B12DF04AF957EC106B00243246BA
:108030003B463046394632F01FFC30B90022234B14
:108040003046394632F0F0FBC8B121490120BDE885
:10805000F84325F0DBBE29F08EFF50B12A461D49BA
:1080600020462CF05DFA40B12DF016FC06460F4676
:10807000DDE714B122461849C9E7184F0026184D0C
:10808000D5F804902AF09AFD1649024648462CF08D
:108090001AFA4246144968682CF0FEF90821134880
:1080A0002AF082FD054628B12146FFF737FF284612
:1080B0002AF0B0FE32463B460D4820F0E9FEBDE80E
:1080C000F8432AF0A7BE00BFC9CE05000000244037
:1080D0001ACF050022CF0500F7CE050000409F40D3
:1080E000482E002033CF05002ACF0500E97D02008D
:1080F000F580020037B5144C00210846FFF70EFF4B
:108100000322124960682CF00BFA002201901049FA
:1081100060682CF005FA0D49054660682CF002FEF7
:108120000B4960682CF0FEFD019B33B12DB101239A
:1081300001AA2946002020F0C3FE294601982BF011
:10814000DCFE03B030BD00BF482E002033CF050059
:108150002ACF05001FB54FF08052D2F8A430D2F8D4
:10816000A820D8B20290C3F307200190C2F30721E0
:10817000C3F3074000901B0ED2B241F0C001034888
:108180002BF0FEF905B05DF804FB00BF4FCF0500F2
:1081900038B52AF016FD1E4D044628682AF026FD43
:1081A0001C49024620462CF08EF968682AF01EFD14
:1081B0001949024620462CF086F9A8682AF016FDD7
:1081C0001649024620462CF07EF9E8682AF00EFD9A
:1081D0001349024620462CF076F928692AF006FD5C
:1081E0001049024620462CF06EF968692AF0FEFC20
:1081F0000D49024620462CF066F9287E2AF0EEFC56
:108200000A49024620462CF05EF9204638BD00BFE0
:10821000C8C200202FD7050028DD050032D7050091
:1082200036D705003AD705003ED7050042D70500EE
:108230002DE9F04786B00D46014601A824F078FEEE
:10824000019838B9044601982AF0E4FD204606B0AA
:10825000BDE8F0872BF0ECFE0022994906462CF091
:108260005FF90746002800F0E18000229449284683
:108270002CF056F93946804602A824F059FE012414
:108280000298002840F0A180414638462BF035FE88
:1082900000228C4930462CF043F90746E0B1002219
:1082A000884928462CF03CF98046384629F0CEFF14
:1082B000002800F0BD80404629F0C8FF002800F0EB
:1082C000B780414638462BF03BFB002841463846F4
:1082D00008BF00242BF011FE00227B4930462CF011
:1082E0001FF9074610B30022764928462CF018F9EA
:1082F0008046384629F061FF98B1404629F05DFF7D
:1083000078B138462BF005FA814640462BF001FA49
:10831000814506D80123002241463846F8F7F4F992
:1083200000B10024414638462BF0E7FD00226749A2
:1083300030462CF0F5F8074680B100226349284604
:108340002CF0EEF80146804638462BF0F9FA41460B
:108350000028384608BF00242BF0CFFD00225C49DE
:1083600030462CF0DDF8804670B129F004FE40B1B3
:10837000414605A824F0DCFDDFF85491059F002F4D
:1083800062D140462AF046FD0022524930462CF088
:10839000C7F8804670B129F0EEFD40B1414605A80E
:1083A00024F0C6FDDFF830A1059F002F6CD14046B8
:1083B0002AF030FD30462AF02DFD01A824F0A7FD5B
:1083C000002C3FF43DAF01243DE7B8F1000F10D081
:1083D0002BF02EFE014603A81AF034FA414604A8F9
:1083E00024F0A6FD4FF00009049838B9B9F1000F48
:1083F00000D1002402A824F08AFD41E72BF018FEEA
:10840000014605A81AF01EFA9DF816209DF80E30B8
:108410009A4207D1BDF81420BDF80C309A4208BF2B
:108420004FF0010904A824F072FDDDE701242FE7D5
:10843000384629F03BFC8146404629F037FCA9EB41
:1084400000035842584140E7B7F80B3003F500737A
:10845000A7F80B300022494628462CF061F88246E6
:1084600080B1002239462CF0EEF9002808BF002424
:108470002AF0D0FC384651462BF03FFD05A824F0E9
:1084800046FD7BE70446F5E7B7F80B3003F50073CC
:10849000A7F80B300022514628462CF041F88146BF
:1084A000014638462BF04CFA49460028384608BFAA
:1084B00000242BF022FD05A824F029FD74E700BF5D
:1084C0003ACF0500F4D90500A0CE05008DD00500F7
:1084D00043CF0500ABCE0500BCCE050073B5054605
:1084E0000E4629F03FFD38B91549032025F08EFCD2
:1084F0000024204602B070BD304629F033FD00282C
:10850000F2D02AF05BFB04460028F2D0294601A8ED
:1085100024F00EFD01980028EBD02BF089FD0546D4
:1085200001463046FFF784FE18B1294620462BF05D
:10853000F1FE28462AF06EFC01A824F0E8FCE9E7E9
:108540007ACE05002DE9F04F87B000AFC7E90201F0
:108550001446002A6CD09149002023F055FD0022DA
:10856000054638618E4920462BF0DAFF8C490246D9
:1085700028462BF0A8FF00228A493D6920462BF0AF
:10858000CFFF8849024628462BF09DFF2AF016FBB4
:1085900080462AF016FB00228246834920462BF0B3
:1085A000BFFF8146E8B102467F4938692BF074FF6E
:1085B000002307F1140148467B612BF0F5F80446CF
:1085C000002844D1484629F01DF90546786124F079
:1085D00047F905F5807383422ED97449012025F0AF
:1085E00015FCB8F1000F07D0D8F8003023B142468F
:1085F0006F4938692BF050FF50462BF0ACF820B192
:1086000052466C4938692BF047FF5246414648466E
:108610002BF066FCFB68002B40F0B78007F11003DD
:1086200001220021B86822F087F838692AF0F2FBAD
:108630001C37BD46BDE8F08FEB1D23F00703ADEB03
:10864000030D6C462A462146484629F0FFF97B690E
:10865000002BC6D0B8F1000FCED0BAF1000FC0D0B9
:10866000002514E0092A09D1A91C2144701ED7F85D
:1086700010B02BF0E1FA5049024619E0911E012991
:1086800027D89B4602239E4216DA013635447B6981
:10869000AB42A6D96319665D5A78082AE2D1A91CB3
:1086A0002144701ED7F810B02BF0C6FA4349024699
:1086B00058462BF008FFE8E73BF8021F40487B6074
:1086C0002AF05EFF014640462BF03DFE7B680233F8
:1086D000D9E7911F012908D8A81C20441AF082F973
:1086E000014640462BF02FFECFE7162A2BD0212A39
:1086F00032D1A81C20441AF075F9122383463B603E
:10870000BBF1000F1BD00122594650462CF09BF8BC
:108710003B6878605919701CC01A21442AF089FB03
:108720007A6803463AB130B10146386010462BF002
:1087300025FBD7E90032194610462BF0DEFB5846E0
:108740002AF068FBA1E759881D482AF019FF2DF08F
:10875000A9FA04238346D2E7FF2A96D1D8789B78DA
:10876000D7F810B043EA00202AF040FA1549024633
:1087700058462BF0A8FE291D2144F01ED7F810B052
:108780002AF057FB1049024692E7D7E90301FFF7A9
:108790004FFD00287FF442AF47E700BF70D20500CD
:1087A0008DD00500F1CD050072DA0500EAD705008D
:1087B0003ACF050043CF0500F4D9050080D205006B
:1087C00012160600BCCE0500ABCE05002DE9F04127
:1087D00086B000AF00238846391D04467B602AF02E
:1087E000E3FF0546002C38D0E0B9204629F00AF80E
:1087F0000646786024F034F806F58073834206D983
:108800004149012025F002FB224640493BE0F31D8F
:1088100023F00703ADEB030D6D4632462946204693
:1088200029F014F97B68002BEED0404629F0BEFBFE
:1088300028B1374B3749186842462BF02DFE364B8E
:108840001A6812F0400F1E460AD13449012025F063
:10885000DDFA1837BD46BDE8F0810028E2D1D3E744
:108860002F4A12884FF6FF71914201D12D49EDE751
:108870001A6812F0800201D02B49E7E77C68102CBF
:1088800005DD2A491022012025F0C0FAE1E7284B36
:1088900093F800C0274BA4B2BCF1000F25D19A7CFD
:1088A00072B3B3F8760188422CD09B8A7C80C7F8DB
:1088B0000AC0A7F80EC03B810123BB7207F1080173
:1088C000BB1CC7E90435FBF7EBF918B97B88A34259
:1088D00018BF0C2040F6BB3112F086FC0028B8D13E
:1088E000336843F080033360B3E7B3F8760188421E
:1088F00008D07C80C7F80A20FA81B3F84E31DAE755
:108900000720E7E70820E5E7EAD70500F6D00500ED
:10891000482E002086D00500BCC2002090D0050063
:108920006A2D0020A4D00500B3D00500CBD00500EF
:10893000F9C20020F0BC00202DE9F04F9D4B91B012
:108940001B681B0700AF044607D59B49012025F093
:108950005DFA4437BD46BDE8F08F15F05BF920465F
:1089600029F009FB0546002800F01A81214607F18D
:10897000140024F0DDFADFF864A2796989B10023DC
:10898000BB61B1F80B3003F50073A1F80B3007F1B0
:10899000180019F057FF024638B18849012025F028
:1089A00035FA78692AF036FAD3E7D7F81480B8F1A7
:1089B000000F03D040462BF03BFB8046414607F1B9
:1089C0001C0024F0B5FAF96985B179B1B1F80B3022
:1089D00003F50073A1F80B3007F1200019F032FF06
:1089E000024670B17649012025F010FAF8692AF0A4
:1089F00011FA40462AF00EFA07F1140024F087FA23
:108A0000BBE707F128003C8C97F822601AF02AF89F
:108A100008B1F9F737FA4FF00009002207F13001E9
:108A2000388DC7F830901AF01BF8052810D043F2A3
:108A3000030290420CD0A8B93B8EA34214D197F800
:108A40003230B34210D1B7F82890B9F1000F0FD1EE
:108A5000386A19F0DDFF5B4904460246012025F023
:108A6000D5F93EE0F9F70EFA3B8D01333B85D4E7AB
:108A7000FC691CB120462BF0DBFA04460022524967
:108A800020462BF04DFD00225049064620462BF093
:108A900047FD2CF0C6F90022B8604D4920462BF066
:108AA0003FFD2CF0BEF9F860C6B1002307F12401A8
:108AB00030467B622AF078FE834620BB304628F0A1
:108AC000A1FE7862786023F0CBFE7A6802F58073AD
:108AD00083420ED93F49012025F098F930462AF00B
:108AE00099F920462AF096F907F11C0024F00FFAB4
:108AF00069E7D31D23F00703ADEB030DEB465946A1
:108B0000304628F0A3FF7A6A002AE7D00021798551
:108B10003A85494607F12802BAF80000C7F82CB098
:108B2000FDF76AFC40F2915112F05EFBBB6880F0E9
:108B30000100C5B213B9FB68002BCFD0BAF80020F2
:108B40004FF6FF719142C9D0FB68BAF80000A7F850
:108B500030900022002BC7F83220FA867A6A7A8297
:108B600014BF0222012287F8322007F1300107F1F9
:108B70001202C7E90E2BFBF793F830F00802ADD0D4
:108B800043F204029042A9D043F201429042A5D0A0
:108B900040F2A65112F028FB002818BF00259DE7DF
:108BA000002C3FF4D6AE22460B49032025F02EF9C7
:108BB000CFE600BFBCC2002020D3050048D305008B
:108BC00061D3050091D30500A1E6050081D305001E
:108BD00088D30500EAD70500B5D305006A2D00202B
:108BE0002DE9F04F9BB000AF0D4604463C2200211A
:108BF00007F12C00F6F796FC022387F82C30284664
:108C0000062387F82F3029F0B6F9002879D0002202
:108C1000844928462BF084FC38B12CF002F9002856
:108C200014BF0223002387F82C3000227E492846F7
:108C30002BF076FC38B12CF0F4F8002814BF062392
:108C4000052387F82F300022784928462BF068FC4E
:108C50008146D0B1002307F10C01FB602AF0A4FD8E
:108C6000064600283CD1484628F0CCFD8046F860F6
:108C700023F0F6FD08F58073834225D96C49012065
:108C800025F0C4F848462AF0C5F82846002269496C
:108C90002BF046FC054640B13B6D6BB32BF0E6F97B
:108CA0003B6D188028462AF0B5F8204629F05AF97D
:108CB00080B3B4F80B3003F50073A4F80B302046F2
:108CC0006C37BD46BDE8F08F08F1070323F00703BA
:108CD000ADEB030D6E4642463146484628F0B6FEDF
:108CE000FA68002ACED084B06B464FF6FF713B6520
:108CF00019809A809E60C5E74F49032025F086F8C9
:108D0000D0E7002DD1D04D492A46032025F07EF82A
:108D10000024D4E7204629F008F905460028C8D1E8
:108D2000204629F028F9002876D020462AF058FA63
:108D30000C235843073020F00700ADEB000D21460F
:108D400007F1080024F0F4F8E846DFF8E4A0444610
:108D5000A946B868F8B987F85850C7F854801F2357
:108D600007F1080207F10C0107F12C003B81FCF729
:108D70003DF818B1324B5B68002BC9D040F2F63198
:108D800012F032FA0028C3D107F10C0138892AF019
:108D900050F8044693E72BF04BF907F10C0183469A
:108DA000C7F80C902AF000FD0646BBF1000F10D06A
:108DB00078B9584628F026FDF860786023F050FD19
:108DC0007A6802F5807383421BD95146012025F051
:108DD0001DF858462AF01EF8B86828B1B0F80B30D4
:108DE00003F50073A0F80B302BF0E2FEFB68208047
:108DF000A380A66007F1080024F089F801350C343F
:108E0000A7E7D31D23F00703ADEB030D6E463146F4
:108E1000584628F01BFEDCE7002CA0D0224609496A
:108E200073E700BF6DCF050076CF0500ABCE050020
:108E3000EAD70500BCCE050083CF0500B7CF0500FB
:108E4000482E0020EDCF050008B5064A136823F42C
:108E50000073136012F056FA40F20B21BDE808408F
:108E600012F0C2B9BCC2002008B5054A136843F429
:108E70000073136012F0B0F8BDE80840FEF754BB71
:108E8000BCC2002008B517F007FE41EC100B08BD6E
:108E900010B50F4B1B884FF6FF729BB293420446EE
:108EA00003D10C4A1288934208D00B4820F076F880
:108EB0000A4A136843F00803136010BD29F076F8DE
:108EC000002814BF20460020BDE8104014F030BC3C
:108ED000682D00206A2D002057D00500BCC200205C
:108EE00010B5044629F047F8224630B92CB10B4999
:108EF0000320BDE8104024F089BF094B0949586898
:108F00002BF021FF12F0EEFB074B1B681B0704D56B
:108F10000020BDE81040FFF7BBBF10BD8AD205009E
:108F2000482E0020B3D20500BCC2002038B5104C3A
:108F300010490022054660682BF0F2FA2BF038FE4B
:108F4000C3B285B143F0010098420FD0646829F0A4
:108F50004DFE0849024620462BF0B5FA0020BDE838
:108F60003840FFF795BF03F0FE00EDE738BD00BFC6
:108F7000482E00209CD105002DE9F0418CB006461A
:108F8000884628F0F8FF40B93EB1324647490320F1
:108F900024F03CFF0CB0BDE8F08100230293019364
:108FA000434B039302AB0593424B069303270B23DA
:108FB000ADF81C300DEB0703012208933E4B8DF8F2
:108FC000032009933A4601AB03A94046ADF810705F
:108FD000ADF828700B932CF0E3F90028DAD0029852
:108FE000364D374C29F016F948B1029A3549686870
:108FF0002BF052FA236843F00803236009E0029B38
:10900000002B37D12F4968682BF08CFE2368590656
:10901000F0D4029829F0FEFE9DF80330002B2ED0EC
:109020002368294968689A065EBF236843F00803ED
:1090300023602BF077FE3246244968682BF083FECC
:109040004246234968682BF07EFE019A1AB12368D4
:1090500043F0080323601F4968682BF074FE0198F1
:1090600029F0D8FE236813F0180F1BD00020FFF75B
:109070000FFF8FE71849384624F0C8FEC9E7236878
:109080006F689B0648BF23684FF0000044BF43F061
:109090000803236029F0A2FD0B49024638462BF055
:1090A00012FAC8E7304614F08FFB73E7B5D305001A
:1090B0008CD00500BBD20500C0D20500482E002090
:1090C000BCC20020CAD20500F9D2050002D30500B7
:1090D0000CD3050016D30500D4D2050013B569469C
:1090E000044619F0F3FB28B90749012024F08EFE4D
:1090F00002B010BD054B0649586822462BF0CCF94A
:109100000020FFF7C5FEF3E70ED10500482E002032
:1091100044D1050038B50A4C05462DB9094B002C41
:1091200008BF1C46204638BD3CB1204631F068FEE1
:10913000013D01300444EDB2EFE7024CF2E700BF1D
:10914000D5BB0500FE59060070B50D4C06462078CB
:109150000D4640B1FFF7DEFF0A490246012024F028
:1091600055FE002070BD09F06DF9074B26701860A0
:10917000284628F07BFC054B18600120F2E700BF71
:10918000C0C200205FCD0500B8C20020C4C20020CC
:1091900037B50546002105208DF80610FFF7D4FFEE
:1091A00058B1074B186828F061FC0199044628461D
:1091B00011F08EFF204603B030BD0446FAE700BF31
:1091C000B8C2002037B505460C4605200021FFF740
:1091D000BBFFB8B1214601A819F09EFA024638B18A
:1091E0000949012024F012FE0024204603B030BDBE
:1091F000064B186828F03AFC01990446284611F0FD
:1092000067FFF2E70446F0E77ED30500B8C200200E
:1092100013B5002104208DF80610FFF795FF50B11B
:10922000064B186828F022FC0446019811F096FFBE
:10923000204602B010BD0446FAE700BFB8C20020C5
:1092400013B50C4604200021FFF77EFFB0B1214684
:1092500001A819F061FA024638B10949012024F049
:10926000D5FD0024204602B010BD064B186828F03A
:10927000FDFB0446019811F071FFF3E70446F1E7A6
:109280007ED30500B8C200202DE9FF4100228846A8
:10929000264906462BF044F90022254907462BF0C3
:1092A0003FF96946054619F011FB044658B92946AD
:1092B00038462AF022FE1F49032024F0A7FD20464D
:1092C00004B0BDE8F081384629F0A4FD00221A4917
:1092D00030462BF025F92BF0A4FD074620B130468F
:1092E00009F010F90446EAE731460220FFF72CFFA7
:1092F00020B90024284629F08DFDE0E748210F48D9
:1093000029F052FC04460028F3D00146022302AAA9
:109310003846CDE902581FF0D3FD204629F07AFDEA
:10932000074B186828F0A2FB0446E3E7C1CD05000F
:109330008DD0050036CE0500E1CD050049C2020002
:10934000B8C2002070B504460E4600200E4922F037
:109350005BFE054610B90025284670BD22460B4924
:109360002BF09AF82846FEF715F90446284629F00E
:1093700051FD002CEFD031462046FFF785FF054612
:10938000204629F047FDE7E770D205008DD00500A3
:1093900070B5064650B128F0EEFD044630B92849B4
:1093A0003246032024F032FD204670BD00222549BC
:1093B00030462BF0B5F8054628F0D4FD0446284683
:1093C00024B929F027FD2A461F49EAE729F022FDA2
:1093D00000221E4930462BF0A3F82CF05DFA02461D
:1093E0000B4604460D4631F047FA30B900220023FF
:1093F0002046294631F022FA08B1154D00242B46AB
:10940000224614481FF044FD054601460120FFF79F
:109410009BFE78B10821104829F0C6FB044628B10C
:109420003146FEF77BFD204629F0F4FC0B4B186813
:1094300028F01CFB0446284629F0ECFCB4E700BFEA
:109440001AD005004FD00500ADD1050022CF050090
:1094500000409F40F1BE02009DC30200B8C2002040
:1094600030B500218FB0044609202AF0E5FB164DE7
:109470000190024680B115496868FF23CDE90213C7
:10948000002313498DF810302BF01DF801A81AF0B5
:10949000D8F901A81AF0DCF901A81AF0D2F901A84C
:1094A0001AF0CCF922460B4968682AF0F5FF0A4BFE
:1094B00002221A70B4F80B30204603F50073A4F8AA
:1094C0000B300FB030BD00BF482E00200300FFFF5F
:1094D000F11B060072D9050000C3002019F080BB03
:1094E00019F0C2BA38B5054609B119F02DFB0022B2
:1094F0000D4928462BF014F82BF093FC10B10B48C3
:109500002AF0F2FB01460446284619F01DFB2046CE
:1095100029F080FC012029F061FB0549024628461C
:10952000BDE838402AF0CFBF09B00500012706008A
:10953000DED7050008B519F007FB002008BD0000C4
:1095400070B58EB0044601A80E4615461AF0DAF939
:1095500090B12046002209492AF0E2FF044658B1A2
:10956000324607492AF098FF2A46064920462AF043
:1095700093FF204629F04EFC0EB070BDB7D4050015
:10958000BBD40500CAD4050010B58EB0044601A8AE
:109590001AF0B8F930B101A8214619F0D7FC01A89A
:1095A0001AF04CF90EB010BD70B506462AF040FD19
:1095B000054628F0FBFC044640B90E48294624F035
:1095C00005FB284629F026FC204670BD284629F0D8
:1095D00021FC0949002022F017FD04460028F3D0A1
:1095E000002119F039FD3246044920462AF054FF83
:1095F000EAE700BFFCD80500BACD050023D9050075
:1096000070B506462AF014FD054628F0CFFC044646
:1096100040B90E48294624F0D9FA284629F0FAFB29
:10962000204670BD284629F0F5FB0949002022F0AC
:10963000EBFC04460028F3D0012119F00DFD324661
:10964000044920462AF028FFEAE700BFFCD80500BD
:10965000E2D7050023D9050030B591B0044603A830
:109660000D461AF04FF948B1002303A800932A468B
:10967000214619F04DFB03A81AF0E0F8002011B0C4
:1096800030BD30B58FB0044601A80D461AF03AF946
:1096900058B11DB129462046FFF7DEFF01A821463B
:1096A00019F054FC01A81AF0C9F80FB030BD000041
:1096B00030B58FB0054601A81AF024F9E8B10021B1
:1096C000114819F0D7FC0446A0B1294601A819F0A9
:1096D0008BFC2946012220462DF080FB054670B107
:1096E000014620462BF06EFA284629F093FB2046CF
:1096F00029F090FB01A81AF0A1F80FB030BD034883
:1097000024F044FAF3E700BF2ED9050034D9050050
:109710002DE9F04391B0804603A80F4614461E463B
:109720001AF0F0F8B8B1002118982AF08FFC05461D
:1097300028F062FC78B320462AF098FC8146304637
:109740002AF094FC06461B2029F0C0F9044628B9EB
:1097500003A81AF073F811B0BDE8F08333464A4607
:10976000394629F0CFFE012118982AF06FFC0646F1
:1097700028462AF07BFC80B20090334622464146C0
:1097800003A819F0C5FABC42E2D032462946204669
:109790002AF0A6FBDCE7284629F03CFB25463C46A0
:1097A000E6E700002DE9F04F8BB08246019128F0EA
:1097B00004FD20B9002630460BB0BDE8F08F29F03B
:1097C00000FA06460028F5D04FF000094FF0FF35AB
:1097D0000022514605A823F098FFCB462C46A84608
:1097E0002F464A464B46DDE90501814200F2B6802C
:1097F000B4F1FF3F08BF5C46089829F00BFBB8F1B5
:10980000FF3F08BFA046002F09DD7A1E0021504609
:1098100029F0A5FEA349024630462AF054FEA2488C
:109820002AF062FAA149024630462AF04CFE791C21
:10983000A8EB0102504629F092FE9D4902463046AF
:109840002AF041FE6FF000422146504629F087FE83
:10985000074629F05EFF18B99649384629F0EBFE15
:109860003A46954930462AF02EFE691C14BF2A1B41
:109870006FF000422146504629F071FE044629F05F
:1098800048FF18B98B49204629F0D5FE22468B495E
:1098900030462AF018FE6A1C00F09E806FF00042ED
:1098A0002946504629F05BFE0246854930462AF09B
:1098B0000AFE09F1FF324FF6FE739A4240F29080A1
:1098C000022029F003F902467E4930462AF0FBFDCA
:1098D0006B1C00F089806FF00042691C504629F033
:1098E0003EFE019B80469BB328F006FB044678BBF6
:1098F0000246414605A823F008FF29F062F9814697
:109900001B2029F0E3F805461B2029F0DFF8074665
:10991000DDE905239A426BD3089829F07BFA40468B
:1099200029F078FA284629F0F4FE002800F08D800E
:1099300028462CF0B7F9394605462AF073F829462F
:1099400048462AF009FC394628462AF0D6FAC84685
:1099500042465D4930462AF0B6FD2CE705A8CDE920
:10996000022323F0CBFD2F28DDE9022312D1B4F12D
:10997000FF3F08BF5C46012A03F1010306D1022B19
:1099800004D1791C02D13D463C465F46B8F1FF3F09
:109990000DD118E03A2807D1791C02F10102F5D067
:1099A000611CF3D1D8460EE0B8F1FF3F0ED0D84588
:1099B0000CDA611C73D12F2805D9392803D8303827
:1099C0000A2101FB09090BF1010B0CE73F28FAD131
:1099D000601CF8D05D46F6E7022029F077F863E7CF
:1099E000484629F003F96EE7022029F06FF878E77E
:1099F00005A823F083FD262822D1284629F089FED8
:109A0000C0B128462CF04EF9394604462AF00AF82F
:109A1000214648462AF0A0FB394620462AF06DFA36
:109A20001B2029F053F805461B2029F04FF8074664
:109A300000246DE7384629F06CFE0028E1D167E785
:109A400054B93D2820D1019C62E7384629F061FED7
:109A500000287FF46DAF76E725280CD105A823F008
:109A60004DFD824605A823F049FD0146504623F0EE
:109A70002CF9C0B254B18DF8130001220DF113017D
:109A8000384629F0BFFDDEE72528E7D08DF8130022
:109A900001220DF11301284629F0B4FDC8E73F2843
:109AA00098D090E7ABDA0500B4DA0500B8DA050023
:109AB000FA1B0600AED90500BFDA0500C4DA0500BE
:109AC000CDDA0500D4DA0500D9DA05002DE9F04F2A
:109AD0002DED028BA3B08B46154629F06FF8824618
:109AE000002800F0C080584628F094FB002800F0C1
:109AF000BA80284628F03FFA002800F0908008AA93
:109B00001892804A199206AA1B927F4A7F4B1C9298
:109B100004AADFF8049216931E920A237C4AADF839
:109B20005C30002600274FF00008ADF86830ADF833
:109B300074301F92ADF88030042202AB16A928467B
:109B4000CDE90867CDE90667CDE90489CDE902676B
:109B500021932BF025FC002800F085809DED028BE1
:109B600032463B4651EC180B30F054FE002851D1E0
:109B7000B0EE480AF0EE680A2EF05AFA53EC102BB9
:109B8000B0EE480AF0EE680ACDE900232EF040FB63
:109B9000DDE9002355EC104BDDE90467304639461A
:109BA00030F0D0FB3246804689463B46204605F1E0
:109BB0000041CDE90A8930F0C5FBDDE90823CDE994
:109BC0000E01CDE91223304622462B46394630F0AD
:109BD000B9FBDDE90623CDE90C01CDE91089CDE91A
:109BE00014230122594616A824F03BFB16A823F0A3
:109BF00057F958B116A823F0E3FA064616A80F46FF
:109C000023F069FA16A823F04BF990BB16A823F0AD
:109C10001BF928E034463D4642464B46BCE7284601
:109C200028F0F8FAC8B1284629F095FD0628044620
:109C300013D12946012216A824F013FB0AAD16A859
:109C400023F0BEFAE5E8020116A823F044FA013C2D
:109C5000F5D116A823F0F8F8C3E72E49032024F025
:109C6000D5F84FF0000A504623B0BDEC028BBDE89A
:109C7000F08F16A823F0A4FA044616A80D4623F088
:109C80002AFADDE90A233046394630F05BFBDDE98C
:109C90000E23804689462046294630F053FB024673
:109CA0000B464046494630F097F9DDE9122330F083
:109CB00093F941EC100B28F087FF014650462AF03B
:109CC00042FBDDE90C233046394630F03BFBDDE951
:109CD000102306460F462046294630F033FB024645
:109CE0000B463046394630F077F9DDE9142330F081
:109CF00073F941EC100B28F067FF014650462AF03B
:109D000022FB73E7E2FC050088D7050022FC050072
:109D10008ED7050095D705000000F03F2DE9F04FE4
:109D200093B00C46164628F049FF0546002800F07F
:109D30008480002C00F081802368062B7DD1214691
:109D4000012207A824F08DFA01AF002407A823F010
:109D50008CFA013447F8040B07A823F0BCF9062C51
:109D6000F4D107A823F070F8304628F004F930B198
:109D70000022354930462AF0D3FB2AF019FFDDF8DE
:109D80000480059EDDF80890069FB8EB060448BFE6
:109D9000A6EB0804B9EB070348BFA7EB09039C42F5
:109DA000A8BF1C46002C08BF01244FF4A04393FB1E
:109DB000F4F4B4F5805F44DA40F299139C42B8BFE2
:109DC0001C460028C8BF4FF480544A46C8BF94FBC5
:109DD000F0F4414628462AF0C0FAC4F5805BA2465A
:109DE0000BFB0BFC0AFB0BF04FEA2C3C049A40F3F4
:109DF000D3200CFB09F302FB0032039B0AFB0AF1A0
:109E00000CFB08FC03FB00C3091301FB072201FB49
:109E1000063102F5006201F50061121309132846AC
:109E2000A2442AF09AFABAF5805FABEB040BD7DDB7
:109E30003A46314628462AF090FA284613B0BDE843
:109E4000F08F40F25554BCE77ED605002DE9F04F67
:109E50009BB0014609A81AF01FF828B90023039304
:109E600003981BB0BDE8F08FBDF829309DF82F4056
:109E7000DB06A4F1020347BFBDF82D70BDF82B60CF
:109E8000BDF82B70BDF82D60012B70D9082CB8BF20
:109E9000082407FB04F31F33082C4FEA6313D8BFD1
:109EA0004FF001094FEA83030093D4BF09FA04F984
:109EB0004FF00009009B09EB490505F11A0803FB67
:109EC000068A504628F05AFD03900028C6D028F094
:109ED000B9F8422303704D2343700C2383733B1264
:109EE00080F802A0C3744FEA2A2A33124FF0010E01
:109EF000082C80F803A080F80A80877406754375E3
:109F000080F816E0047634DD0123A340013B06937C
:109F1000009A0823B3FBF4F30193E3100593731E37
:109F200002FB0355431902934FF00008B04597DA3E
:109F300008F101030493029B072C03F11A0547DD86
:109F40004FF00009B94549DA4246494609A819F0D7
:109F500054FF2A46002308339C4202F8010B4FEAC3
:109F60001020F8DC059B09F101091D44EAE70424EF
:109F70008FE79DF82F30032B00F11A0315D0002135
:109F80009DF82F200EFA02FC8C4503F10303BBDD84
:109F9000C1EB012292FBFCF2D2B203F8032C03F8CE
:109FA000022C03F8012C0131EAE700224A4503F1B3
:109FB0000303A9D042F3000103F8031C42F340015C
:109FC00003F8021C42F3800103F8011C0132EDE7A3
:109FD000DDF804B04FF0000ABA451CDB029B009A82
:109FE000DDF810809B1A0293A0E74B1C424609A89B
:109FF000079319F002FF069B1840079B09FA04F922
:10A0000040EA090919465945EFD1019B05F8019B22
:10A010009A449B44E0E751464FF00009F3E7000003
:10A0200038B5FFF713FF054610B90025284638BD9F
:10A030000AF020FF0446284628F0ECFE002CF4D05D
:10A040002146044829F09CFA0546204628F0E2FE05
:10A05000ECE700BFFDD4050010B5FFF7E1FF0446B3
:10A0600008B120F0E1FA204628F0D4FE0248BDE80D
:10A0700010401FF011BE00BF0027060000B593B0CE
:10A08000014601A819F008FF10B101A8FDF7EAF98F
:10A0900013B05DF804FB000000B593B0014601A8C1
:10A0A00019F0FAFED8B1BDF8180010F460430AD0D8
:10A0B000B3F5005F0D4918BF00211B0405D429B971
:10A0C00028F094FD0BE00A49F7E70A4941F6FE73D0
:10A0D000184207D0C0F30C02074829F051FA13B018
:10A0E0005DF804FB084629F0FFFDF8E73ED60500C1
:10A0F00037D6050077D6050042D6050030B593B0B7
:10A100000C46014601A8154619F0C6FE20B12A46A4
:10A11000214601A819F071FE13B030BD2DE9F041C0
:10A12000B2B00546884601460CA819F0B5FE0028D5
:10A1300000F0D4800BAA1F92694A20920AAA2292A8
:10A14000684A694B239209AA1D9325920923674AFD
:10A15000ADF87830ADF88430ADF890302692ADF897
:10A160009C3008AAADF8A830ADF8B43006AB289200
:10A170002E935F4A5F4B29922F9307AA0B2300244B
:10A180002B92ADF8C0305C4ABDF83770BDF839602D
:10A190008DF817400DF117034046CDE90A44CDE98B
:10A1A0000844CDE906442C92319327F0E4FE40B9EF
:10A1B0005249012023F02AFE0025284632B0BDE88E
:10A1C000F08107221DA940462BF0EAF80028EFD0C5
:10A1D0000B99099A00290A4404DA079B09925B1A31
:10A1E00007930B940A98089B0028034405DA069904
:10A1F0000893091A069100210A91D21B002AC8BFB0
:10A2000009990B98C8BF8A1AA3EB0603C8BF099225
:10A21000002BC8BF089A0A99C4BFD31A0893079B9A
:10A22000099A002B1A4404DAC31A0B9300230992EB
:10A2300007930698089B0028034404DA091A0A9138
:10A24000002108930691D71B002FC8BF099A0799D0
:10A250000698C8BFD71BA3EB0603C8BF0997002BFE
:10A26000C2BF089AD31A0893DDE90823002B01DC4A
:10A27000002A2CDDCDE901100092DDF86B40DDE90C
:10A280000A210CA8A0479DF8173003B3DDE906109A
:10A29000BDF95340099A089BA0420244B8BFADF8EB
:10A2A0005300BDF957008242C8BFADF85720BDF931
:10A2B00055209142BDF95920B8BFADF855100B4457
:10A2C00093420CA8C8BFADF8593019F0C1FDB5F8DC
:10A2D0000B3003F50073A5F80B306EE705466CE70D
:10A2E00019D5050017EC050016D505002DFD050054
:10A2F0001CD5050022D505001FD505002ED505006B
:10A3000030B593B00D46014601A819F0C5FD0028EF
:10A310004CD0BDF92720BDF92B309A4244DC28F0FF
:10A3200050FC044618B3BDF9270028F05FFC204913
:10A33000024620462AF0C7F8BDF9290028F056FC4D
:10A340001C49024620462AF0BEF8BDF92B0028F031
:10A350004DFC1949024620462AF0B5F8BDF92D00FA
:10A3600028F044FC1549024620462AF0ACF8C5B155
:10A3700000226FF07F038DF82B208DF82C308DF8A4
:10A380002D208DF82E304FF0FF327F2301A88DF85D
:10A3900027208DF828308DF829208DF82A3019F0E3
:10A3A00057FD204613B030BD0024E0E70446F8E72F
:10A3B00016D5050019D505001CD505001FD50500CB
:10A3C00070B592B004460D46014601A8164619F034
:10A3D00063FD58B3BDF80930022D23F070039BB222
:10A3E0001ED0032D1FD0012D08BF43F03003ADF860
:10A3F00009304EB1BDF80930DA064CBF83F0400396
:10A4000083F02003ADF8093001A819F021FDB4F85C
:10A410000B3003F50073A4F80B30204612B070BD6A
:10A4200043F06003E3E743F05003E0E70446F4E75A
:10A4300070B592B004460E46014601A8154619F0C3
:10A440002BFD78B101A8ADF81A60ADF81C5019F0D9
:10A45000FFFCB4F80B3003F50073A4F80B30204672
:10A4600012B070BD0446FAE7F0B593B004460E464C
:10A47000014601A815461F4619F00EFD08B3012E2E
:10A480009DF81E10A8BF0126012DA8BF012546EA90
:10A49000E67666F3010145EAE57565F3830187F326
:10A4A000020767F3051101A88DF81E1019F0D0FC02
:10A4B000B4F80B3003F50073A4F80B30204613B04A
:10A4C000F0BD0446FAE700002DE9F04792B00446DB
:10A4D0008A46014601A8914698461A9F19F0DCFC6D
:10A4E000002859D0504627F068FE40B92B4901207A
:10A4F00023F08CFC0024204612B0BDE8F087B9F1AF
:10A50000FF0F01D92649F2E7404627F056FE28B949
:10A51000404627F027FF08B92249E8E7C7F3072696
:10A52000002E4FEA274308BF0126012B05DD022B31
:10A530002CD0042B2DD01C49D9E74FF400455246AE
:10A540001A49204629F0A8FF42461949204629F019
:10A55000A3FFF8B228F04AFB16490246204629F02C
:10A56000B2FF484628F042FB13490246204629F034
:10A57000AAFF354401A8ADF8185019F069FCB4F8E9
:10A580000B3003F50073A4F80B30B4E74FF420450B
:10A59000D5E74FF44045D2E70446ACE79ED6050028
:10A5A000BBD60500D8D6050002D7050020D7050088
:10A5B00025D7050048D605002AD70500F0B593B089
:10A5C00004460F46014601A816461D4619F064FCD4
:10A5D000A0B1189BADF8253001A8ADF81F70ADF8FB
:10A5E0002160ADF8235019F033FCB4F80B3003F5BB
:10A5F0000073A4F80B30204613B0F0BD0446FAE710
:10A600002DE9F0419AB007460D46014609A81446C7
:10A6100019F042FC4FF000080646002800F09D802B
:10A6200006AA05A909A8CDE90754CDE9058819F0BE
:10A6300051FB08AA07A909A819F04CFB059B079D27
:10A64000089CBDF84120BDF84310BDF845000791B6
:10A65000ED1A069B0890E41ABDF82B3006929D4235
:10A66000C8BF1D46C3F10003C8BF4646AB42C8BFC2
:10A670001D46BDF82D30C8BF00269C42C8BF1C46F1
:10A68000C3F10003C8BF0026A342C4BF1C46002676
:10A69000BDF83F30059346B1CDE901100092DDF8D9
:10A6A00063602246294609A8B047DDE90512BDF9D5
:10A6B0004760DDE90730B142BDF94B60B8BFADF886
:10A6C0004710B342BDF94960C8BFADF84B30B24244
:10A6D000BDF94D60B8BFADF84920B042C8BFADF874
:10A6E0004D00002D23DD6B180D9DDDF85760CDE981
:10A6F0000005013B09A8B047002C23DD069A0D9BFD
:10A7000001931444013CDDF85750079B00940599D0
:10A7100009A8A84709A819F09BFBB7F80B3003F567
:10A720000073A7F80B3038461AB0BDE8F081E3D0CB
:10A730000D99DDF8576003F1010CCDE900010CEB38
:10A740000501D7E7E6D0089B0D99DDF857505A1C54
:10A75000CDE900312244079BD9E70746E3E7000033
:10A760002DE9F04F99B006460D46014607A819F0AD
:10A7700093FB044620B90024204619B0BDE8F08FB1
:10A780008DB15C49284628F0DBFD804658B95A490E
:10A79000284628F0D5FD044630B92A4657490120FD
:10A7A00023F034FBE8E7A0460021304606F0C6FE61
:10A7B00001218346304606F0C1FE9DF8277000FB5C
:10A7C0000BF47C4307340646E410B8F1000F35D093
:10A7D00028F0F7F905460028CDD0584628F006FAAB
:10A7E00047490246284629F06EFE304628F0FEF919
:10A7F00044490246284629F066FE012F07D0384614
:10A8000028F0F4F940490246284629F05CFE9DF8FC
:10A810002030ABB9082F05D0BDF8213003F00F036D
:10A82000042B0DD100223949079829F079FE024600
:10A830003649284629F047FE2C469DE70334454615
:10A840002046002129F0F8F9044618B9284628F0D6
:10A85000E1FA91E70146002202A822F056FFB8F182
:10A86000000F0CD15FFA8BF102A822F076FDF1B255
:10A8700002A822F072FD394602A822F06EFD0026E1
:10A88000B1463346B24627E01A46514607A8009320
:10A8900019F0B3FA0AF1010A09FA07F9D34549EAAE
:10A8A000000907EB0602009B02DC01334FF0000AAF
:10A8B00016460AE0083E29FA06F1C9B202A8CDE917
:10A8C000003222F04AFDDDE90032072EF2D8D60828
:10A8D0006FF0070101FB0626DDE902129142D3D396
:10A8E000059828F097FAB8F1000F3FF445AF2246DB
:10A8F0009EE700BF971C0600B4E00500D6D4050013
:10A90000ECD40500F2D40500F9D4050018EA0500DE
:10A910002DE9F04FCDB005460E46014617A8174663
:10A920000293569C19F0B8FA002800F06783382289
:10A93000002109A8F4F7F6FD304627F01CFB00289B
:10A9400054D0B049304629F009FE00284ED0314697
:10A9500028A819F0A1FA002800F0A8809DF8A4808A
:10A96000B8F1000F40F0A280BDF8A7300993BDF800
:10A97000A930A5490A9342469DF8AB300B93304667
:10A9800029F0CEFD064628F0FBFC0E90304628F05C
:10A9900041FACDF83C809DF8303013B94FF0FF33C9
:10A9A0000D93109B5BB90B9B012B08D11B9AADF843
:10A9B00054201A9AADF8562015AACDE910230E9806
:10A9C00027F0FBFB064648B10999002906DD0A9BE2
:10A9D000002B03DD0B9B202B40F32C818B490120A6
:10A9E00023F014FA0E9828F015FA5FE0304627F0AD
:10A9F000C2FA002872D000228549304629F090FD25
:10AA00002AF0D6F8002283490990304629F088FDC3
:10AA10002AF0CEF8002280490A90304629F080FDC5
:10AA20002AF0C6F80028CCBF0B9001234FF000029B
:10AA30007A49D8BF0B93304629F072FD031C18BF2A
:10AA400001238DF830302AF0B3F800220D907449BC
:10AA5000304629F065FD804688B327F066FA50B38A
:10AA6000B8F80430022B26D1002328A940462893A9
:10AA700028F09AFE1090404628F0CCF9289B102B25
:10AA800005D9B3F5807F06D00023109305E0654A11
:10AA9000DA40D107F8D5013B1193DDF84080B8F1D9
:10AAA000000F0CD16049012023F0B0F900252846A1
:10AAB0004DB0BDE8F08F404628F0ACF9EDE700223C
:10AAC0005149304629F02CFD064628F059FC0E90DD
:10AAD000304628F09FF900230F935CE7304627F0BB
:10AAE0006CFB58B1304627F020FA70B9B6F80B303D
:10AAF0000E9603F50073A6F80B300AE0304627F0F7
:10AB000014FA0028EED14949CDE7304628F038FC48
:10AB10000E9000210E9828F0DEFC012109900E987D
:10AB200028F0D9FC02210A900E9828F0D4FC0206E5
:10AB30000B902CD500F07F0001230B9003210E9881
:10AB40008DF8303028F0C7FC04230D900B9E0F9336
:10AB500073067FF520AF06F03F064FF0010808FAB4
:10AB600006F808F1FF39022E0B96CDF8449028DC48
:10AB7000DDF83C9015AB4FF0000AD04509DC15AB71
:10AB80001093022303FA06F60F9B3344A4E7032332
:10AB9000DCE749460E98039328F09DFC09F1020278
:10ABA000834609F101010E98009228F094FC039B62
:10ABB000009A4BEA002023F8020B0AF1010A9146A1
:10ABC000DBE7082E16DC002328A90E982893DDF871
:10ABD0003C8028F0E9FD0B9B082B0BDC50B10223D5
:10ABE000B340289A434493423FBF0F9BCDF8449013
:10ABF000C0181090DDF84080B8F1000FC1D10C49A9
:10AC000051E700BF3ED5050018EA05000DD6050046
:10AC1000ECD40500F2D40500F9D4050047D50500B1
:10AC200053D50500140101005BD50500D8D50500FA
:10AC3000A6D5050001229A40013A072B1292DCBFEB
:10AC4000082292FBF3F203FB01F3D4BF02F1FF32BF
:10AC5000002207331392DB10DDE90E1204A81493CF
:10AC600022F053FD002C40F08C80BDF8613013F0D1
:10AC7000700F1AD0DFF89CA3029E4FF000084446E4
:10AC80000A9B029A1344B34279DC079828F0C2F871
:10AC90000E9828F0BFF817A819F0DAF8B5F80B30BD
:10ACA00003F50073A5F80B3001E7BDF87700BDF898
:10ACB0007910029B099ABDF87DC08742B4BF344623
:10ACC00038463A448B42BDF87B30A8BF029902F166
:10ACD000FF3EB8BF34469E45C8BF9E460A9A029BB7
:10ACE000134403F1FF33C8BF34466345C8BF63460E
:10ACF000BDF97FC0BDF98120C8BF34468445C8BFB7
:10AD0000ADF87F00BDF98300C8BF34467045BCBFB5
:10AD10003446ADF883E08A42BDF98520C4BFADF862
:10AD2000811034469A4202DAADF88530A2E7002C51
:10AD3000A0D1DDF88BA09FE704A822F0DFFB083448
:10AD400040EA08280B9BA342F6DC129AE41A28FA80
:10AD500004F313400D9A9A4209D0109A1AB111992E
:10AD60000B4032F813303246494617A8D04709F154
:10AD70000109099B3B444B45E4DC013680E7B946B9
:10AD8000F7E7204627F0F7F800283FF47EAF0022CF
:10AD90009D49204629F0C4FB2AF07EFD824621F021
:10ADA00000498B464FF0FF32984B504649462FF0F2
:10ADB00063FD70B94FF0FF32944B504649462FF077
:10ADC00051FD30B900220023504659462FF036FD80
:10ADD00018B1DFF844B24FF0000A00228C49204637
:10ADE00029F09EFB2AF058FDCDE90001DDE9008342
:10ADF00023F000494FF0FF32844B404649464FF064
:10AE000001042FF039FD40B94FF0FF327F4B40462F
:10AE100049462FF027FD00B9044684F001044FF0A5
:10AE2000FF327A4B40464946E4B22FF025FD38B94F
:10AE30004FF0FF32754B404649462FF013FD18B1D5
:10AE40009FED6F7B8DED007B029B299309AE0FCEAA
:10AE5000289731AF0FC70FCE0FC70FCE0FC796E899
:10AE6000030004AE87E803000FCE3FAF0FC79DED90
:10AE7000007B33683B6028A80023CDE92EAB8DED25
:10AE80002C7B8DF8C0408DF8C130F6F73BFDBDF846
:10AE90007780289BBDF879402A9F2B9E9845B8BFA4
:10AEA0009846299B9C42B8BF1C46BDF87B30013FA9
:10AEB0009F42A8BF1F46BDF87D30013E9E42A8BFFD
:10AEC0001E46BDF97F309845BDF98330B8BFADF857
:10AED0007F809F42BDF98130C8BFADF88370A34227
:10AEE000BDF98530C8BFADF881402246B342414626
:10AEF00028A8B8BFADF88560FBF739FEBDF8613012
:10AF000013F0700F0CBFDDF88BA0DFF808A1B4427E
:10AF100006DD3FAE0FCE04AC0FC433682360B4E649
:10AF200028A8FBF71BFEC146B94504DD28A8FBF79E
:10AF3000ECFD0134EBE74A9A7F322BD44B9B13F1A3
:10AF40007F0B27D4449B9A4224DA459B9B4521DA08
:10AF50004FEA222C339A082A4FEA2B2BDDE93610D0
:10AF600023D13C9A0CEB000302FB0B323FA826F0E6
:10AF700037FB439B0BB13F9A9B5C359A9A4209D0B1
:10AF8000389A1AB139990B4032F8133022464946A3
:10AF900017A8D0474A9B469A13444A93479A4B9B1B
:10AFA0009B1A4B9309F10109BEE7319B03FB0BCBC5
:10AFB0000BFB02F200EBE2023FA826F011FB439BE1
:10AFC0000BB13F9A9B5C08213398814207DB3B9A87
:10AFD00022EA0B0250433A9AC3401340CDE73FA800
:10AFE0000091029322F037F8029B439A00991B02CA
:10AFF0000AB13F98125C13430831E5E7054656E570
:10B00000000000000000000088D70500FFFFEF7F70
:10B010008ED70500333E04000000F03F70B594B0B9
:10B0200004460E46014603A8154618F035FFC0B188
:10B030003346BDF92420BDF92210009503A818F06D
:10B0400067FE03A8ADF82260ADF8245018F000FFA9
:10B05000B4F80B3003F50073A4F80B30204614B09D
:10B0600070BD0446FAE7F0B595B004460D460146BA
:10B0700003A816461F4618F00FFF98B11A9B0093BD
:10B0800032463B46294603A818F042FE03A818F0B2
:10B09000DFFEB4F80B3003F50073A4F80B30204644
:10B0A00015B0F0BD0446FAE72DE9F04F99B0064619
:10B0B0008946014607A818F0EFFEB0B3BDF830404E
:10B0C00004F460480FFA88FABAF1000FC4F30C04D4
:10B0D0002EDA00223049304629F022FA00222F4988
:10B0E0000546304629F01CFA29F062FD074648461D
:10B0F00029F0F0FE00220146814602A822F005FB5D
:10B100000026A3000093B346DDE902218A4212D350
:10B11000059827F07FFE284627F07CFE484627F05A
:10B1200079FEB3455846B8BF304619B0BDE8F08F38
:10B1300000273D46DBE7069939B1895C0A2904D12D
:10B140005E45B8BF5E464FF0000BB8F1000F07D167
:10B150002046F6F78BFA834402A821F07CFFD3E760
:10B16000B8F5005F02D1009B9B44F5E7BAF1000FF0
:10B17000F2DA2846019127F020F848B10199B94246
:10B18000EADBC91B284628F0A6F900FB04BBE3E76D
:10B19000284628F06BFFF8E725D705002AD70500D9
:10B1A0002DE9F04FE1B00D4602901C4601469DF896
:10B1B000A831159324A8924618F06EFE002800F0DE
:10B1C000A582BDF8A43024A803F46042C3F30C099F
:10B1D0000592FCF747F9BDF914300C90002B119340
:10B1E00080F29380059BB3F5204F00F08C80B3F57F
:10B1F000404F14BF012304230022B0490298039357
:10B2000029F08EF900220E90AD49029829F088F9B4
:10B2100000220690AB49029829F082F929F0C8FC77
:10B2200004909DF8AA20BDF89530ADF8583002F092
:10B230003002102A9BB270D183F03003BDF8972002
:10B24000ADF895300AF10103A246D41A9DF8AA3050
:10B2500003F00303012B0DD829460298FFF724FFC2
:10B260009DF8AA3003F0030303FB000000EBD0704D
:10B27000AAEB600A9DF8AA30C3F38103012B9FBF9C
:10B280000C9A03FB022303EBD373A4EB6304BDF816
:10B29000AB300A93BDF8AD300993BDF8AF300893D9
:10B2A000BDF8B1300793BDF89530DB0642BFDDE94C
:10B2B0000923CDE90932DDE90732284648BFCDE947
:10B2C000072329F007FE0022129001461FA822F052
:10B2D0001CFA039A01239340013B18934FEA890318
:10B2E0001793C2F1080356461D93DDE91F239A42C6
:10B2F00045D21FA822F002F90A2805462BD10C9B43
:10B3000056461C44F1E7022376E701230022CDE9EB
:10B310000332002306930E9383E7202A0ED183F095
:10B320006003BDF89720ADF895300AF10103A2EB58
:10B33000030ABDF8993001341C1B87E7302A85D1F8
:10B3400083F05003BDF89920ADF89530631C544646
:10B35000A2EB030A7AE7059B002B40F0928001469E
:10B36000BDF8A400F6F782F90A9B0B901B1AB342B2
:10B3700022DB0B9B1E4421F06BFA0028B5D02298EB
:10B3800027F048FD129827F045FD06990E9828F001
:10B39000B4FDBDF85830ADF8953024A818F058FD2C
:10B3A000029B029AB3F80B3003F50073A2F80B303E
:10B3B000029861B0BDE8F08F089B9E42D9DABDF8D3
:10B3C000A480099BA3EB0803A342D2DA079B9C420B
:10B3D000CFDA202DCDD93C49059AA5F121033B4D6B
:10B3E000DBB20846D7B29F422AD3C75C002DC0D03B
:10B3F0003301083B0D932301083B0F932F444FF07B
:10B400000D0BBD42B5D015F8012BC82A22D8304B00
:10B4100030499B5C14932E4B00205FFA80FE9645CA
:10B4200013D3149B0DF1D40C01EB030E8E450CF1DC
:10B43000040C11D135AA149924A818F0CDFAE0E72C
:10B4400011F8017B01323D44CCE713F801EB0130E8
:10B450007144E2E70021E4E711F8012BB2FBFBF0B5
:10B460000BFB10220D9BD2B212FB08F21A440238D9
:10B470000F9B2CF8042C10FB08F018442CF8020C3D
:10B48000D4E7059BB3F5005F26D10A9B033BB3428B
:10B4900012DC089B9E420FDA099B053BA3420BDCA2
:10B4A000079B9C4208DA159B2246CDE90093314662
:10B4B000034624A818F0CCFD179B5BE720D70500B6
:10B4C00025D705002AD705004BB105002AB2050093
:10B4D00085B305004EB40500119B002BBFF64BAFA2
:10B4E000069826F06AFE00285ED0049BAB4200F36B
:10B4F0000A810DF1D40800220699404622F005F990
:10B50000049B0027ED1ADDE935239A4203D2379BCD
:10B510001344AB4241DB399B002B43D013F802802C
:10B52000389827F077FC0A9BA3EB0803B34245DA6F
:10B53000089B9E4242DA099B0C9A9B1AA3423DDA71
:10B54000079B9C423ADA92FBF9F3039A1393534315
:10B550005F43FA100E9935A822F0D7F8399D07F00D
:10B5600007070DB1359BED5C039B7B439D4006EBCC
:10B5700009030D9300230F930F9B434580F2BF8077
:10B580000D9BA3EB09031B930D9B013B1C9304EB49
:10B5900009030B930023109377E0404621F0AEFFA0
:10B5A0000744B0E79846BBE7069828F05FFD049B88
:10B5B000EF1AAB42804600FB07F7B4DD08FB0966D3
:10B5C000D9E61D9BE8B21841159B0BB9002851D054
:10B5D0000B9B9DF89BC0A3EB09031A930B9B013BAC
:10B5E00019930002189BB0FBF3F0B0F5807F014681
:10B5F000A8BF4FF48071BCF1080FDDE9273223D9D1
:10B60000BCF1100F4CD1C3F34510C1F5807EC2F3DD
:10B61000451C4843C3F3C42B0EFB0C0C01FB0BFB76
:10B62000C2F3C4200EFB00B0000A03F01F034B431B
:10B630004FEA1C2CC00202F01F0240EA4C1C0EFB19
:10B6400002324CEA12230CE04FF48A7E2EFA0CFCF4
:10B650001CF0010F46D0C1F580704B4302FB003354
:10B660001B0A0193199B0093DDE91A211C9B24A856
:10B6700018F0ABFB039B1F44072F37DC9D40109B4A
:10B68000013310930B9B4B440B93109B139A9342E3
:10B6900097DB0F9B01330F930D9B4B440D936BE78F
:10B6A000BCF1180F1ED1C3F30720C1F5807EC2F391
:10B6B000072C48435FFA83FBC3F307430EFB0C0CD4
:10B6C00001FB0BFBD0B24B43C2F307422CF0FF0C43
:10B6D0000EFB00B00EFB02334CEA10201B0A40EABE
:10B6E0000343BEE77F28D8BF1346BAE735A821F049
:10B6F000B2FC399D0DB1359BED5C0027BFE7389852
:10B7000027F088FB5AE74FF0000857E702904FE612
:10B7100030B595B00546014603A818F0BDFBA0B1B1
:10B7200027F04CFA044668B1094828F0DDFA0146D2
:10B73000204628F008FE01220094064B11462846B8
:10B740000BF0B0FB204615B030BD0446FAE700BF51
:10B750003ED6050059B7020038B5054608460C46E6
:10B7600027F0D7FF072824D901221249204627F0C5
:10B77000DFFDF0B11049204627F0E2FDC8B90F49BE
:10B78000204627F0DDFDA0B90D49204627F0D8FD61
:10B7900078B96FF000420721204627F0E0FE04460A
:10B7A0000146284628F0B6FD2046BDE8384027F07F
:10B7B00031BB38BD4DD6050055D6050063D6050012
:10B7C00070D60500000000002DE9F04F97B09046BC
:10B7D0000191014605A81F4618F05EFB002856D0CF
:10B7E000019826F0EAFC002879D00023092202A95A
:10B7F00001988DF81030CDE9023329F0EBFC9DF86B
:10B800000C609DF809009DF80A909DF80B70002EC1
:10B8100040D121F045FA2EF02BFD0022904B2EF066
:10B82000BBFE044648460D4621F03AFA2EF020FDB4
:10B8300000228B4B2EF0B0FE824638468B4621F01C
:10B840002FFA2EF015FD864B00222EF0A5FE0022C9
:10B8500006460F460023204629462EF0E5FF88B90C
:10B8600000220023504659462EF0DEFF50B9002238
:10B870000023304639462EF0D7FF18B99DF80F3017
:10B88000002B3BD00120774922F0C0FA002017B0EE
:10B89000BDE8F08F494621F018FA2EF0E9FC6EA3BE
:10B8A000D3E900232EF078FE04460D463846314693
:10B8B00021F00BFA2EF0DCFC67A3D3E900232EF075
:10B8C0006BFE82468B469DF80D009DF80E1021F010
:10B8D000FCF92EF0CDFC60A3D3E90023B5E7019875
:10B8E00029F0ECFC404655EC104B29F0E7FC3846BB
:10B8F0005BEC10AB29F0E2FC57EC106B25F0004933
:10B900004FF0FF32584B204649462EF0B5FF002835
:10B9100040F09E804FF0FF32534B204649462EF0B8
:10B92000A1FF002840F094802BF000494FF0FF3237
:10B930004D4B504649462EF09FFF002840F088802E
:10B940004FF0FF32484B504649462EF08BFF0028FF
:10B950007ED127F000494FF0FF32434B3046494635
:10B960002EF08AFF002873D14FF0FF323E4B304655
:10B9700049462EF077FF00286AD100223B4B204633
:10B9800029462EF0DFFC2EF08DFF0022374B0446B7
:10B99000594650462EF0D6FC2EF084FF0022334B41
:10B9A0000546394630462EF0CDFC2EF07BFFBDF823
:10B9B000191011F4607184F3080385F3080280F311
:10B9C000080008D0B1F5C07F19D010D880291AD04E
:10B9D000B1F5807F1CD09DF81F1010291FD1911048
:10B9E000DA10D20242EA411242EAE0004FE7B1F532
:10B9F000007F11D0B1F5207FEDD1114601E019464D
:10BA00001346024606E01946034610460A46E2E798
:10BA1000194603460846DEE719461346F6E720298D
:10BA200006D11B0443EA0223034343F07F402EE781
:10BA3000182904D11B0443EA0223184327E71344BF
:10BA40000344B3F5C07F4FF0FF30B8BF00201EE7BE
:10BA5000019828F00BFB1AE70000000000E06F409F
:10BA600000002E4047D70500FFFFEF7F0000704029
:10BA700070B5044608460D4626F07DFA002875D0BC
:10BA800000223E49284628F04BFD064650B10023CF
:10BA90001A4601462046FFF797FE394B186030469C
:10BAA00027F0B8F900223749284628F039FD064624
:10BAB00050B100231A4601462046FFF785FE304B61
:10BAC0005860304627F0A6F900222F49284628F072
:10BAD00027FD064650B100231A4601462046FFF7CF
:10BAE00073FE274B9860304627F094F900222749CF
:10BAF000284628F015FD064650B100231A46014697
:10BB00002046FFF761FE1E4BD860304627F082F9D1
:10BB100000221F49284628F003FD064650B10023A5
:10BB20001A4601462046FFF74FFE154B1861304676
:10BB300027F070F900221749284628F0F1FC064644
:10BB400050B100231A4601462046FFF73DFE0C4B3C
:10BB50005861304627F05EF900220F49284628F048
:10BB6000DFFC18B129F05DF9054B1876B4F80B30FD
:10BB700003F50073A4F80B30204670BD2FD70500E5
:10BB8000C8C2002028DD050032D7050036D70500E1
:10BB90003AD705003ED7050042D70500F0B593B06F
:10BBA00004460E46014601A815461F4618F074F9D2
:10BBB000F0B1AFB9049B2A46314601A818F039F913
:10BBC00001A8ADF81A60ADF81C5018F041F9B4F8AE
:10BBD0000B3003F50073A4F80B30204613B0F0BD12
:10BBE00000231A4639462046FFF7EEFD0346E2E7FA
:10BBF0000446F2E72DE9F043ADB000AF00238846DC
:10BC000007F108010646BB6027F0CEFD0546AEB33E
:10BC1000F8B9304625F0F6FD0446B86020F020FE65
:10BC200004F58073834209D96649012022F0EEF8B9
:10BC30002E463046B437BD46BDE8F083E31D23F001
:10BC40000703ADEB030D6D4622462946304625F02D
:10BC5000FDFEB8F1010F14BF4FEAE80014204FF0C9
:10BC60000009391DC7F80490F5F7ACF87C68064662
:10BC70003CB9554821F0AAFF2646DAE70028E8D16A
:10BC8000D7E7B8F1010F40F08C805C22494607F1FC
:10BC90005400D7F80880F3F745FC4C4BFB6503F1E3
:10BCA00088333B6603F12943A3F59613A3F68B6310
:10BCB0007B66A3F18833BB66454BFB66B8F1000F8A
:10BCC00005D04246294607F1540016F0A9FC7A6DCA
:10BCD000B96D530F43EAC1031BBAFB60D30002F0F6
:10BCE0003F02372A94BFC2F13805C2F178051BBA6A
:10BCF0004022002107F114003B61F3F713FC80237D
:10BD00002A4607F1140107F154003B7516F088FC30
:10BD100007F10C01082207F1540016F081FC97F896
:10BD20005F302370B7F85E306370FB6D1B0AA37041
:10BD3000FB6DE37097F863302371B7F8623063717D
:10BD40003B6E1B0AA3713B6EE37197F86730237259
:10BD5000B7F8663063727B6E1B0AA3727B6EE37268
:10BD600097F86B302373B7F86A306373BB6E1B0AA6
:10BD7000A373BB6EE37397F86F302374B7F86E301C
:10BD80006374FB6E1B0AA374FB6EE37400231946F5
:10BD900007F154021A4401335D2B3FF44AAF11708E
:10BDA000F6E7B8F1E00F06D101232246B96828462C
:10BDB00016F06CFB3DE7B8F5807F7FF43AAF4B4659
:10BDC000F3E700BFEAD7050033D405000123456738
:10BDD000F0E1D2C3024B03495868002228F0A0BB0F
:10BDE000482E002055CD050070B5174B1C788442B5
:10BDF0000DD0FDF78FF905462046FDF78BF92A4651
:10BE0000034612490420BDE8704021F0FFBF104CEA
:10BE100000201870206840B189B1114604F07CF808
:10BE2000206826F0F7FF002323600A4C206826F0E4
:10BE3000F1FF00232360084B01221A7070BD1146E8
:10BE400004F0B2F9ECE700BFC0C2002024CD050029
:10BE5000B8C20020C4C20020E1C2002010B50A46CA
:10BE60000C460021FFF7C0FF2046BDE8104026F039
:10BE7000D1BF000038B5194D2A884FF6FF719142A5
:10BE8000044613D001460320FDF75EF918B1144BA8
:10BE9000186825F0EBFD044613212888F8F7FEFE0C
:10BEA00040F66B410FF0A0F9204638BD0D4B1D78D0
:10BEB000022D0DD10C4827F017FF01462846FFF749
:10BEC000CDFFFAF71EFE2046BDE8384006F01ABB4B
:10BED0000649012021F09AFFF5E700BF682D0020F8
:10BEE000B8C20020C0C20020C8CD0500DDCD0500CD
:10BEF00010B5094B1C78012C0CD100210846FCF729
:10BF00000DF8064827F0F0FE01462046BDE8104037
:10BF1000FFF7A4BF10BD00BFC0C2002036D005008F
:10BF20000A460021FFF760BFF7B5002234490446F6
:10BF300028F0F6FA28F03CFE324B3349064603223D
:10BF4000586828F0EDFA054630B12246B1B228F023
:10BF50002AFA284626F05EFF00222C49204628F0C7
:10BF6000DFFA0746002839D121460820FDF7ECF812
:10BF700018B90025284603B0F0BD254B254E18689A
:10BF800025F074FD33884FF6FF729A42054607D1BB
:10BF9000214827F0A9FE01460820FFF75FFFE9E7E7
:10BFA0003A461749204628F0BBFA28F001FE013036
:10BFB00080B2ADF80400ADF8060001A930880FF09A
:10BFC00021FD0FF021F804460028D3D001460820B7
:10BFD000FFF7A6FF204626F01DFFCBE726F01AFF4D
:10BFE00000210920FDF7B0F80028C2D0084B1868DE
:10BFF00025F03CFD0121054620460FF093FCB9E7F2
:10C0000002CE0500482E00200FCE0500F6CD05001B
:10C01000B8C20020682D0020DDCD050070B50146B6
:10C0200006460720FDF790F868B3184B184D1868BE
:10C0300025F01CFD2B884FF6FF729A42044608D16A
:10C04000144827F051FE01460720FFF707FF20465E
:10C0500070BD00221049304628F062FA28F0A8FD91
:10C060002B8881B2002218460FF0CAFC0EF0CCFFDC
:10C0700005460028EBD001460720FFF751FF284670
:10C0800026F0C8FEE3E70446E1E700BFB8C200209F
:10C09000682D0020DDCD050002CE05002DE9F04F12
:10C0A00085B00D4600AF00238046394628463B60E8
:10C0B00027F07AFB0446002D39D0F8B9284625F040
:10C0C000A1FB0646386020F0CBFB06F58073834267
:10C0D00009D93749012021F099FE0026304614374E
:10C0E000BD46BDE8F08FF31D23F00703ADEB030D54
:10C0F0006C4632462146284625F0A8FC0021062041
:10C10000FDF722F80028E8D02A4B2B4D186825F0BF
:10C11000ADFC2B884FF6FF729A4206460AD127489B
:10C1200027F0E2FD01460620FFF798FED6E700283B
:10C13000E4D1D2E700222249D7F80090404628F007
:10C14000EFF928F035FD00221FFA80FA1D4940461C
:10C1500028F0E6F9834640B300221B4928F0E0F9B5
:10C1600028F05FFE8046584626F054FE002398458E
:10C170003B8114BF022301233B71391D0123288811
:10C180007B71FC60A7F806A0A7F80A900FF0C8FB27
:10C190000EF03AFF04460028A0D001460620FFF723
:10C1A000BFFE204626F036FE98E78046DEE700BF59
:10C1B000EAD70500B8C20020682D0020DDCD0500BB
:10C1C00002CE050016CE050021CE050038B50D467D
:10C1D00001460A20FCF7B8FF60B3174B186825F03A
:10C1E00045FC164B1A884FF6FF719142044608D160
:10C1F000134827F079FD01460A20FFF72FFE20465D
:10C2000038BD18880F4B1B7880B28BB100232A46AB
:10C210001946F8F70BFB0EF0F7FE05460028EED0A6
:10C2200001460A20FFF77CFE284626F0F3FDE6E7EC
:10C230000820F0E70446E2E7B8C20020682D00209D
:10C24000DDCD050070BE0020F0B58BB06D460C460C
:10C25000294616F03BFB002800F0848000220123D1
:10C2600095E80300ADF818208DF81830A023ADF83C
:10C270001A303F4BADF80C10CDE907323D4B029020
:10C28000090C58688DF80E103B49099228F048F9BE
:10C2900028F08EFCC3074CBF384B394B089320461F
:10C2A0004FF0C873099325F066FE002841D00022A4
:10C2B0003449204628F034F929F0EEFA02460B46BC
:10C2C00006460F462EF0D8FA90B900222E4B304683
:10C2D00039462EF037F824A3D3E900232EF05CF979
:10C2E00000222A4B2DF078FE2EF004FBADF8200042
:10C2F00000222749204628F013F929F0CDFA0246FA
:10C300000B4604460D462EF0B7FA90B900221E4B9C
:10C31000204629462EF016F813A3D3E900232EF069
:10C320003BF90022194B2DF057FE2EF0E3FAADF841
:10C33000220002AB93E80300ADF81410090C04903E
:10C340008DF8161008AA06A904A80FF05DFB0EF0E0
:10C350005BFE044630B101460220FFF7E1FD2046B6
:10C3600026F058FD0BB0F0BD00000000008893409F
:10C3700090000400482E00209CD10500900120036D
:10C380001000A00084D1050000408F400000E03F75
:10C3900090D105000A460121FFF726BD70B50D4B6F
:10C3A0001C78012C054613D100210846FBF7B6FD89
:10C3B0002146094827F0E4FF064608F04DFA3046CA
:10C3C00026F028FD29462046BDE87040FFF7E2BF71
:10C3D00070BD00BFC0C20020C4C200207CDF704717
:10C3E0002DE9F04F964C85B0236800AF054603F069
:10C3F000040308460E463B6025F0BDFD002800F012
:10C40000AB8000228F49304628F08AF8B0B128F07E
:10C41000CFFB4FF47A73584340F2712390FBF3F053
:10C4200080B2B0F5804F884B28BF4FF48040202861
:10C430001A8838BF2020824218BF18800022834902
:10C44000304628F06DF838B128F0EBFC236800285E
:10C4500062D023F40063236000227D49304628F037
:10C460005FF838B128F0DDFC2368002857D023F4AA
:10C470008053236000227749304628F051F88146E6
:10C48000002873D0002307F10C01FB6027F08CF922
:10C490008046002852D1484625F0B4F98246F8601B
:10C4A00020F0DEF90AF5807383423BD96A49012006
:10C4B00021F0ACFC484626F0ADFC284625F05BFD9B
:10C4C000814608B9002D54D131462846FCF788FB37
:10C4D000002D40F0B2800025604C614960682A461A
:10C4E00028F031FC32465F49606828F02CFC284671
:10C4F00026F090FC3B680BB10EF06EFD4FF45B71C3
:10C5000040460EF071FE3B6863B30EF0FBFE40F256
:10C510006E310EF069FE25E043F400639BE743F4BF
:10C520008053A6E70AF1070323F00703ADEB030DE1
:10C53000E84652464146484625F088FA11234146CE
:10C54000BA893B7207F10800FFF748FF40F22D312E
:10C5500080460EF049FEADE746B13246424903201F
:10C5600021F054FC1437BD46BDE8F08F4FF00008B1
:10C57000A3E7284625F0F6FC786000284BD0B5F8F4
:10C580000B3003F50073A5F80B30236823F07F739D
:10C5900023F40033294607F10C00236020F0C8FC87
:10C5A000CB46F86850B9B9F1000F95D0BBF1010F37
:10C5B00092DD236843F4003323608DE727F038FDD4
:10C5C000824625F0D8FC10B9BAF1000F0FD13146E0
:10C5D0005046FCF705FB8146F86810B1494627F044
:10C5E000CDFB484626F016FCD7F8049009E05046EB
:10C5F00025F0B8FC0028F7D1504625F096FC00281D
:10C60000F2D1504626F006FC07F10C000BF1010BAD
:10C6100020F07DFCC5E7284625F087FC00283FF484
:10C620005AAFB5F80B3003F50073A5F80B3023684B
:10C6300023F07F7323F40033BEE705464CE700BFC9
:10C64000BCC200204CD105002C2D002055D1050086
:10C6500061D10500F4D90500EAD70500482E002075
:10C660006BD1050075D10500B7CF050072DF7047AB
:10C67000F0B5284B284983B0044600AF02465868FD
:10C6800028F061FB204625F06DFC48B10023391DE0
:10C6900020467B6027F088F805466CB970BB1BE02C
:10C6A000204625F042FC0028F0D1CCB122461B499F
:10C6B000032021F0ABFB13E000BB204625F0A2F8DD
:10C6C0000646786020F0CCF806F5807383420AD9DC
:10C6D0001349012021F09AFB1249032021F096FB17
:10C6E0000C37BD46F0BDF31D23F00703ADEB030D82
:10C6F0006D4632462946204625F0A8F900213B79AF
:10C700002A460846FFF7B2FF40F225410EF06CFDC5
:10C71000E6E700BF482E00200AD205003FD2050000
:10C72000EAD7050013D2050070B5294C29492068C5
:10C73000002227F0F5FE054618B1002101200EF079
:10C740001FFC284626F066FB00222349206827F0BC
:10C75000E7FE054610B101200FF05CF9284626F0EF
:10C7600059FB00221D49606827F0DAFE00220546C9
:10C770001B49606827F0D4FE014606462846FFF7AD
:10C780002FFE2846314627F0B8FB00221549606885
:10C7900027F0C6FE054611F017F8284626F03AFBAA
:10C7A00060681149002227F0BBFE044608B1FFF77C
:10C7B0005FFF204626F02EFB0EF094FF0B4B1B680C
:10C7C0009B0503D5BDE87040FCF73EBB70BD00BFC4
:10C7D000482E0020FFD10500EBCD05006BD10500F0
:10C7E00075D1050002D305000AD20500BCC20020A5
:10C7F0002DE9F043B0F80B3091B003F50073044617
:10C80000A0F80B3003A88846174617F07BF890B3C2
:10C810000121294816F02EFC054648B31FFA88F07E
:10C8200026F0E4F925490246204627F04CFE002276
:10C830002349204627F074FEDDF826900090064636
:10C840001FFA88F30022394603A8C847002816DAE1
:10C850001C49042021F0DAFA012026F0BFF91A4918
:10C860000246204627F02FFE2946304627F045FB9A
:10C8700003A816F0E3FF204611B0BDE8F0830130B5
:10C8800026F0B4F911490246204627F01CFE022F7B
:10C890000DD101210E4816F0EDFB07460028E3D02C
:10C8A000214627F037FD384626F0B4FADCE721466A
:10C8B000284627F02FFDD7E72ED90500D4DA05004A
:10C8C000B7D4050046D905005FD9050066D9050033
:10C8D0006BD9050037B50190B0F80B300C4C03F55F
:10C8E0000073A0F80B300D46214627F0D5FD2946F0
:10C8F00002220198FFF77CFF26F08CFA01980123B1
:10C9000001AA21461CF014FB019803B030BD00BF02
:10C91000AFD405002DE9F0478EB00546884616468F
:10C9200025F04BFC814620B128460021FCF73AFF58
:10C930000546284625F01FFB044638B946482946D7
:10C9400021F044F920460EB0BDE8F087B8F1000FA1
:10C9500007D0404625F02AFB044610B941463F481F
:10C96000EEE7022E16D101A816F072FF90B1002258
:10C970003B49284627F0D4FD28F01AF9DDF80D30A0
:10C98000834204DACDF80D0001A816F05AFF01A881
:10C9900016F054FF0121334816F06CFB07460028BF
:10C9A00058D0012E4BD1304900201FF02DFB0446FA
:10C9B00048B9384626F02EFAB9F1000FC2D0284601
:10C9C00026F028FA2CE0294900201FF01DFBA24682
:10C9D0000446F4B13146204616F03EFBB8F1000F94
:10C9E00006D0234A4146204627F0EFFD26F012FAF2
:10C9F0002146384627F08EFCBAF1000F04D052468B
:10CA00001C49204627F048FD2A461B49204627F0AE
:10CA100043FD3946504627F070FAB9F1000FCED1E8
:10CA2000002E8FD101A816F06DFF00288AD001A832
:10CA3000214616F0F7F801A816F000FF82E7022E53
:10CA40000CBF0E490E4900201FF0DEFA4FF0000A1D
:10CA50000446BEE70446E0E79AD80500FCD8050086
:10CA6000CAD80500D9D80500E0D80500E8D80500E7
:10CA700023D9050030E40500B7D40500F0D805003F
:10CA8000F5D80500F0B58FB0054601A80F4616F0A1
:10CA900039FFA0B3284625F06EFA58B1194827F09F
:10CAA00023F9194A01460446284627F081FD21460C
:10CAB00027F023FA384627F0BBFA064668B125F07E
:10CAC00075FA044648B91148314621F07FF83046DE
:10CAD00026F0A0F920460FB0F0BD304626F09AF9B6
:10CAE000012239462846FFF715FF044618B10146D2
:10CAF00001A816F02BFA01A816F0A0FEEAE70446FA
:10CB0000E8E700BFB4DA0500B8DA0500FCD8050094
:10CB100070B592B004460D46014601A8164617F0BE
:10CB2000BBF960B33EB140F2FF339D42A8BF1D4642
:10CB3000012DB8BF0125BDF91830002B11DA2B04E7
:10CB40000FD41049204628F0EDF80F49204628F070
:10CB5000E9F80E49204628F0E5F80D49204628F06E
:10CB6000E1F801A8ADF8185017F072F9B4F80B30DD
:10CB700003F50073A4F80B30204612B070BD0446D4
:10CB8000FAE700BF20D7050025D7050048D60500E5
:10CB90002AD705002DE9F843074608460D461446F6
:10CBA00025F00BFB002800F0848001224249284632
:10CBB00026F0BEFB0646C8B3284626F0AAFD062886
:10CBC00094BF4FF0FF384FF006083A21284626F070
:10CBD0005FFC00282DDB00F1010841466FF00042A8
:10CBE000284626F0BCFC27F0E3FFB8F1010FB8BFE0
:10CBF0004FF00108044608F1FF322846002126F0D4
:10CC0000AEFC054641F6FF739C42A8BF1C46012CB2
:10CC1000B8BF0124BEB1A4B2284626F0FBF83246C4
:10CC200021463846BDE8F843FFF772BF4FF0FF38A2
:10CC3000CBE7B8F1FF3FD0D1B5F80B3003F5007367
:10CC4000A5F80B30DEE715B904F50054E3E72846F4
:10CC500026F05FFD0028F7D01849284626F070FB23
:10CC60000028F1D12946164826F08AFC32460146B2
:10CC70008046384621F0D0F98146B8B13346324675
:10CC800039461DF059FD26F0C5F8A4F50044A4B2BC
:10CC90004146484627F031F94FF6FF739C42BBD11D
:10CCA0002A460849012021F0B1F8B5E74FF6FF7494
:10CCB000EEE7BDE8F88300BF37D605003ED6050095
:10CCC00084D605008ED6050001381F289DBF034B72
:10CCD00023FA00F000F00100002070478B80808074
:10CCE00030B551EC100B85B053EC112B8DED000BD2
:10CCF00055EC124B8DED021B2DF096FD9DED000BBA
:10CD000028B19DED021BB0EE410AF0EE610A53EC32
:10CD1000102B204629468DED000B2DF085FD9DED55
:10CD2000000B08B145EC104B05B030BD38B555ECE3
:10CD3000104B0022002310EE100A29462DF074FD3E
:10CD400010B105F100431D4645EC104B38BD10B441
:10CD500013460A4653F8044B0021A4465DF8044BE1
:10CD6000604728F00FB800000022014921F0DAB92D
:10CD700043E0050000B593B0014601A817F08CF818
:10CD800008B19DF80F0013B05DF804FB2DE9F04FDA
:10CD90009DB00BAD80460F460146284616461C4600
:10CDA00017F07AF80290002800F09B80269B0A93E7
:10CDB00008AA07A92846CDE90776099416F08AFF44
:10CDC0000AAA09A9284616F085FF0798099B089921
:10CDD0000A9CC21802EBD27252101B1A009203EB8B
:10CDE000D3730A19641A5B1004EBD47464100593AE
:10CDF0005B43039302EBD27204FB04F352100493DF
:10CE00000192DDE903326600013E03FB162600278E
:10CE1000009B03EB070B019B03EB040A52460E9B9E
:10CE20005946284616F0C4FE009BA3EB070952465C
:10CE30000E9B4946284616F0BBFE019BA3EB040A55
:10CE400052460E9B5946284616F0B2FE28460E9BC7
:10CE50005246494616F0ACFE049A7B0003FB0222C0
:10CE600071009142BFBF049A0298033302FB03662C
:10CE70004FEA440C039BCCF1010203FB02F2B4BF66
:10CE800001370020914208DD039AACF10303013C15
:10CE900002FB1366002CBBDA01E00028FAD1059BE7
:10CEA000BB4207F101040CDC284616F0D1FFB8F8AC
:10CEB0000B3003F50073A8F80B3040461DB0BDE8F9
:10CEC000F08FDDE900120E9B2144284616F070FE1B
:10CED000DDE900120E9B091B284616F069FE274665
:10CEE000DDE7DDF80880E8E713B51C46134400933E
:10CEF000121B0B19091BFFF749FF02B010BD2DE9EA
:10CF0000F04F9FB00DF1340A80460E460146504660
:10CF100015461C4616F0C0FF0390002800F08980DB
:10CF2000289B0C930AAA09A95046CDE909650B94E0
:10CF300016F0D0FE0CAA0BA9504616F0CBFE0999AC
:10CF40000B9B0C9CCDF818A0CA1802EBD2725210A1
:10CF500002920A9A1519A41A5B1A04EBD47464108D
:10CF600003EBD3735B10660005EBD575059304FBEB
:10CF700004F95B43013E6D10049303FB16960027F2
:10CF80007B0003FB099271009142BCBF033309FB94
:10CF900003660498B8BF039A4FEA44030793C3F1AA
:10CFA000010300FB03F3B4BF0137002299421FDDE8
:10CFB000029B069803EB070AA3EB070B109B2A19A9
:10CFC000CDE9002351465B4616F0B6FC109B06984F
:10CFD0002A1BCDE9002351465B4616F0ADFC079BAA
:10CFE000049A033B013C02FB1366002CC8DA01E003
:10CFF000002AFAD1059BBB4207F101040CDC0DA805
:10D0000016F026FFB8F80B3003F50073A8F80B30C4
:10D0100040461FB0BDE8F08F109B0299CDE9005348
:10D02000029B2A461B1B21440DA816F085FC2746AF
:10D03000E0E7DDF80C80EBE713B51C4613440093E2
:10D04000121B0B19091BFFF75AFF02B010BDF0B5F8
:10D0500099B004460F46014607A816461D4616F02D
:10D060001BFF002840D01E9B069304AA03A907A813
:10D07000CDE90376059516F02DFE06AA05A907A8A9
:10D0800016F028FE049A0A9B0399CDE9002307A80D
:10D09000059B16F051FC0A9B0193069B0093DDE96A
:10D0A000042307A8194616F047FC069A0A9B039921
:10D0B000CDE9002307A8059B16F03EFC0A9B0193CF
:10D0C000049B0093039B069A194607A816F034FCAC
:10D0D00007A816F0BDFEB4F80B3003F50073A4F8F2
:10D0E0000B30204619B0F0BD0446FAE7F0B595B014
:10D0F00004460D46014603A816461F4616F0CCFE10
:10D10000A8B1079B01931A9B009332463B462946E0
:10D1100003A816F05AFE03A816F09AFEB4F80B30D6
:10D1200003F50073A4F80B30204615B0F0BD04469B
:10D13000FAE7F0B595B004460D46014603A8164639
:10D140001F4616F0A9FEA8B1069B01931A9B0093F7
:10D1500032463B46294603A816F037FE03A816F0D0
:10D1600077FEB4F80B3003F50073A4F80B302046BB
:10D1700015B0F0BD0446FAE770B592B00546014619
:10D1800001A816F089FE68B39DF80830012B83BF13
:10D19000154B1A6804924FF0FF338EBF5B680493FF
:10D1A00000230593BDF80B30013BADF82330BDF8EB
:10D1B0000D30013BADF82530079B03F440030024FC
:10D1C00042F2010643F4702301A806960793ADF8D6
:10D1D00020408DF8224016F03BFE2246314628467C
:10D1E000FFF796FC12B070BDC8C2002010B504460F
:10D1F00094B019B1FFF7C0FF25F00CFE214603A83B
:10D2000016F04AFEC8B1079A0192BDF81520BDF884
:10D210001330013A00920022013B114603A816F098
:10D220008BFB03A816F014FEB4F80B3003F5007363
:10D23000A4F80B30204614B010BD0446FAE70000F5
:10D240002DE9F0478AB0804624F0B7FF044638B98C
:10D250004849032020F0DAFD20460AB0BDE8F087F7
:10D2600000224146684620F050FA00273D463E46DF
:10D270003C464FF00009DDE900329A4225D8039878
:10D2800025F0C8FD25F09DFC04460028E4D030467A
:10D2900025F0ACFC38490246204627F014F9284610
:10D2A00025F0A4FC35490246204627F00CF905FB81
:10D2B00006F007300021C01026F0BEFC0546C0B9BC
:10D2C000204625F0A7FD2C46C6E7684620F016F953
:10D2D0000A2805D159EA040308BF01270134C8E729
:10D2E000AC4209F10109A8BF651C4E45B8BF4E46C6
:10D2F000C1E73A464146684620F007FA4FF0000879
:10D3000047464FF08009DDE900239A4208D303988D
:10D3100025F080FD2A461A49204627F0D4F89BE7DD
:10D32000684620F0EBF80A2803D108F1010800272D
:10D33000E9E720281CD0284624F03FFFC0B106FBB7
:10D34000087A29464FEADA0205A820F0DEF90999A1
:10D3500009B1059BC95C0AF0070A49FA0AFA41EAD1
:10D360000A0105A8C9B220F02DF8089825F052FD51
:10D370000137C8E7BFDD0500ECD40500F2D4050095
:10D3800018EA0500024B03495868002227F0C8B884
:10D39000482E0020AB17060070B5002286B00E465E
:10D3A000114927F0BDF8054624F007FF044660B197
:10D3B0000022294601A820F0A8F90024DDE9012374
:10D3C0009A4208D3049825F025FD284625F022FD31
:10D3D000204606B070BD01A820F090F8B04208BF0A
:10D3E00044F00104E4B2E9E784E4050070B50446C2
:10D3F00024F0C1FD30B900242546204625F00AFD61
:10D40000284670BD00221449204627F089F80546B9
:10D4100024F0B1FD044618B9284625F0FBFCEBE7E3
:10D42000002DE8D000220D49284627F079F804465F
:10D4300024F0BCFD50B1284625F0ECFC002CDBD0DC
:10D44000074D2368EB1A5D425D41D6E72946204629
:10D4500026F053FDCFE700BF43E005005EEC05007A
:10D4600069240300014900201EF0CEBD73AF050002
:10D47000014900201EF0C8BD6CE5050001490020EF
:10D480001EF0C2BD45AF05002DE9F04390461D4694
:10D49000421E47F6FE739A4293B006460F4602D8E4
:10D4A0004A1E9A4208D93249012020F0AFFC0024DC
:10D4B000204613B0BDE8F0834046FFF705FC044664
:10D4C00020B92C49012020F0A1FCF1E7284624F0E6
:10D4D00052FDD8B100222849284627F021F8002221
:10D4E00004462649284627F01BF82546814628464B
:10D4F00024F05CFD044688B92A462149012020F029
:10D5000085FC4946284626F0F8FCD1E7B5F80B30F3
:10D5100003F50073A5F80B308146E8E7B9F1000F79
:10D5200006D0484624F042FD044608B94A46E4E7DE
:10D53000144900201EF068FD04460028B8D00123DD
:10D540008DF808303A464346314601A816F030FDC2
:10D550002A460D490194204626F09EFF4A460B4973
:10D56000019826F099FF01A816F072FCC9E700BFE8
:10D570004CDD050059DD050065DD05006EDD0500AB
:10D5800077DD05003ED50500ABDD0500B5DD050006
:10D5900070B506460D4624F010FE044630B93246FA
:10D5A0001349032020F032FC204670BD11490020B1
:10D5B0001EF02AFD32461049044626F06DFF45B1A3
:10D5C000284624F0FAFD68B932460949032020F0C4
:10D5D0001DFC002025F00AFB08490246204626F0E3
:10D5E00072FFE1E72A460649204626F055FFF0E79C
:10D5F00041E405006CE4050073E405007AE40500ED
:10D6000084E4050038B500220849054626F088FF65
:10D61000044640B906491EF0F7FC04490446024698
:10D62000284626F039FF204638BD00BFEB2406000F
:10D6300034E405002DE9F04391461D46421E47F6AD
:10D64000FE739A4293B00746884602D84A1E9A4211
:10D6500005D96749012020F0D9FB002408E048469D
:10D66000FFF732FB044638B96249012020F0CEFBB7
:10D67000204613B0BDE8F0835F4900201EF0C4FCD3
:10D6800004460028F4D0002601A84B4642463946FD
:10D690008DF8086016F08CFC28468DF809608DF82E
:10D6A0000A60019424F067FC00285CD0324653499C
:10D6B000284626F035FF27F0B4FB28B1BDF8093025
:10D6C00043F00103ADF8093000224D49284626F009
:10D6D00027FF27F0A6FB28B1BDF8093043F004036B
:10D6E000ADF8093000224749284626F019FF27F0F7
:10D6F00098FB28B1BDF8093043F00803ADF80930B4
:10D7000000224149284626F00BFF27F08AFB88B10A
:10D710009DF80F0001280BD1BDF8093043F002033A
:10D72000ADF80930BDF80D305B0703D0374992E7FB
:10D7300037498FE728460022364926F0F1FE054694
:10D7400088B1354925F0FCFD50B93449284625F00B
:10D75000F7FD08BBBDF8093043F08003ADF8093090
:10D76000284625F057FBBDF80D00BDF80B304343AC
:10D770009DF80F0058430730C00808F045FC284AC0
:10D7800005460146019826F020FF294626F0B5FB04
:10D7900001A816F05DFB6BE72249284625F0D0FD75
:10D7A00020B9BDF8093043F48073D7E71E492846F5
:10D7B00025F0C6FD20B9BDF8093043F4C073CDE7AC
:10D7C0001A49284625F0BCFD20B9BDF8093043F4BC
:10D7D0000073C3E71649284625F0B2FD20B9BDF80D
:10D7E000093043F42073B9E7124820F0CFF9B7E7C6
:10D7F0004CDD050059DD05003ED5050079DC05004E
:10D8000080DC050084DC050090DC0500CEDC050032
:10D810009EDC050007DD050013DD050017DD0500B2
:10D8200018EA05001BDD05001FDD050023DD0500EE
:10D8300027DD05002BDD050008B500222DED028B4C
:10D84000B0EE408AF0EE608A002351EC100B2CF011
:10D85000FFFF98B1B0EE480AF0EE680A2AF0C0FD6A
:10D860000B4B51EC100B00222CF06CFDBDEC028B2D
:10D8700041EC100BBDE808402AF02EBDBDEC028B38
:10D880009FED010B08BD00BF000000000000F87F05
:10D890000000E03F00000000F8B555EC104B25F00B
:10D8A00000474FF0FF32284B204639462CF0E4FF6A
:10D8B00060B94FF0FF32244B204639462CF0D2FF9E
:10D8C00020B9B5F1004F08BF002C05D145EC104B35
:10D8D000BDE8F84025F078B900220023204629460B
:10D8E0002CF0A2FFC8B912A1D1E900012B462246B3
:10D8F0002CF072FB06460F462DF084F804460D46C8
:10D9000054EA05030DD100220023304639462CF09D
:10D910008BFF30B19FED080BDAE709A1D1E90001D7
:10D92000E4E720462946BDE8F84025F074B900BF79
:10D930002083E4FFFFFFDF3F0000000000000080C5
:10D940002083E4FFFFFFDFBFFFFFEF7F2AF0C0BCB3
:10D950002AF042B938B555EC104B10EE102A2B4680
:10D9600010EE100A29462CF0EDFC02460B46002072
:10D9700009492CF02FFB41EC100BFFF75DFF20460F
:10D9800053EC102B29462CF007FEBDE8384041EC43
:10D99000100B2AF021B900BF0000F03F2AF038BC7C
:10D9A00030B591B0054624F035FC044638B92A4616
:10D9B0001F49032020F02AFA204611B030BD012271
:10D9C000294605A820F04DFC00231A4605A9194850
:10D9D00016F0ECFB044605A81FF036FA204600219D
:10D9E00026F02AF9044618B9134820F0EFF8E3E7C7
:10D9F0002946012205A820F034FC21460022684671
:10DA00001FF083FE6B460D4A0A4805A916F0CEFBAF
:10DA1000039825F0FFF905A81FF016FA002120460B
:10DA200025F001FF0546204625F0F4F92C46C3E712
:10DA3000D2DD05002709040033D40500490904009C
:10DA400030B591B0054624F0E5FB044638B92A46C6
:10DA50001F49032020F0DAF9204611B030BD012221
:10DA6000294605A820F0FDFB00231A4605A9194800
:10DA700016F090FC044605A81FF0E6F920460021A8
:10DA800026F0DAF8044618B9134820F09FF8E3E7C7
:10DA90002946012205A820F0E4FB21460022684621
:10DAA0001FF033FE6B460D4A0A4805A916F072FCBA
:10DAB000039825F0AFF905A81FF0C6F9002120460C
:10DAC00025F0B1FE0546204625F0A4F92C46C3E713
:10DAD000D2DD05002709040033D4050049090400FC
:10DAE000F8B5051E0C4606DC2949012020F08EF908
:10DAF00000242046F8BD084624F03DFA0646A8B1A9
:10DB000000222449204626F00BFD27F08AF9002246
:10DB100021490646204626F003FD27F049F830F05B
:10DB2000080309D0102809D01C49DEE724B1224699
:10DB30001B49012020F06AF9012400E00224294653
:10DB4000204625F08DF907469EB12946204625F04E
:10DB500087F90546134900201EF056FA044610B115
:10DB60000FB146B13DB92A463946204626F0B8F9EC
:10DB7000BEE73546EEE73A460B49204626F0A3FCC1
:10DB8000002DB6D02A460949204626F09CFCB0E775
:10DB9000A7E60500C6E60500E5E60500D3E60500B4
:10DBA000EAE6050021E7050018EA05002AE7050076
:10DBB00038B5044624F0DFF988B10022094920462F
:10DBC00026F0AEFC054624F0F8FA10B1284625F000
:10DBD000A0FD0446284625F01DF9204638BD044620
:10DBE000FBE700BF5AE60500F8B506460D460AB346
:10DBF000104626F03BFA002D044603DA304625F0A5
:10DC000088FD0544002C03DA304625F082FD0444EB
:10DC10001B2024F05BFF25EAE57524EAE47407463F
:10DC200030B1A54204DA631B2A46314625F06AFC6E
:10DC30003846F8BD00296FF00044E9DADEE7F8B5B0
:10DC400005460C46C2B1104626F010FA20EAE076EE
:10DC5000002C05DA284625F05CFD044424EAE4742F
:10DC60001B2024F033FF074620B1334622462946C5
:10DC700025F048FC3846F8BD6FF00046E8E7F8B5F7
:10DC800007460C46CAB1104626F0F0F920EAE075C6
:10DC900024EAE474A542B8BF23464FF01B00BCBF82
:10DCA0002C461D4624F012FF064620B12B1B2246AF
:10DCB000394625F027FC3046F8BD6FF00040E5E717
:10DCC00070B50D1E064606DA0B49012020F09EF8BD
:10DCD0000024204670BD1B2024F0F8FE044615F1F8
:10DCE000FF35F6D31EF0B4FD0028F2D131462046B0
:10DCF00025F030FCF3E700BF93E60500F8B50646D3
:10DD00000F46154624F059FA044698B1284624F0E7
:10DD100073F988B1284626F0A9F90446384627F059
:10DD2000D9F8054625F0F5FC241A09D50024284623
:10DD300025F070F82046F8BD304625F0EAFCECE707
:10DD4000284625F0E6FC0719304625F0E2FC87421C
:10DD5000ECDC2246012329463046F2F7D5FCB0FA26
:10DD600080F46409E3E7F8B507460E46154624F04B
:10DD700024FA044648B1304627F0ACF8002D064698
:10DD800005DA0024304625F045F82046F8BD25F098
:10DD9000C0FC4419384625F0BCFC8442F1DC012368
:10DDA0002A4631463846F2F7AFFCB0FA80F46409EF
:10DDB000E8E72DE9F04186B027F08CF80546E0B1A0
:10DDC0000146002201A81FF0A0FC4FF0FF340026FE
:10DDD000DDE90183984514D3049825F01BF8A64289
:10DDE000DABFA21B013200223146284625F0B7FBDC
:10DDF0000446284625F00EF82546284606B0BDE81C
:10DE0000F08101A8039F1FF079FB1EF07BFF002823
:10DE1000DED107EB080336EA240628BF1E461C465F
:10DE2000D6E7000070B505460E4624F0A4F858B9B0
:10DE3000284624F061F8044630B92A460E490320EA
:10DE40001FF0E4FF204670BD304624F094F818B16E
:10DE50000A4901201FF0DAFF24F0B3FE044600282F
:10DE6000F0D0284624F087F80028EBD02A46044951
:10DE7000204626F011FBE5E7CADE0500FDDE0500C1
:10DE800043E0050008B508B1036823B91B20BDE8CD
:10DE9000084024F01BBE002126F0D8F8BDE8084059
:10DEA00027F017B908B525F016FB08BD70B5054673
:10DEB00086B01B200E4624F009FE0446E0B1284639
:10DEC00024F07BF9C0B1002E16DB3246294601A8AA
:10DED0001FF01BFCDDE901239A420AD2059B03B126
:10DEE0009B5C8DF8033001220DF10301204625F0E3
:10DEF00089FB049824F08EFF204606B070BD37B52C
:10DF000005461B2024F0E2FD044628B1294601A85D
:10DF10001FF00EF8019810B9204603B030BD26F06E
:10DF200087F826F045FE01228DF803000DF103016C
:10DF3000204625F067FB01A81EF0E9FFEAE7000094
:10DF4000F8B507460E4624F016F888B300221949A2
:10DF5000384626F0E5FA054624F02FF918B328468E
:10DF600025F0D7FB002E01DD86420AD31149384641
:10DF700026F0D8FE2C460025284624F04BFF2046EC
:10DF8000F8BD32460021284625F0E9FA314604461C
:10DF90006FF00042284625F0E2FA0649024638466C
:10DFA00026F091FAE8E71B2024F090FD0446E3E711
:10DFB0000446E4E75AE605002DE9F041CB1D23F0C5
:10DFC000070300AFADEB030D134614466E460D4636
:10DFD00053F8048B0A463146C047A3692B44A3611A
:10DFE00063692B44636135441C34AE4202D1BD46A3
:10DFF000BDE8F081204616F8011B1FF0EAF9204623
:10E000001FF04FF8F1E700002DE9F0478EB002AFA6
:10E010000D46144680461AF0E7FF4FF00109064608
:10E02000F91D284687F80790F3F748FC002C824634
:10E0300005DC002630463037BD46BDE8F0871EF0CF
:10E040000FFC04F58073834204D93A4948461FF017
:10E05000DDFEEEE7E31D23F00703ADEB030D122E0B
:10E0600002AD3AD1344B1B78C3B1002307F108024B
:10E070004FF040213148C7F80A30C7F80E307B8294
:10E0800087F8089087F809A0BC72FD60F7F78EFA50
:10E09000024618B12A4904201FF0B8FE214601208B
:10E0A00024F0DEFE06460028C3D00146002207F118
:10E0B000080020F0A7F82C4415F8011B07F1080010
:10E0C0001FF087F907F108001EF0EBFFA542F3D11E
:10E0D00007F108001EF0B2FEACE7002EA9D11949E5
:10E0E0003246404626F01CFA8146014607F10800F8
:10E0F0001AF0E0F988B132461349404626F010FA8A
:10E1000026F08FFEFB79B873009322462B465FFA08
:10E110008AF107F108001AF025F9B87B24F05EFDBA
:10E1200009490246404626F0B7F9494625F0E5FE82
:10E13000B4E700BFF7DD050098C200203CBB00201B
:10E140002CDE05003FDE050048DE05002DE9F04F1E
:10E1500089B002AF0C46164681461AF045FF4FF0D3
:10E16000010BF91D0546204687F807B0F3F7A6FB1B
:10E170000023824607F108013046BB6025F014FBFE
:10E180000446002E43D0F0B9304623F03BFB8046D6
:10E19000B8601EF065FB08F58073834207D93349E8
:10E1A00058461FF033FE1C37BD46BDE8F08F08F11E
:10E1B000070323F00703ADEB030D02AC42462146F3
:10E1C000304623F043FCBB68002BECD0122D21D14C
:10E1D000274A1278002AE6D0F97926483C610022C5
:10E1E0009142FA607A61BB734FF0402114BF13462D
:10E1F000202307F10C0287F80DA0F7F7D7F90246A4
:10E200000028D0D01C4904201FF000FECBE70028D6
:10E21000C9D0D8E7002DC6D118492A46484626F06D
:10E220007FF90646014607F10C001AF043F988B160
:10E230002A461349484626F073F926F0F2FDFB7989
:10E24000B8740093BA6823465FFA8AF107F10C00AC
:10E250001AF0EAF8B87C24F0C1FC094902464846A5
:10E2600026F01AF9314625F048FE9CE7EAD705006A
:10E2700098C200203CBB00209CDE05003FDE05006C
:10E2800048DE05002DE9F74F0D4603210446CDE990
:10E29000002313F009F94FF0000B4FF0010A4FF083
:10E2A0008008D94615F1FF3502D203B0BDE8F08FE2
:10E2B000009B0AEA0306019B0BEA030756EA0703E1
:10E2C00016D088F311880021204612F073FE0A2030
:10E2D000F3F74EFC0121204612F06CFE89F3118801
:10E2E0003720F3F745FC1AEB0A0A4BEB0B0BD9E787
:10E2F00088F311880021204612F05CFE4120F3F7DC
:10E3000037FC0121204612F055FE89F311880520C3
:10E31000E7E710B40C7802460023204608215DF898
:10E32000044BFFF7AFBF00002DE9F04F89B08946DD
:10E3300000901AF059FE4946044602A81AF0BAF8AD
:10E34000F0B1122C40F0F8809DF80C4020461AF0F5
:10E3500045FF9DF80D5018B128461AF03FFF90B9BF
:10E360002246294685481FF031FCB9F1000F00F024
:10E370000081834A0098494626F01AF924F04AFDA4
:10E3800009B0BDE8F08F7F49029E7F4B04EB840407
:10E3900005EB85050C440D449E4294F801806F788E
:10E3A00058DD7A4B9E42D4BF4FF080664FF0CD6669
:10E3B000774A784C13785BB323681BB1764B1021F6
:10E3C000C3F880104FF040234FF0FF31C3F808131B
:10E3D000D3F800120021C3F80012C3F80015012180
:10E3E00084F8221094F8271079B9D3F808154FF063
:10E3F000A04001F5E07140F2023540F82150D3F819
:10E400000C3503F5E07340F82350002384F82230E4
:10E4100094F8223001251570FBB108225F490420D1
:10E420001FF0F4FC9DF80C4020461AF0D7FE20B1F6
:10E430004FF42071204612F0B7FE9DF80D402046A3
:10E440001AF0CCFE002890D04FF49451204612F0E0
:10E45000ABFE8AE74FF0CC76AAE79DF81E2084F841
:10E4600027209DF81D20A360C4E9003384F82530DF
:10E4700084F8243072B34FEA8800B90000F1A0405C
:10E4800001F1A04140F20C624FF0A04BC0F8002710
:10E4900005FA08FAC1F80027BD4040F20D62019369
:10E4A000CBF808A5CBF80855C0F80027C1F800271D
:10E4B0000420F3F719FB019BDBF810150D422BD05C
:10E4C00043B14FF0A04A0420CAF80C55F3F70CFBF7
:10E4D000CAF808554FF0A04308F5E07140F20C620D
:10E4E00043F8212007F5E07143F821204FF0402345
:10E4F0001D46C3F80885C3F80C75C3F82465226867
:10E500001AB106210420F7F72DFA0523C5F80035C6
:10E51000022384F8223085E701930420CBF80CA570
:10E52000F3F7E2FACBF808A50420F3F7DDFA019B34
:10E530000133092BC0D1C4E7002C7FF416AF9DF83E
:10E540000C00FF2807D0012112F034FD03219DF8B3
:10E550000C0012F0A9FF9DF80D00FF283FF405AF55
:10E56000012112F027FD03219DF80D0012F09CFF00
:10E57000FBE60349009826F0D5FB01E750DE0500D5
:10E580003FDE05003CB0050097AB020087F50400B4
:10E5900098C200203CBB002000E100E07FDE0500C7
:10E5A000F0B58DB00D4616461C461AF01DFD11281B
:10E5B0009DF8487005D02F4901201FF027FC0DB0B1
:10E5C000F0BD16B90CB90F2403262B4B1B78F6B2FD
:10E5D000E4B25BB92949ADF810306FF0FF02CDE924
:10E5E000011201A8264A039212F0FCFDFF2F03D06E
:10E5F000002138461BF0A0FA284623F0FDFC80B12C
:10E60000284625F033FD22463146C0B2F2F7F8FF26
:10E61000F2F7A6FEFF2FD2D0012138461BF08CFA6C
:10E62000CDE7284623F0F6FDE8B1802383F3118877
:10E630000122294601A81FF014FE01A81EF030FC9B
:10E64000054601A825B91EF0FFFB85F31188DFE719
:10E650001EF00BFE22463146C0B2F2F7D1FF01A8F0
:10E660001EF039FDE9E72A46064901201FF0CEFBDE
:10E67000CEE700BF70E505007CC20020A086010047
:10E680000001080098E50500F0B58DB00D4616466E
:10E690001C461AF0A9FC11289DF8487005D0304995
:10E6A00001201FF0B3FB0DB0F0BD16B90CB9032467
:10E6B00001262C4B1B7806F00F0604F00F045BB903
:10E6C0002949ADF810306FF0FF02CDE9011201A821
:10E6D000264A039212F086FDFF2F03D00021384610
:10E6E0001BF02AFA284623F087FC80B1284625F043
:10E6F000BDFC22463146C0B2F2F742FFF2F730FECF
:10E70000FF2FD0D0012138461BF016FACBE7284660
:10E7100023F080FDE8B1802383F31188012229468C
:10E7200001A81FF09EFD01A81EF0BAFB054601A836
:10E7300025B91EF089FB85F31188DFE71EF095FDF2
:10E7400022463146C0B2F2F71BFF01A81EF0C3FCFF
:10E75000E9E72A46064901201FF058FBCEE700BF33
:10E7600048E505007CC20020A086010000010800E9
:10E7700098E50500F0B58BB004460D461AF034FC60
:10E7800001AE07463246694620461AF03BFC98B374
:10E79000009B059396E80F0006AC07C423807DB369
:10E7A000296800292CDD0139284625F04FFC064652
:10E7B00023F0FCFD10B330461AF098FC04462846BE
:10E7C00026F07AFA24F026FB304624F023FBFF2CB7
:10E7D00003D0002120461BF0AFF905AA09492846BD
:10E7E00022F016FF112F01D1F2F7BAFDFF2C03D052
:10E7F000012120461BF0A0F90BB0F0BDFF24E3E798
:10E80000FF24EAE74FCD02002DE9F041B8B00D46F4
:10E81000164607A908AA1AF0F5FB002877D0FF2EA4
:10E8200003D0002130461BF087F9284623F0E4FB93
:10E8300080462846B8F1000F18D025F017FC18A91B
:10E840008DF8600008AB08460122079CA0479DF8A0
:10E85000600024F0CBF90446FF2E03D0012130469E
:10E860001BF06AF9204638B0BDE8F08123F0A5FC22
:10E870000746002831D01B2024F028F942460446E0
:10E88000294602A81EF041FFDDE902239A4203D384
:10E89000059824F0BFFADFE71DF0DAFF0028F7D172
:10E8A00001AA694602A81EF0ADFB019D002DEBD028
:10E8B000802D28BF802508AB2A4618A90098079FFD
:10E8C000B8472A4618A9204624F09CFE019B5B1BF2
:10E8D0000193009B1D440095E7E7284622F092FF34
:10E8E0000146012024F0BCFA04460028B4D03A4680
:10E8F00001460EA8CDE90C771FF084FC07AA054954
:10E90000284622F085FE0EA81EF098FAA4E70446D9
:10E91000A8E700BFB9DF02007FB50C4605461AF034
:10E9200063FB21460646684619F004FB60B1112ED0
:10E930000CD1684612F056FC04B3134A214628460F
:10E9400025F036FE24F066FA04B070BD002EFBD12F
:10E950009DF80500FF2802D0012112F0A5FD9DF8C9
:10E960000600FF2802D0042112F09EFD9DF807004A
:10E97000FF28E1D0012112F097FDDDE7024928468A
:10E9800026F0D0F9E0E700BF3FDE05002DE9F043B7
:10E9900000228DB02449064625F0C2FD05AD014692
:10E9A000284627F003FD1B22541E295D09B1144699
:10E9B00002E02246002CF7D10CAB4FF001081C44BA
:10E9C0000DF1240904F81C8C99E807008DE8070074
:10E9D00095E80F0027F03BFB08F1010807460028E7
:10E9E000F0D1012024F002F910490246304625F00A
:10E9F0006AFD384624F0FAF80D490246304625F003
:10EA000062FD384624F0F2F80A490246304625F005
:10EA10005AFD384624F0EAF80749024630460DB060
:10EA2000BDE8F04325F04FBDF4D90500E9E5050048
:10EA3000EFE50500F6E505003BF405002DE9F04F94
:10EA40000022A1B00E466E49054625F069FD26F06C
:10EA5000AFF8C0B2722808D06A4901201FF0D6F979
:10EA60000027384621B0BDE8F08F002266492846CD
:10EA700025F056FD26F09CF88046002800F0BD8069
:10EA800000226249284625F04BFD26F091F800222D
:10EA90005F498146284625F043FD26F089F800228B
:10EAA0005C498246284625F03BFD26F081F800228D
:10EAB00059498346284625F033FD014609A827F029
:10EAC00075FC1B22531E09A9C95C09B1134602E05B
:10EAD0001A46002BF6D120AAD318069303F85CBC83
:10EAE000F30F059318BF202600273EBB7CE04FF0B4
:10EAF000000846E012F8011BFF291CD005980133DD
:10EB000000286CD00A296AD100221C46059237B928
:10EB10001B20079323F0DAFF079B074630B12246FC
:10EB200010A93846079324F06DFD079B059AA14470
:10EB30001AB91E1BD9E71C4654E02026AAEB09048B
:10EB4000002C3DDCBBF1FF0FD1D0069B0BF1010B7C
:10EB500003F85CBC18AB03930DAB93E807008DE89A
:10EB6000070009AB0FCB27F080F9189B23F07F4AF1
:10EB70008046504624F03AF825490246284625F0BA
:10EB8000A2FC404624F032F81F490246284625F0F0
:10EB90009AFC002024F02AF81C490246284625F059
:10EBA00092FC584624F022F81A490246284625F0DD
:10EBB0008AFCB8F1000F3FF454AF54464FF00009FF
:10EBC000202E3346A8BF20239C42A8BF1C462246C5
:10EBD00009EB080110A82CF0C9F810AA0023A342E1
:10EBE00088DB3346002C92D1484623F0FFFF0749CB
:10EBF0000246284625F067FC33E7074631E700BFA9
:10EC00003BF40500FBE50500F6E50500EFE5050032
:10EC100013E60500E9E50500F4D905004FF0FF31E2
:10EC2000FFF70CBF21EAE171FFF708BF2DE9F04FB4
:10EC300000229BB00C469B49054625F071FC25F04F
:10EC4000B7FFC0B2772808D0612806D096490120C6
:10EC50001FF0DCF81BB0BDE8F08F204626F03AF933
:10EC600007460028F6D024F054FD81460028F1D054
:10EC700000228E49284625F053FC25F099FF0022FA
:10EC80008B498246284625F04BFC25F091FF002257
:10EC900088498346284625F043FC25F089FF002259
:10ECA00085498046284625F03BFC0BAC01462046B2
:10ECB00027F07CFB1B22531EE15C09B1134602E0E6
:10ECC0001A46002BF7D11AAA1A44CDE9082302F8F4
:10ECD0003C8C7A490022284625F022FC25F068FF6A
:10ECE0000646002845D0099BA0F120020DF1480EF0
:10ECF00010685168F446ACE803000832B242E646B8
:10ED0000F6D15A1C214613A82CF022F8A8B112AB58
:10ED100003930FAB93E807008DE8070094E80F001A
:10ED200027F0A3F8064608B9654990E723F05EFF8F
:10ED300062490246284625F0C6FBABEB0A0BD945D3
:10ED400056444FDB5A460021384624F008FC314631
:10ED5000824606F06BFB504624F05CF8B8F1FF0FDA
:10ED60004BD1584901201FF051F8384624F052F891
:10ED700070E74FF47E63CDE905034023CDE90373CB
:10ED80000FAE96E807008DE8070094E80F0027F023
:10ED90009FF90028E9D012AB039396E807008DE8AD
:10EDA000070094E80F0027F060F80646129820F05C
:10EDB0007F44484623F01AFF3C490246284625F086
:10EDC00082FB204623F012FF39490246284625F0EF
:10EDD0007AFB304623F00AFF38490246284625F0E0
:10EDE00072FBC2E73846314606F020FB09EB0A0009
:10EDF00023F0FCFE2D490246F0E7089B08F10100D4
:10EE000003F83C0C23F0F2FE2A490246284625F07E
:10EE10005AFB6FF000425946384624F0A0FB00230D
:10EE20004FF47E62CDE905324023CDE903030FAEF6
:10EE3000804696E807008DE8070094E80F0027F069
:10EE400047F9002891D012AB039396E807008DE8AC
:10EE5000070094E80F0027F008F80646129820F003
:10EE60007F44484623F0C2FE10490246284625F05A
:10EE70002AFB204623F0BAFE0D490246284625F01B
:10EE800022FB304623F0B2FE0C490246284625F00C
:10EE90001AFB404624F03DFC0446404623F0BAFFEE
:10EEA0002046A5E73BF4050017E60500EFE5050061
:10EEB00013E60500E9E50500F4D90500F6E50500CF
:10EEC00030E605004CE605002DE9F04F0022A5B024
:10EED0003B4925F025FB05AC01460546204627F0B9
:10EEE0004BFA284623F096FF1B235E1EA25D0AB153
:10EEF0001E4602E03346002EF7D124AB1E444FF0ED
:10EF000001080CAF06F87C8C0DF1240B03979BE8ED
:10EF100007008DE8070094E80F0026F0A6FF0546DD
:10EF2000002847D00C9B23F07F4303444FF0000997
:10EF300013F8013C0C9AFF2B22F07F4A02D0B8F163
:10EF4000FF0F1ED10024AAEB0406002E14DD412E73
:10EF500028BF40263246611914A82BF007FF14AAD7
:10EF6000002312F8011BFF2922D001339E42F8D161
:10EF700000221C44002AE6D004EB090025B0BDE8BD
:10EF8000F08F08F1010806F87C8C03979BE80700D6
:10EF90008DE8070094E80F0026F067FFD14405468E
:10EFA00058B10C9B23F07F43034413F8013CC1E7A5
:10EFB0000122DEE781460446DEE70446DCE700BFC7
:10EFC000F4D905002DE9F04F0C46A7B00646674975
:10EFD000204624F0B5F998B96549204624F0B0F9E7
:10EFE00050BB6449204624F0ABF9054638BB2246A5
:10EFF000614901201EF00AFF284627B0BDE8F08FC6
:10F000004FF0720A5D4900201CF0FEFF0546002803
:10F01000F2D01C220021304624F0A1FA0DF11C0888
:10F0200001460646404627F0A7F91B214B1E18F85B
:10F0300003203AB10B4608E04FF0770AE2E74FF0C1
:10F04000610ADFE71946002BF0D126AAD3184C49F4
:10F0500005933246284601240EAE03F87C4C0DF190
:10F060002C0925F030FA039699E807008DE807008F
:10F0700098E80F0026F0F9FE0E9BBAF1770F0746CD
:10F0800023F07F4B09D100286ED02846FFF77EFC85
:10F090004FF0000B5F46002629E0BAF1610FFAD16C
:10F0A000002F61D007EB0B0313F8013CFF2B01D0BD
:10F0B000FF2C45D10026ABEB0608B8F1000F16DD9A
:10F0C000B8F1400FA8BF4FF040084246F11916A80A
:10F0D0002BF04CFE16AA002312F8011BFF2941D089
:10F0E00001334345F8D100221E44002AE3D02046D4
:10F0F00023F07CFD23490246284625F0E4F93046FA
:10F1000023F074FD20490246284625F0DCF93846F4
:10F1100023F06CFD1D490246284625F0D4F95846D7
:10F1200023F064FD1A490246284625F0CCF95046E2
:10F1300023F05CFD17490246284625F0C4F95BE739
:10F14000059B013403F87C4C039699E807008DE891
:10F15000070098E80F0026F088FE0E9B074623F074
:10F160007F4B9DE70122BFE73E46C0E715570600EB
:10F1700017EC0500351F0600CDE50500DDE50500AF
:10F18000F4D90500E9E50500EFE50500F6E5050021
:10F1900013E605003BF4050010B58CB005AC014644
:10F1A000204627F0E9F80CAB13E907008DE80700CB
:10F1B00094E80F0026F04BFF0CB010BDF1F764BDD2
:10F1C00026F0D0BD70B5002290B006460846114624
:10F1D00008F00CFC09AC05463146204627F0CCF877
:10F1E0000023CDE90533CDE9035310AB13E9070044
:10F1F0008DE8070094E80F0026F06AFF04462846D1
:10F2000023F008FE204610B070BD2DE9F041804685
:10F2100090B008460C4617461E4622F0ACFE10B3CE
:10F2200000221146204608F0E1FB0026054637463D
:10F2300009AC4146204627F09FF80023CDE903534F
:10F24000CDE9057610AB13E907008DE8070094E8D7
:10F250000F0026F03DFF0446284623F0DBFD204644
:10F2600010B0BDE8F081204622F000FC0546DFE743
:10F2700030B58FB007AC01460025204627F07CF85A
:10F28000CDE903550EAB13E907008DE8070094E8BC
:10F290000F0026F031FE044638B1294624F0C3FAA7
:10F2A0000546204623F0B6FD2C4620460FB030BD63
:10F2B00070B58EB007AC16460D460146204627F0C5
:10F2C0005BF8CDE903560EAB13E907008DE80700A4
:10F2D00094E80F0026F010FE0EB070BD70B58EB031
:10F2E00007AC0E460146204627F046F80023CDE93C
:10F2F00003330EAB13E907008DE8070094E80F0015
:10F3000026F0FAFD054668B104F040FB04462846A5
:10F3100023F080FD1EB11DF037FA23F07BFD20465F
:10F320000EB070BD0446FAE74FF4D82026F0F0BFC7
:10F3300013B50C4619F058FE8DF80700093804285B
:10F3400005D80DF107020349204622F069FA02B000
:10F3500010BD00BF59F302000B78C1B2184619F076
:10F360007FBC00002DE9F04389B0984605460E4663
:10F37000174619F039FEA0F10903DBB2042B04464D
:10F380002ED80D280FD1274BDB7863B94FF0FF3211
:10F390004FF41651CDE9041204A8234A06928DF8C1
:10F3A0001C30F6F705FB8DF80040204C1FB13046AD
:10F3B00025F090FD06466A462146304622F030FA96
:10F3C00017B1304623F026FDB8F1000F05D069468D
:10F3D0000D20A04769460A20A04709B0BDE8F08388
:10F3E0000028FAD102461249284625F099F822460B
:10F3F00081461049284625F093F804AD0246494657
:10F400000446284618F0BAFE204623F003FD48467D
:10F4100023F000FD95E80F006C4607C42370064CEE
:10F42000C4E700BF99C20020080001007D9C0400D1
:10F430006ADB05003FDE0500FD91040000231A464B
:10F44000FFF790BF01231A46FFF78CBF002301226C
:10F45000FFF788BF2DE9FF47044619F0C5FD0022DC
:10F4600005464049204625F05BF8002207463E4904
:10F47000204625F055F8A5F109068246002F4CD00C
:10F4800001463A46684618F079FE9DF80600FF28C6
:10F4900002D0002112F008F89DF80700FF2802D0E2
:10F4A000002112F001F89DF80400FF2802D000218D
:10F4B00011F0FAFF9DF80500FF2802D0002111F09D
:10F4C000F3FFF3B2042B28D900222849204625F067
:10F4D00027F810B325F06CFB5FFA80F80021404656
:10F4E00011F056FC002018F0DDFD8146A8B1414620
:10F4F00023F06FFD804618B10146484625F062FBB7
:10F50000484623F06DFE20B9194B1A49586825F07A
:10F5100009FC4946404624F0F0FC5146384624F0A8
:10F52000ECFC1149204625F0FDFBF6B20D492046C2
:10F5300025F0F8FB042E11D80D2D0AD10E4BDB78E7
:10F540000BB111F01BFAFF220021284619F0D6FE5C
:10F5500004E0A5F10C03DBB2012BF4D904B0BDE843
:10F56000F08700BF3FDE05006ADB05003AE50500D5
:10F57000482E00203FE5050099C20020F0B585B077
:10F5800005460F46144619F02FFD064684B922465B
:10F590005249284624F0C4FF0446224639466846AC
:10F5A00018F0ECFD58B9204623F034FC05B0F0BD4E
:10F5B000B4F80B3003F50073A4F80B30EDE70098B6
:10F5C00023F014FB46490246284624F07CFF7CB118
:10F5D00022464249284624F076FFA6F10903DBB211
:10F5E000042B0AD80D2EE1D16846F6F7E1F9DDE7E4
:10F5F0003A49284625F096FBEFE7002ED6D19DF834
:10F600000500FF2807D0012111F04EFF01219DF8D0
:10F6100005001AF091FA9DF80400FF280BD005218F
:10F6200011F042FF602023F0A9F9044660B92D498A
:10F6300001201EF0EBFB9DF80630FF2BB6D02A49C7
:10F6400001201EF0E3FBB1E702462849284624F0DA
:10F650003AFF204622F0F6FC002680F8406004467F
:10F6600011F0C2FC009B9DF80A2084F85860C4E9A0
:10F6700014369DF8083013449DF80920B24218BF93
:10F680000133C4E9120184F8593001219DF80400C6
:10F6900011F07EFB0446C8B123F0A8FA14490246D3
:10F6A000284624F010FF012018F0FCFC0646002834
:10F6B000C1D02A46214624F076FE304623F0AAFB2C
:10F6C000013C0C4B0C4A43F82420B4E79DF804207D
:10F6D0000A4901201EF09AFBADE700BF3FDE05009E
:10F6E0006ADB0500B5E4050012E50500DBE4050072
:10F6F0003AE5050010C30020C1800400E3E40500E2
:10F7000010B50C4619F070FCA0F10903DBB2042B14
:10F7100004D82146BDE810401AF0A2BC02490120DD
:10F72000BDE810401EF072BB8AE405002DE9F74FDA
:10F730009846012313600D6907468A4616460DB1A7
:10F740000B68ED5C38782E2800F0FA805B2836D103
:10F75000012388F8093097F801B0BBF15E0F02D1A0
:10F760003368013333604FF0000907E02E2C19D1C4
:10F770002E2D08BF49F00109013333603368FC5C6A
:10F78000F818002C00F0DE805D2CEFD101333360DF
:10F79000002388F80930BBF15E0F14BF484689F09A
:10F7A000010019E0434601AA5146FFF7BFFF336845
:10F7B000019A49EA00095FFA89F91344DDE75C28F8
:10F7C0006CD1022333607878642808D1A5F1300029
:10F7D00009288CBF0020012003B0BDE8F08F442829
:10F7E00006D1A5F13000092894BF00200120F3E7DD
:10F7F00066286ED062286ED06E286ED072286ED0C9
:10F80000732805D1284603B0BDE8F04F1DF07ABA41
:10F81000532806D128461DF075FA80F00100C0B2C9
:10F82000DAE774285DD076285DD077280ED1A5F16F
:10F830003003092B40F2848028461DF057FA002837
:10F840007ED15F2D14BF00200120C5E757280CD1C1
:10F85000A5F13003092B12D928461DF047FA70B9DB
:10F86000B5F15F0018BF0120B6E730283DD0A0F108
:10F870003103082B05D8364901201EF0C7FA0020B5
:10F88000AAE778280AD1BB7843B1FB7833B10423C7
:10F890003360F978B8781DF018FAC0B298F80930DA
:10F8A0002BB33368FA5C2D2A21D13B445B785D2B66
:10F8B0001DD0A8F80A00306801303060434601AA24
:10F8C00051463844FFF732FF3368019A13443360DE
:10F8D00082E70C20E2E70820E0E70A20DEE70D20BF
:10F8E000DCE70920DAE70B20D8E70020D6E798F814
:10F8F000082062B1A5F14103192B98BF2035A0F172
:10F90000410398BFEDB2192B9CBF2030C0B2B8F9AB
:10F910000A30B3F5807F11D0DBB22AB1A3F14102E6
:10F92000192A9CBF2033DBB24FF480729D42A8F8A5
:10F930000A20A4D38542A2D8984255E7854281E7A0
:10F94000012049E7012003491EF060FA204643E701
:10F95000FDE705001AE8050082B02DE9F047ACB0DC
:10F960000C4634A9054681E80C001CF071FF30B14B
:10F97000002630462CB0BDE8F04702B070472B7827
:10F980000BB17C2B43D1582234A90DEB02002BF094
:10F99000EDF9DDE93457DDF8DC9023F00FF9236849
:10F9A000A2681A440646D21B3946284623F0D7FDE2
:10F9B000002104460246304624F0F5FC204623F0A0
:10F9C00029FA0DF1680800244C450DDB384623F078
:10F9D0000DF970490246304624F075FD2A466E49FD
:10F9E000304624F059FDC4E758F8041BD8F820200D
:10F9F0002846521A23F0B3FD0134824602462146BE
:10FA0000304624F0D0FC504623F004FADCE75E2BAD
:10FA100009D12368A268D342AAD11EF0B9FB0028FD
:10FA2000A6D0013507E0242B1DD1D4E900329A423B
:10FA300005F101050CD8502236A968462BF096F93D
:10FA400034AB0CCB21462846FFF786FF064690E7ED
:10FA50004C2237A968462BF089F934AB0ECB2846E7
:10FA600000F026FAF2E7282B0FD1379B2168A26815
:10FA700034A80A44191D082B40F8212000EB83010B
:10FA80004A63CADC01333793C7E7292B0AD1379B76
:10FA9000002BC2DD34AA02EB83032168A2680A446A
:10FAA0001A63BAE734AB15AA21462846FFF73EFE93
:10FAB000159FEB5DA3F12A02012A804605EB07069C
:10FAC0004ED801372F4450B92B2B08D14C2237A9DF
:10FAD00068462BF04BF934AB0ECB3846C0E72146D5
:10FAE00016A81DF03EFD502236A968462BF03EF9BF
:10FAF00034AB0CCB16A93846FFF72EFF06461998F3
:10FB000023F088F9D4E900239A42BFF432AFB8F168
:10FB1000000F3FF42EAF20461DF09DFA34AB15AA1E
:10FB200021462846FFF702FE2146804616A81DF012
:10FB300018FD502236A968462BF018F934AB0CCBCF
:10FB400016A93846FFF708FF8146199823F062F995
:10FB5000B9F1000FD6D0304623F05CF94E46D1E71C
:10FB6000D4E900239A420BD250B120461DF073FA1B
:10FB70001EF00EFB00283FF4FBAE159B1D445AE718
:10FB80004C2237A968462BF0F1F834AB0ECB304647
:10FB900066E700BF3CE8050042E805002DE9F047B4
:10FBA000B4B00646084614AF25F094F90022544933
:10FBB0008046304624F0B4FC24F0FAFF00220546CB
:10FBC0005049304624F0ACFC044622F0F6FA48B91D
:10FBD0002146404624F091F9002420468037BD4656
:10FBE000BDE8F087404623F094FDA842F0D32046BC
:10FBF00023F08FFD00F1080323F00703ADEB030DA5
:10FC00000DF1500A421C5146204625F0E3FA2046E9
:10FC100023F000F969213046FDF7BEFB4FF48072F6
:10FC2000002387F830007A8641462A46384687F80E
:10FC300031307B63C7F828801DF067FD394607F136
:10FC400014001DF08EFC502207F130016846FD6261
:10FC50002BF08CF807F1280999E80C0007F1140142
:10FC60005046FFF779FE0446386A23F0D3F8384649
:10FC70001DF0F1F92CB9D7E900239A4205F10105ED
:10FC800014D3F86823F0C6F8404623F0C3F8D4B97B
:10FC9000022022F01BFF00250446284622F0A6FF82
:10FCA00017490246304624F00EFC96E7394607F124
:10FCB00014001DF056FC502207F130016846FD6229
:10FCC0002BF054F8C8E767213046FDF765FBA0B17B
:10FCD0000021204624F0BAF9002280460A49204635
:10FCE00024F01EFC24F064FF0546404623F011FD7D
:10FCF0000544404623F08EF8CFE70546CDE700BF28
:10FD00007AE4050073E405003CE805002DE9F84FAE
:10FD100004460D4622F051FA20B94FF00008404643
:10FD2000BDE8F88F22F04AFF80460028F5D01DB9C3
:10FD3000214624F0EFFAF2E75149284624F00EFC60
:10FD400000285FD0002022F051FF4E49024628468D
:10FD500024F0B9FB21462846FFF720FF002706467E
:10FD600026B1304622F0C8F88146D0B1304623F0A3
:10FD700051F8002022F03AFF42490246284624F07A
:10FD8000A2FB204623F0C5FCB842C8DB39466FF021
:10FD90000042204623F0E3FB0146404624F0D3FA1C
:10FDA000BDE74946304624F051F94A463649824675
:10FDB000304624F0B5FB24F0FBFE8146504623F08C
:10FDC000A8FC8346504623F025F8A9EB07023946E4
:10FDD000204623F0C4FB0146404624F0B4FA0BEB66
:10FDE0000907304623F016F8384622F0FFFE254971
:10FDF0000246284624F067FB21462846FFF7CEFE40
:10FE00000646ADE7284625F065F8814688B123F01F
:10FE100080FC0746204623F07CFC002600F1010B05
:10FE2000ABEB070A3546554522DC7FB925BB0135CA
:10FE3000F9E70746EEE75D4612E00146404624F04A
:10FE400069FA304622F0E6FFEE19F0E75545F2D0A8
:10FE500001232A4649462046F0F756FC0028E6D101
:10FE6000AA1B3146204623F07AFB06460028E4D13F
:10FE7000484622F0CFFF52E75545F1D1F8E700BFE1
:10FE80006CE405007AE405003CE8050038B5FFF7AE
:10FE900085FE054650B122F02FF880F00100C4B273
:10FEA000284622F0B7FF04F0010038BD0446F7E70A
:10FEB00084B0F0B59BB021AE054686E80E001EF07A
:10FEC00067F968B9044620461BB0BDE8F04004B0AD
:10FED00070475C2C03D16C78002CF4D03D46013582
:10FEE0002C78002CEFD07C2C05F10107F1D1DDE955
:10FEF000211215A81DF009FC23A9502268462AF0FA
:10FF000035FF96E80C0015A93846FFF725FD044695
:10FF1000189822F07FFFD6E737B5054601910B48C8
:10FF200048F2080122F040FE044660B12A46084922
:10FF300024F0B2FA2846012301AA214618F0C0FF96
:10FF4000204622F067FF03B030BD00BFFF0303006F
:10FF5000FAD105002DE9F743054608460F469046BD
:10FF600022F024F838B93A46254903201DF04EFF07
:10FF700003B0BDE8F083B8F1000F0BD00022214997
:10FF8000284624F02FFA0446E8B124F055F8044638
:10FF90001D4E01E01D4E444600223146284624F005
:10FFA000BFFA814688B93A463146284624F074FAA9
:10FFB000B8F1000FDCD028462146FFF7ADFF204600
:10FFC00022F028FFD4E78046E2E721F0CBFF38B1EA
:10FFD0003946484624F09EF9484622F01BFFE7E7E1
:10FFE00002216846CDE9009724F0CAF93146074658
:10FFF0000246284624F050FA384622F00BFFEBE781
:020000023000CC
:100000001DDB050041DB050013DB050018DB0500E7
:1000100010B500220446FFF79DFF2046BDE81040C2
:10002000FDF7F0BA38B5154601220446FFF792FFF6
:1000300025B1002229462046FFF78CFF2046BDE867
:100040003840FDF7DFBA00002DE9F74F054622F0F2
:10005000E1F8044640B92A46344903201DF0D6FE93
:10006000204603B0BDE8F08F314900201BF0CCFFE3
:1000700004460028F4D048F208012E4822F094FDEE
:100080008146D8B122462C4924F006FA22F096FD8A
:100090002946824601A81CF04BFF002635460198F0
:1000A00080B9A81B22F0A2FD24490246204624F074
:1000B0000AFA52462249204624F005FA484622F020
:1000C000A9FECDE723F0B4FF8046FDF78FF930B3EA
:1000D00048F260011B4822F067FD0746284622F0DF
:1000E00085FD002102468346384624F0B8FC584678
:1000F00022F090FE22461049384624F0CDF93946C8
:100100004A464046FFF78EFF394623F0F6FE40464A
:1001100022F080FE01A801351CF0F9FEBFE742463F
:100120002946504624F03FF90136F0E7D2DD0500BC
:1001300034E40500E5010300FAD1050029E40500D7
:100140002FE40500490103002DE9F0410F469046D8
:1001500013490022054624F0E3F924F029FD00228A
:1001600004461049284624F0DBF90646B0B1424661
:100170003946013C24F017F9204622F037FD0849A2
:100180000246284624F09FF91CB931462846FFF75D
:10019000C3FE3046BDE8F04122F03CBEBDE8F08130
:1001A00029E405002FE4050037B5054601910B4809
:1001B00048F2080122F0F8FC044660B12A460849DA
:1001C00024F06AF92846012301AA214618F078FE96
:1001D000204622F01FFE03B030BD00BFF90303002C
:1001E000FAD1050038B500220D460949044624F02D
:1001F00097F958B122F00EFE2046054924F092FDF1
:1002000029462046BDE83840FFF7CEBF38BD00BFC5
:100210002FE405002DE9F04385B0064601914149E0
:10022000144624F07FFD4049304624F07BFD002237
:100230003E49304624F074F93C490546304624F0E6
:1002400071FD204621F08EFE074660B3214603A8CB
:100250001CF06EFE0024039878B91CF095FA8046D5
:1002600058B301462846FFF79FFF2A4621464046DD
:1002700023F036FE05B0BDE8F08323F0D9FE01ABD4
:100280000122314681461AF057FA804617B922F00A
:10029000C1FDA046484622F0BDFD03A81CF037FE74
:1002A00000274446D7E7002CD7D0204601AB0122D7
:1002B00031461AF041FA0446CFE74DB32046FDF728
:1002C00095F850B348F20801194822F06DFC48F245
:1002D00008010646174822F067FC0746A6B198B108
:1002E0002A461549304624F0D7F82A46124938469E
:1002F00024F0D2F8012231462046FFF72BFE424679
:1003000039462046FFF726FE3946304623F0F5FDF4
:100310002946204623F0F1FDACE721462846FFF7A9
:10032000FBFDF5E713DB050018DB0500EB240600F9
:1003300019FF0200A9010300FAD10500294B2DE99C
:10034000F047B2F10009284E08BF1E460D460022B4
:100350003146804624F0E4F8044670BB0246234947
:10036000DFF888A0404624F0DBF804464CB9B9F128
:10037000000F25D12A461E490120BDE8F0471DF097
:1003800045BD00223146204624F0CAF80746024601
:1003900048B129462046FFF73DFF21463846BDE8D3
:1003A000F04723F0AABD5146204624F0B9F807468D
:1003B000204622F02FFD3C46D8E7B9F1000F05D0CA
:1003C0002A460C49404624F067F84CB14046224684
:1003D0002946FFF71FFF2046BDE8F04722F01ABD6F
:1003E000BDE8F08718DB050013DB0500EB240600F1
:1003F0004ADB050041DB05000022FFF79FBF012219
:10040000FFF79CBF2DE9F74F10F0EEFD8946074638
:1004100022F076F8834610F0E7FD80468A4622F007
:10042000D0FB0446002800F0A680564B5649586879
:10043000002224F075F80546002800F0A08022F084
:10044000ABFE0646284622F0E5FC002501230D21DF
:100450004E485A1E01FB0202B2F80B0080060FD074
:1004600010460193009221F0E3FD0135019B0D211F
:1004700030B1009A12680C32B2FBF1F21344154409
:10048000013340F6C4229342E2D9B018AB1B401BA3
:10049000009322F0ABFB3E490246204624F013F8BD
:1004A000009B184622F0A2FB3A490246204624F05F
:1004B0000AF840F6C42022F099FB3749024620464C
:1004C00024F001F8304622F091FB2F4902462046E5
:1004D00023F0F9FF584622F089FB304902462046B6
:1004E00023F0F1FFB8EB07006AEB090129F0FCFEED
:1004F00000222B4B29F026FF2A4B002229F022FF55
:1005000041EC100B22F060FB27490246204623F005
:10051000DAFF0D2022F06AFB24490246204623F030
:10052000D2FF234822F062FB22490246204623F0F4
:10053000CAFF002022F05AFB1F490246204623F042
:10054000C2FF1E4822F052FB1D490246204623F0FE
:10055000BAFF4FF4D82022F049FB1A490246204640
:1005600023F0B1FF4FF4002022F040FB1649024671
:10057000204623F0A8FF204603B0BDE8F08F0646D2
:1005800063E700BF482E0020B1E30500682E00207D
:10059000B9E30500BEE30500C4E30500CAE30500B6
:1005A00000408F400000B03ECDE30500D4E30500DD
:1005B00088D00020DEE30500EEE30500CC5F0600F6
:1005C000FAE305000BE405001CE405000000000050
:1005D00010B522F0F6FA0446374823F085FB374978
:1005E0000246204623F06FFF354823F07DFB354956
:1005F0000246204623F067FF334823F075FB33495A
:100600000246204623F05FFF4FF4002022F0EEFA6E
:100610002F490246204623F056FF2E4B1878022819
:1006200003D003283AD001283DD122F0DFFA024658
:100630002949204623F047FF4FF4204022F0D6FA04
:1006400026490246204623F03EFF4FF4803022F038
:10065000CDFA23490246204623F035FF04F0BAF9CB
:1006600020490246204623F02EFF03F04DF81E4994
:100670000246204623F027FF1C4823F035FB1C4987
:100680000246204623F01FFF1A4822F0AFFA1A490B
:100690000246204623F017FF204610BD9FED040BB5
:1006A00022F092FAC3E70020C1E700BFAFF3008059
:1006B000CDCCCCCCCCCC004011E3050042E305000E
:1006C00019E3050022E305002DE3050034E30500EE
:1006D0003AE3050070C3002040E305004AE305004B
:1006E00009FC050052E3050059E3050061E305003C
:1006F000A3E30500A82D0020ABE3050038B50849A9
:10070000054600201BF080FC044638B1284622F044
:1007100075FA04490246204623F0D5FE204638BD2E
:10072000CEE1050078E705002DE9F8430D460321E9
:10073000074610F0B9FE002401264FF08008A146BC
:1007400015F1FF3502D22046BDE8F88388F3118801
:100750000021384610F02EFC0320F1F709FA0121A0
:10076000384610F027FC0A20F1F702FA384610F05C
:100770000DFC00B1344389F311883520F1F7F8F905
:100780007600DDE710B50321044610F08DFE002150
:10079000204610F00FFC4FF4FA70F1F7E9F901214F
:1007A000204610F007FC5020F1F7E2F9204610F047
:1007B000EDFB04464FF4D270F1F7DAF984F0010052
:1007C000C0B210BD08B50022034923F0A9FEBDE860
:1007D000084018F0E1BC00BF78E705002DE9F04FB4
:1007E0008BB00C46FFF7EEFF064618F0F7FC28B971
:1007F0004FF0000840460BB0BDE8F08F22F0DEF964
:1008000080460028F4D0631EFF2B28BFF024224628
:10081000E317CDE900234FF000093046FFF7B2FFA0
:100820000028E7D0DDE9002308213046FDF72AFD46
:1008300001240025AA46274601213046FFF774FF10
:1008400001215FFA80FB3046FFF76EFFBBF1010F1D
:10085000C0B22BD101283AD1402FCBDD9DF80C300E
:10086000002BC7D005AC0DF10C090025A34619F8E3
:10087000017B38091BF0FEFF207007F00F001BF012
:10088000F9FF0135082D607004F10204EFD1002357
:1008900058468DF8243023F027FA0146404623F0CD
:1008A00052FDD146BAF1000FA4D0B6E70AAB2B44F3
:1008B000834513F81C3C2DD14F4524DA1C4214BF4C
:1008C0004FF0010B4FF0000BBBF1000F21D00AAB32
:1008D0002B444FF0010B13F81C3C23430AAA2A4473
:1008E000012102F81C3C30465A4600236400FDF703
:1008F000C9FC14F0FF0404BF01350124072D07F1E2
:10090000010799DDA8E70CBF4FF0010B4FF0000B7A
:10091000DAE7BA4623EA0403E0E770B58AB00C468A
:10092000FFF750FF064618F059FC68B3204621F047
:1009300063FB18B3204623F099FB014605460120CE
:1009400022F08EFA044650B10146002268461DF09E
:1009500059FC15F1FF3505D268461CF06FFA2046A8
:100960000AB070BD08213046FFF7DEFEC1B268460E
:100970001CF02FFD68461CF094FBEAE70821304686
:10098000FFF7D2FE22F032F90446E8E737B50D460C
:100990001446FFF717FF8DF8070018F01FFC80B111
:1009A0000DF107020C49284620F03AFF9DF8070098
:1009B0004CB1012110F0FEFA01219DF8070010F062
:1009C00073FD03B030BD042110F06EFD01219DF8D0
:1009D000070010F0EFFAF4E713E3020010B5FFF799
:1009E000F1FE044618F0FAFB38B12046CC22002371
:1009F0000821BDE81040FDF745BC10BD2DE9F041D0
:100A000086B00C46FFF7DEFE054618F0E7FB40B166
:100A1000204621F0D2FB38B92246264903201DF09A
:100A2000F5F906B0BDE8F081204622F072FE1028EC
:100A3000F2D12846FFF7A6FE2146002201A81CF0AD
:100A400064FE002427462646A04601A81CF056FD59
:100A50008DF8000001A81CF051FD00231A468DF806
:100A60000100102168468DF802801CF056F9A4F1AF
:100A70002002C4F12003A14000FA02F220FA03F39D
:100A80001143A04008341943402C47EA000746EAC6
:100A90000106DAD1049822F0BDF928465522002338
:100AA0000821FDF7EFFB3A46334621462846FDF77D
:100AB000E9FBB6E7D6E1050010B5FFF783FE044673
:100AC00018F08CFB20B12046BDE81040FFF75ABE5D
:100AD00010BD00002DE9F74305460F46914621F071
:100AE00065FA044640B92A46574903201DF08EF99D
:100AF000204603B0BDE8F083284621F006FA60B333
:100B0000A988286822F050F804460028F0D0294629
:100B100068461CF00DFA009D7DB3B5F80B3003F567
:100B20000073A5F80B30284623F082FA8046284649
:100B300021F099FBD8B1B8F1000F2AD00121284645
:100B400023F054FD064630B10146204623F004FB55
:100B5000304622F05FF901260AE0284621F01CFA0F
:100B6000002814BF0820072021F0B0FFCCE706467C
:100B70004146284623F0C1F96EB9B9F1000F0ED1F4
:100B8000009D002D45D13A463049204623F084FC93
:100B9000AEE74646ECE768461CF0B9F9BBE74946C4
:100BA00001A81CF0C5F901980028E9D023F040FA0B
:100BB000009D064665B1B5F80B3003F50073A5F846
:100BC0000B30284621F04FFB40B9284622F022F98D
:100BD00032460021204623F042FF13E0012200218B
:100BE000284623F0BDFE3146804623F0C7F8414633
:100BF000204623F0B1FA2846414623F07EF96846A4
:100C00001CF085F9304622F005F901A81CF07FF9A7
:100C1000C9E7B5F80B30012203F50073A5F80B30D6
:100C20001146284623F09CFE064630B10146204678
:100C300023F092FA304622F0EDF8284622F0EAF846
:100C400068461CF064F99BE71FDC0500FAD105003B
:100C50002DE9F04F8FB0814602AF10468A46164606
:100C600021F0D8FA0446002856D0304622F073FD11
:100C7000B0F5807F044680460AD902462B49012000
:100C80001DF0C4F8002420463437BD46BDE8F08F7F
:100C90008300DA1D22F00702ADEB020D02AD2A46F9
:100CA0002B440021934219D101223146381D1DF0F9
:100CB000D8FA381D1CF0F4F898B9381D1CF0C4F8A7
:100CC00000231946CDE90085524648461FF07EFFB5
:100CD00029460446404623F0E6F8D4E742F8041BD0
:100CE000E0E7381D1CF085F8064621F069FB60B18D
:100CF000304623F0BBF9B0F1000B06DB5C4504DDA8
:100D0000381D1CF0BEFC45F82B00304622F082F85E
:100D1000381D1CF0E0F9CCE72EB132460449012021
:100D20001DF074F8AFE7B0463546C9E79BDB050018
:100D3000E4DB05002DE9F34704460D4621F036F9C2
:100D400030B9444903201DF061F802B0BDE8F087D6
:100D5000284621F02BF90028F3D0204621F0D5F8C1
:100D60000646284621F0D1F886420AD0284621F0CE
:100D7000CCF8B4F80B30002842D043F04003A4F87C
:100D80000B30204621F008F90646284621F004F9E8
:100D900086420BD0284621F0FFF8B4F80B3023F040
:100DA0003F0380B343F00803A4F80B3000222A4924
:100DB000DFF8A490DFF8A4A0204623F013FB002264
:100DC00026490746204623F00DFB0646204623F021
:100DD000C4FF294601A81CF0ABF8019DB5B91FB1AD
:100DE0003946204623F0B8F9384622F013F81EB1F0
:100DF0003146204623F0B0F9304622F00BF8A4E744
:100E000023F04003BBE743F00703CDE7B5F80B3011
:100E100003F5007301A8A5F80B301CF078F84946DB
:100E2000284622F08DFA88B95146284622F088FAE1
:100E300060B90121284623F0D9FB804630B1014634
:100E4000204623F089F9404621F0E4FF284621F0AE
:100E5000E1FFC2E756DC050074DC0500382106001E
:100E60002DE9F74305460F46144621F0C9FA30B97B
:100E7000354903201CF0CAFF03B0BDE8F0833846B3
:100E800021F09BF908B93149F3E7204621F08EF8AB
:100E900028B9204621F091F908B92D49E9E73946EA
:100EA0002C4822F06DFB80460028E5D00146012247
:100EB000284623F0C8FC0646404621F0ABFF3046EA
:100EC00023F0B6F8804620BB2146304622F056FF7C
:100ED0003146404623F011F81F49384622F030FAD7
